:10000000000002203982000061820000638200004B
:100010006582000067820000698200000000000025
:100020000000000000000000000000006B820000E3
:100030006D820000000000006F82000071820000ED
:100040007382000049580000FD85000071810000A6
:1000500065810000738200007382000073820000DB
:100060001539000073820000738200007382000063
:1000700073820000738200007382000073820000AC
:10008000738200008186000073820000738200008A
:10009000738200007382000073820000738200008C
:1000A000738200007382000073820000738200007C
:1000B0007382000073820000000000000000000056
:1000C000738200007382000073820000738200005C
:1000D000738200007382000073820000738200004C
:1000E000738200000000000000000000000000001B
:1000F0000000000073820000000000007382000016
:1001000000000000000000000000000000000000EF
:1001100000000000000000000000000000000000DF
:1001200000000000000000000000000000000000CF
:1001300000000000000000000000000000000000BF
:1001400000000000000000000000000000000000AF
:10015000000000000000000000000000000000009F
:10016000000000000000000000000000000000008F
:10017000000000000000000000000000000000007F
:10018000000000000000000000000000000000006F
:10019000000000000000000000000000000000005F
:1001A000000000000000000000000000000000004F
:1001B000000000000000000000000000000000003F
:1001C000000000000000000000000000000000002F
:1001D000000000000000000000000000000000001F
:1001E000000000000000000000000000000000000F
:1001F00000000000000000000000000000000000FF
:1002000010B5054C237833B9044B13B10448AFF350
:1002100000800123237010BD440200200000000074
:10022000BCDC000008B5034B1BB103490348AFF326
:10023000008008BD0000000048020020BCDC000077
:10024000154B002B08BF134B9D46A3F5803A0021A8
:100250008B460F461348144A121A0AF0A5FC0F4B9E
:10026000002B00D098470E4B002B00D09847002061
:10027000002104000D000D48002802D00C48AFF307
:1002800000800AF049FC2000290008F00FFA0AF06B
:100290001DFC00BF0000080000000220000000005C
:1002A00000000000440200209490012000000000A3
:1002B0000000000010F0010310D104280CD90368DD
:1002C000C3F30F1343B1013B9B001A1DC1180979F9
:1002D00011B101339342F9D1184670470023FBE76F
:1002E000037883B11A0601D40130704703F0C003CC
:1002F000C02B08BF0130024610460132037803F0DC
:10030000C003802BF8D0704708B5002103780BB9E3
:10031000084608BDFFF7E4FF0131F7E738B50022D2
:1003200004460D46411C092003F028FE40B163003D
:10033000024643F0010342F8043F0023A34200DBDE
:1003400038BD55F8231042F8041F0133F6E70128A1
:1003500038B504DC1C20BDE8384001F01FBA0D6838
:10036000EA0701D41120F6E74868C30706D4042839
:1003700004D9036803F00F03042B01D00E20EAE731
:1003800003F060FC6D10002D044603DDFFF7BCFF99
:10039000A84206DA1220DEE72046FFF7A1FF013D62
:1003A0000446012DF8D120787F2808DDDF280ADCFB
:1003B0006378800100F4F86003F03F0318434000C5
:1003C00040F0010038BDEF280ADC637800039B0190
:1003D00080B203F47C630343A07800F03F00EDE7B4
:1003E000F72810DC637880041B0303F47C3300F4EB
:1003F000E0101843E37803F03F030343A078800143
:1004000000F47C60DAE74FF0FF30D8E7486838B591
:10041000C3070D4606D4042804D9036803F00F026D
:10042000092A04D00B20BDE8384001F0B7B9446870
:10043000C3F30F1364105A1EA2420BD8032194FB7E
:10044000F1F16429A8BF64210329ACBF5918D91C54
:1004500003F0D0FD0368C3F30F13013B9C4208D2A5
:10046000A31C013464002A6840F8232044F00104EE
:100470004460002038BD01282DE9F84304DC1C202D
:10048000BDE8F84301F08AB902284E680CD08C68A8
:10049000E70709D56410012CB8BF0124F50705D57D
:1004A0004FF0FF30BDE8F8830124F7E7042EF7D9B9
:1004B00033680D6803F00F02042A30D1E80706D430
:1004C000042D04D92B6803F00F03042B01D00E2058
:1004D000D6E73046FFF7EEFEA042E1DB304603F000
:1004E000B1FB0646284603F0ADFB03780146002B1E
:1004F000D6D0601E30440AF026FF01460028CFD037
:10050000012433780BB18E4203D3640044F0010020
:10051000C8E73046FFF7E4FE01340646F1E7092A52
:1005200038D177687F10BC42BADCE90729D4042DA2
:1005300027D92B6803F00F03042B22D1284603F0A0
:1005400081FB804604F1010956F82900854203D158
:10055000600040F00100A5E7C2070ED404280CD9C2
:10056000036803F00F03042B07D103F06BFB014674
:1005700040460AF0AFFE0028C7D0B9454C46E1DD41
:100580008EE7631C56F82320AA42BED0BB421C460D
:10059000F7DD85E7032A83D1C3F30F17C3F3417354
:1005A000C3EB8707BC423FF77BAFEB0728D4042D92
:1005B00026D9286800F00F03032B17D1C0F30F13BF
:1005C000C0F3417005F10408C0EB83003F1A013C01
:1005D00040440336BC423FF763AF3219434683427F
:1005E00019460FD315D1601C4000B2E7042B07D188
:1005F000284603F027FB80462846FFF75BFEE5E729
:100600000F203DE712F8015F09788D4203F10103E5
:10061000E5D00134DEE7000001282DE9F0470E4661
:1006200004DC1C20BDE8F04701F0B8B80868C20738
:1006300006D4042804D9036803F00F03042B01D067
:100640000E20EFE74B6813F00109F9D1042BF7D91D
:100650001B6803F00F03042BF2D103F0F3FA0446F6
:10066000706803F0EFFA82460AF03EFE804670B9E9
:100670002046FFF749FE05460122A918092003F08C
:100680007DFC354F386098B90020BDE8F0875146B1
:1006900020460AF058FE231A5D425D4120466F1C39
:1006A0000028E9D0514640440AF04DFE3D46F6E7A9
:1006B0006B0043F001034360B8F1000F19D12046ED
:1006C000FFF70EFE4D45064601DC3868DDE7311BBD
:1006D000204603F0D4FC0028D6D009F102023B6882
:1006E00043F822003046FFF7FBFD09F101093446CB
:1006F000E8E7012D02D133688360C6E75146204602
:100700000AF021FE01268146B9F1000F14D0B5424E
:10071000DBDBA9EB0401204603F0B1FC0028B3D0D9
:100720003B68013609EB080443F826005146204691
:100730000AF009FE8146E7E7B542C6DB20460AF02B
:10074000D3FD0146204603F09AFC00289CD00136D8
:100750003B6843F82600B8E7546D012008B503F064
:1007600055FA400040F0010008BDC30711D4042829
:100770000FD9026802F00F03032B0AD101F0030323
:10078000C3F104035B0703F0C04322F0C0421343EC
:1007900003607047002838B504DC1C20BDE83840F1
:1007A00000F0FCBF0C68E50701D40D20F6E7012836
:1007B0001CD04B68DA07F8D55B10FF2B01D913204A
:1007C000ECE71A0442EA03621A4342EA0322641085
:1007D00024EAE474E11C8910032003F0CFFB0546F2
:1007E00010B12146FFF7C1FF284638BD0022EEE7D1
:1007F00001282DE9F0470546884604DC1C20BDE8A9
:10080000F04700F0CBBF4C6814F0010701D10D2078
:10081000F5E7022802D08B68DA07F8D5D8F800602F
:10082000F30700F1A980042E40F2A680326864101C
:10083000012C02F00F03B8BF0124092B28D17668E0
:10084000022D4FEA660605D0D8F808305B109E42AC
:10085000A8BF1E46351B0135012225EAE575A918FA
:10086000092003F08BFB074648B16D00034645F0B5
:100870000105D8F8002043F8045FA64202DA3846A2
:10088000BDE8F087013452F8241043F8041FF4E760
:10089000042B43D1304603F0D5F9FFF735FD022D87
:1008A000824605D0D8F808305B109842A8BF9A4617
:1008B000A24504DA0020BDE8F04703F0D9BB30467A
:1008C00003F0C0F90546A74222DB304603F0BAF92F
:1008D000A94606462846FFF703FD0134A245054612
:1008E000F8DAA0EB0905284603F0C2FB074600280A
:1008F000C5D003F0A7F90446D8F8000003F0A2F928
:10090000A9EB060101442A4620460AF029F9B6E778
:100910002846FFF7E5FC01370546D4E7032B2BD12A
:10092000C2F30F13022DC2F34172C2EB830205D052
:10093000D8F808305B109A42A8BF1A46A24206DADD
:10094000002211460320BDE8F04703F017BB151B3A
:100950000423291D002291FBF3F1032003F00EFB79
:10096000074600288BD001352946FFF7FEFEE11C23
:100970002A4631440430C8E7212040E70028F8B572
:1009800004DC1C20BDE8F84000F008BF0C6814F03F
:10099000010711D06410FF2C01D91320F2E70022C7
:1009A0000121032003F0EAFA054618B10121FFF7FF
:1009B000DCFE04712846F8BD042CEED9256805F04C
:1009C0000F05042D19D12046FFF774FC3A46C11CCF
:1009D000064691FBF5F1032003F0D0FA0546002806
:1009E000E8D03146FFF7C1FE204603F02BF932462E
:1009F0000146281D0AF0B4F8DCE7092D1DD1666810
:100A000076100423F11C3A4691FBF3F1032003F026
:100A1000B5FA05460028CDD03146FFF7A6FE0434CE
:100A2000B742C7DA54F8043FDA0704D55B10FF2B4E
:100A3000B3D8EA1913710137F2E7032DADD125467A
:100A4000B8E77F2902DC017001307047B1F5006F13
:100A50000CDA03468A1162F03F0203F8022B01F020
:100A60003F0161F07F01417018467047B1F5803F4A
:100A70000FDA0B1363F01F030370C1F3851301F04A
:100A80003F0163F07F0361F07F01437081700330A9
:100A90007047B1F5883F0DDAF0230370902343705F
:100AA0008B1101F03F0163F07F0361F07F018370E0
:100AB000C1700430704700000028F7B50F4603DC12
:100AC0001C2000F06BFE0CE00A6812F001000AD056
:100AD0006C4651102046FFF7B4FF011B204603F07F
:100AE000CEFA044616E0042A3BD9136803F00F033C
:100AF000092B36D155681C496D100124AC420CDD20
:100B000003F0B6FA044628B13F6803F09BF80126CB
:100B1000AE421DDD204603B0F0BD013452F8243052
:100B200013F0010601D12720CBE75B107F2B09DDF5
:100B3000B3F5006F08DBB3F5803F07DB8B42D4BF12
:100B4000042600263044D9E70226FBE70326F9E70E
:100B5000013657F82610CB07E5D54910FFF771FF8E
:100B6000D6E70B20ADE700BFFF0F010010B510F076
:100B7000010402D04410204610BD042812D9026896
:100B800002F00F02042A07D103F05CF80A22214682
:100B9000BDE810400AF06CBC032A03D10A222146AA
:100BA0000430F5E70D2000F0F9FDE4E710B5044648
:100BB00011F0010011D104290ED90B6803F00F03C5
:100BC000042B09D1084603F03DF8014620460AF0FF
:100BD00081FBB0FA80F0400910BD0020FCE7000066
:100BE0000128F8B50D4604DC1C20BDE8F84000F0F3
:100BF000D5BD4E68F20706D4042E04D9336803F03D
:100C00000F02092A01D00B20EFE77468096864100D
:100C1000C3F30F13A34298BF03F1FF3411F0010790
:100C20000DD0481000283ADD844238DB06EB800303
:100C3000844218DD9A6843F8042F0130F8E71A4817
:100C4000FFF7B4FF40B10123BC4201DA0020F8BD38
:100C5000013746F82730F7E729681448FFF7A6FF61
:100C600050B1002CF2D00122631C013C944014438B
:100C700046F823207460E9E72868C30711D40428E4
:100C80000FD9036803F00F03042B0AD1FFF76EFF9F
:100C90000028C8D129680648FFF788FF08B112204C
:100CA000A3E71120A1E700BF67C200006BC20000EC
:100CB00070C20000002310B50B70C3070C4606D5A8
:100CC0000E4942102046BDE810400AF0C7BA28B9C4
:100CD0000B492046BDE810400AF0E0BA042801D1D3
:100CE0000849F6E709D9036803F00F03042B04D180
:100CF00002F0A8FF04490246E4E710BD34CE00002C
:100D000072C2000078C200007DC200002DE9F043ED
:100D100001288FB081460E4607DC1C2000F03EFD06
:100D2000054628460FB0BDE8F0830B6813F00104B8
:100D300040F0A180042B40F2D5801B6803F00F0324
:100D4000092B40D1274656F8273013F0010806D169
:100D5000042B04D9186800F00F00092801D02220C4
:100D6000DCE75B680137B94504EB6304EBD1012292
:100D7000A11803F003F9054608B90025D1E764007E
:100D800044F001044460424600F1080456F8221081
:100D90004B6808685B10C0F30F10984298BF00F1D1
:100DA000FF3304310020834207DC013223EAE3737E
:100DB000BA4204EB8304E9DBB3E751F804CF44F80B
:100DC00020C00130EFE7032B40F08C80274656F817
:100DD000270010F00108C2D10428C0D9036803F02D
:100DE0000F02032A38D1C3F30F12C3F34173C3EBCD
:100DF00082031C440137B945E9D10423E11C0022D8
:100E000091FBF3F1032003F0B9F805460028B4D0B4
:100E10002146FFF7AAFC00F1040956F82840E10733
:100E200020D4042C1ED9206800F00F03032B19D105
:100E3000C0F30F13C0F34170C0EB830003344B4683
:100E4000A3EB0902824211DB08F101080028A8BFC8
:100E50008144B845E1DB64E7042A80D1FFF72AFA30
:100E60000444C7E72046FFF725FAE7E714F8012F07
:100E700003F8012BE4E700252C4656F82500C207AD
:100E800032D4042830D9036803F00F02042A32D187
:100E9000FFF710FA04440135A945EED1204603F0CE
:100EA000E7F8054600283FF468AF041DB04606EB9E
:100EB000890958F8046BF30728D4042E26D933681F
:100EC00003F00F02042A34D13046FFF7F3F9074646
:100ED000304602F0B7FE3A460146204609F040FE91
:100EE0003C4421E02546C8E701A9FFF7E3FE01A83D
:100EF0000AF0FAF9CEE7032A7FF431AFC3F30F12F9
:100F0000C3F34173C3EB82031C44C4E701A9304619
:100F1000FFF7D0FE01A80AF0E7F901A9064602464C
:100F2000204609F01DFE3444C145C2D10023237080
:100F3000F7E6032AF8D1C3F30F17C3F34173C3EBEA
:100F400087073A46311DC8E72DE9F04F002893B0D6
:100F50000F4607DC1C2000F021FC0546284613B094
:100F6000BDE8F08F0D6815F0010806D1042D04D9F5
:100F70002B6803F00F03092B01D00B20EBE76E6801
:100F80007610002E03DC404603F072F8E5E70128F6
:100F900026D04868C20723D4042821D9036803F067
:100FA0000F03042B1CD102F04DFE044620460AF02C
:100FB0009BF90435731E8146009303FB00FB05EB90
:100FC000860A55F8040FC30771D404286FD9036843
:100FD00003F00F02042A05D1FFF76CF983440AE0FD
:100FE000384CE3E7032A69D1C3F30F12C3F341730B
:100FF000C3EB82039B44AA45E3D1584603F038F87B
:1010000005460028AAD0D7F800A0B9F1000F03D0F8
:10101000786802F017FE0446284602F013FE0AF133
:10102000040307460193019B53F804AF0193504614
:1010300002F008FE1AF001030146029302D1BAF150
:10104000040F04D805A95046FFF734FE05A9084649
:1010500003910AF049F9DDE9023183468BB9BAF10F
:10106000040F0ED9DAF8000000F00F0CBCF1030FEA
:1010700001BFC0F30F13C0F341700AF10401C0EBCC
:10108000830B38465A4609F06BFD5F44B9F1000FF7
:1010900008D0009B434505DD38464A46214609F005
:1010A0005FFD4F4408F101084645BCD156E705A94C
:1010B000FFF700FE05A80AF017F98FE702F0C2FD5E
:1010C000F9E700BF99C70000021E10B513DD0B68D9
:1010D00013F001041CBF5C1024EAE474012A00D060
:1010E0004A68611C092002F049FF18B1640044F00D
:1010F0000104446010BD00240122F2E70A6838B5FB
:1011000012F0010436D1042A34D91368496803F077
:101110000F00092818D15068C3F30F134010834201
:1011200098BF03F1FF30151DA04205DC01330220FA
:10113000984205DB002038BD45F8041F0134F3E771
:1011400042F820100130F3E7032813D1C80704D474
:101150001320BDE8384000F021BB4910FF29F7D823
:101160000432C3F30F1302EB83039A42E2D202F874
:10117000011BFAE70B2000F011FBDBE72DE9F04142
:101180004E6816F00107884629D1042E27D9326807
:1011900002F00F03092B12D17068C2F30F12451031
:1011A000AA4200D8551ED8F8008018F0010F1AD0B6
:1011B0004FEA6804002C49DDA54220DA46E0042B02
:1011C00004D13046FFF776F80546ECE7032B08D14B
:1011D000C2F30F10C2F34172C2EB8005E3E70025B2
:1011E000E1E73D46DFE741463248FFF7DFFCA8B1C3
:1011F00009F0CCFF90FBF5F303FB1500441C002F16
:1012000055D1042E53D9336803F00F03092B26D18F
:10121000013456F824402046BDE8F0814146264876
:10122000FFF7C4FCC8B9B8F1040F11D9D8F80030E1
:1012300003F00F03042B0BD14046FFF797FC041E6D
:10124000B9D141461D48FFF7B1FC08B1122000E0BA
:101250001120BDE8F04100F0A1BA2C46CFE7042BE5
:101260001DD1304602F0EEFC012C05460FDCFFF7E5
:1012700037F8461B304602F0FBFE04460028CAD071
:1012800002F0E0FC3246294609F06AFCC3E72B78FD
:10129000013C002BDAD02846FFF722F8E4E7032BC5
:1012A00005D13444E478640044F00104B3E70B2032
:1012B000CFE700BF60C200006BC2000070C2000038
:1012C0002DE9F0414C6814F0010788462ED1042C1A
:1012D0002CD923688E6803F00F02092A13D16568A0
:1012E000C3F30F136D10AB4200D85D1ED8F8001089
:1012F0003448FFF75BFC68B3236803F00F03092B46
:101300001ED1012317E0032A10D1F20704D41320C1
:10131000BDE8F04100F042BA7710FF2FF7D8C3F3D1
:101320000F15C3F34173C3EB8505DFE70B20EFE730
:10133000013344F823609D42FADA0020BDE8F081D1
:10134000032BFAD1033401239D42F6DB04F8017F1D
:101350000133F9E7D8F8008018F0010F0ED04FEAFA
:101360006800002822DD854220DB236803F00F039C
:10137000092B21D1013044F82060DEE741461248B4
:10138000FFF714FCB0B9B8F1040F11D9D8F8003048
:1013900003F00F03042B0BD14046FFF7E7FB0028B7
:1013A000E0D141460948FFF701FC08B11220AFE740
:1013B0001120ADE72846D8E7032B04BF2418E770B7
:1013C000BBE700BF67C200006BC2000070C2000034
:1013D000086808B5C3071BD4042819D9036803F0AB
:1013E0000F02092A01D1406808BD032A09D1C3F3BD
:1013F0000F12C3F34170C0EB8200400040F00100C7
:10140000F2E7042A04D102F01DFCFEF77DFFF4E7A9
:101410000120E9E7024A03480D2104F0DFBA00BFCA
:10142000F8C10000F0C100000020704704207047A0
:1014300001207047002002F01BBE002070470020F2
:101440007047002070470020704700207047002040
:10145000704700207047002070470000024A034890
:101460000C2104F0BBBA00BF04C3000064C3000039
:101470007047037883B11A0601D40130704703F036
:10148000C003C02B08BF013002461046013203786A
:1014900003F0C003802BF8D070470000F8B511F0BE
:1014A000010506461446084626D104293FD90B6893
:1014B00003F00F03042B3AD1D30714D4042A36D9EE
:1014C000136803F00F03042B31D102F0BBFB054678
:1014D000204602F0B7FB0146284609F0FBFE002833
:1014E0002DDB1ED126E002F0ADFB29460A2209F0D1
:1014F000BFFF0546601011E012F0010715D1042A64
:1015000015D9136803F00F03042B10D110464D10AA
:1015100002F098FB0A22394609F0AAFF85420EDB49
:1015200008DD002E09DC00200CE04D10E2E7064B40
:101530000F221A700136022EF5D8042002E070172F
:1015400000F00400F8BD00BF840200202DE9F04146
:101550002E4F06460024E500EB191B79032B0BD018
:101560000134FF2CF7D1304604F04CFA002814BFA8
:1015700004464FF0FF3445E0304609F0B5FE3146F1
:101580000246E0B204F0C6FA00283BD1EB59596894
:101590001A1D8842E4D052F8045FF02D00F10100DA
:1015A000F7D1800008301A18D107D9D4042AD7D926
:1015B0001B5803F00F010429D2D1C3F30F130133D9
:1015C00002EB8300C507CBD40428C9D952F82330D5
:1015D00003F00F03042BC3D102F034FB4FF00308D8
:1015E00005460921284609F068FE0028B8D0B8F160
:1015F000010800F10105F4D13146284609F0A3FEA7
:101600008542ADD12046BDE8F08100BF688601204B
:1016100010B510F0010402D04410204610BD04287B
:1016200012D9026802F00F02042A07D102F00AFB65
:101630000A222146BDE8104009F01ABF032A03D14F
:101640000A2221460430F5E7014B0D221A70E4E727
:101650008402002010F0010210B516D1042802D92E
:101660000268C2F30F1211F0010310D1042902D94C
:101670000B68C3F30F13934216D1043000EB8302BF
:101680000331904205D301200BE00022EBE7002359
:10169000F1E710F8014B11F8013F1CB9B3FA83F0E0
:1016A000400910BD9C42ECD00020FAE72DE9F74F2D
:1016B000804689469A46304F304E6AB102233B70CD
:1016C000012333603368DFF8D0B00024FC54444574
:1016D00004DB03B0BDE8F08F3260F3E759F8240073
:1016E0003168C30707EB0105C1F5487105D5244AE8
:1016F0004310284609F07EFD04E0C8B9214A284677
:1017000009F078FD1C4809F0EFFD3060BAF1000FD8
:101710000CD008F1FF33A34208DDB0F5487F05D2B5
:10172000431C20223A540022FA5433600134CEE79D
:10173000042801D1144AE2E71BD9026802F00F0322
:10174000042B06D1019102F07DFA104A019903465B
:10175000CFE7092B03D143685A465B10C9E7032B37
:1017600008D1C2F30F13C2F34172C2EB8303084ADC
:10177000BFE70123074ABCE785020020A805002037
:1017800034CE000072C2000078C200005FD40000B6
:10179000E3C50000EEC50000D4C50000014B187081
:1017A000002070478402002010B501F089FF084C2A
:1017B000231D01461F22184609F0B0FD09F094FDD3
:1017C00004308008000140F004002060204610BD75
:1017D000600200202DE9F04F85B000F11801046986
:1017E0000291D0E90232824601EB8404BC4F416988
:1017F000029800EB8109397803EB820529BB53F885
:101800002230B84A1E1203F07F03043552F8233009
:10181000904643F0010318479AF8010004F0AAFD2E
:1018200000238AF8003021E03B7873B92B681E1240
:1018300003F07F03043558F82330EAE7029A231DAA
:101840009A1AD82A26DD1A233B70DAF808209AF86B
:10185000023039789AF80100AA1A921043EA02225B
:1018600004F08EFD00238AF800303B70DAF808306F
:10187000ED1A029BE41AA9EB0309AD10A4104FEA7C
:10188000A903CAF80C50CAF81040CAF8143005B0C1
:10189000BDE8F08F22461C463B781660002BD4D161
:1018A0002B681E1203F07F03043558F82330B0E78D
:1018B000029A231D9A1AD82A02DD1A233B70C4E724
:1018C00021461C462B680B603B782A1D0BB1154640
:1018D000BBE76B681E1203F07F03083558F823300E
:1018E00097E7029A231D9A1AD82A02DD1A233B7021
:1018F000ABE722461C463B7805EB86061660002BBC
:10190000A3D12B681E1203F07F03043558F823304F
:101910007FE7029A231D9A1AD82A02DD1A233B7008
:1019200093E722461C46704B53F8263013603B78F1
:10193000002B8AD12B681E1203F07F03043558F860
:10194000233066E7684B54F8042D43F826203B7893
:10195000002B7FF47AAF2B681E1203F07F0304354F
:1019600058F8233055E7DFF880B15BF82600FFF721
:101970004FFE3A785AB9009054F8040DFFF748FE2C
:10198000009B1844400040F001004BF826003B78D3
:10199000002B7FF45AAF2B681E1203F07F0304352F
:1019A00058F8233035E7029B221DD31AD82B02DDCD
:1019B0001A233B7049E7029B21464B4534BF59F837
:1019C0000C3C01230B603B781446002B7FF43DAFA9
:1019D0002B681E1203F07F03043558F8233018E7F4
:1019E000029B221DD31AD82B02DD1A233B702CE751
:1019F000029B4B4518D259F80C3C06F180465B100F
:101A0000C3EB8373033E334459F8233023603B78A0
:101A10001446002B7FF419AF2B681E1203F07F03CE
:101A2000043558F82330F4E618233B700023EDE723
:101A3000029B4B4518D259F80C3C54F8042D5B100E
:101A400006F18046C3EB8373033E334449F82320F9
:101A50003B78002B7FF4F9AE2B681E1203F07F0356
:101A6000043558F82330D4E618233B70F0E7029B86
:101A70004B4529D259F80C3C06F180465B10033ED9
:101A8000C3EB8373334459F82300FFF7C1FD83464A
:101A900054F8040DFFF7BCFD59F80C3C5B10C3EB88
:101AA000837358441E44400040F0010049F826006A
:101AB0003B78002B7FF4C9AE2B681E1203F07F0326
:101AC000043558F82330A4E618233B70F0E7029A57
:101AD000231D9A1AD82A09DD1A233B70B5E600BFE8
:101AE00084020020D4C30000608E012022461C46E0
:101AF00059F8263013603B78002B7FF4A6AE2B6894
:101B00001E1203F07F03043558F8233081E654F8A1
:101B1000043D49F826303B78002B7FF496AE2B68C5
:101B20001E1203F07F03043558F8233071E659F88C
:101B300026004FEA600B54F8040DFFF769FD584486
:101B400040003B7840F0010049F82600002B7FF46C
:101B50007CAE2B681E1203F07F03043558F8233047
:101B600057E6029BA4EB8604A3420BD83B78002BDC
:101B70007FF46BAE2B681E1203F07F03043558F818
:101B8000233046E6C24802F04DF83B78002B7FF444
:101B90005CAE2B681E1203F07F03043558F8233027
:101BA00037E6002E05EB8605FFF660AE3B78002B8E
:101BB0007FF44BAE2B681E1203F07F03043558F8F8
:101BC000233026E654F8043D042B04D1002E05EB07
:101BD0008605FFF64BAE3B78002B7FF436AE2B68C4
:101BE0001E1203F07F03043558F8233011E654F831
:101BF000043D042B04D0002E05EB8605FFF636AE1F
:101C00003B78002B7FF421AE2B681E1203F07F037C
:101C1000043558F82330FCE554F8040CC307A4F14C
:101C2000040B0BD54010013800280ADB400040F0BF
:101C3000010005EB8605CBF8000017E6FFF7E8FC8E
:101C4000F1E73B780BB15C46FFE52B681E1203F011
:101C50007F035C4658F823300435DAE5730003F45B
:101C6000FF7343F001032360DAF80830EB1A9D108C
:101C70009AF8023043EA05235B0043F001036360F6
:101C8000029BA9EB030322465B1043F001033612CB
:101C900093608AF802607F4B3A78F6B20C4653F8AC
:101CA0003630CAF808301AB103F108058946CCE588
:101CB00003F10C059B681E1203F07F03894658F858
:101CC0002330A6E5029B54F8046C4B452FD1F7074F
:101CD00020D4042E17D9336803F00F03042B13D13B
:101CE000304601F0AFFF09F0FFFAB0F5487F28BF9A
:101CF0004FF448700630643003F03EFF70B9043D85
:101D0000DDF80890B2E507D0002E14BF4FF4007044
:101D10000720F0E70A20EEE70720ECE731469AF8C3
:101D2000010004F044FB00238AF80030E8E759F88A
:101D30000C3C58495A106FF0030353430C3B09EB1A
:101D4000030449F8036059F8083C5A108AF8022045
:101D5000D2B2C3F3552351F83220CAF8082059F8FB
:101D6000041C4FEA6109029901EB890939780434AE
:101D700002EB830500297FF468AD52F823301E1270
:101D800003F07F03043558F8233042E554F8040C7F
:101D9000FFF73EFC1E288346A4EB860425DC0028C2
:101DA0000BDC3B78002B7FF450AD2B681E1203F048
:101DB0007F03043558F823302BE501F06BFCABF1C1
:101DC000030B354E834401F065FCA0EB0B00B042E1
:101DD000F9D83B78002B7FF438AD2B681E1203F046
:101DE0007F03043558F8233013E501238AF80030C7
:101DF00001F050FC0A385844CAF8040036E554F89B
:101E0000040CFFF705FCA4EB8604061E0BDC3B78F4
:101E1000002B7FF41AAD2B681E1203F07F030435EC
:101E200058F82330F5E41D4B9E4202DD1D233B7024
:101E30000BE501238AF8003001F02CFC4FF47A7393
:101E400003FB06000A38D7E700233046A4EB8604DC
:101E5000134E1A462146FFF729FC3168114802F05B
:101E60000EF9114B316818600E4804F061F93168C1
:101E70000C4804F0A1FA3B78002B7FF4E6AC2B6809
:101E80001E1203F07F03043558F82330C1E400BF6D
:101E900000C60000688601203F420F0080EE360039
:101EA000A805002085020020080000203B78A4EB54
:101EB0008604002B7FF4C9AC2B681E1203F07F034D
:101EC000043558F82330A4E4504603F0B9FE3B78BB
:101ED000002B7FF4BAAC2B681E1203F07F0304358D
:101EE00058F8233095E454F8043C002B44D154F8BE
:101EF0000C0C10F0010B1ED04FEA600B4FEA4B03A5
:101F000043F0010344F8083CBBF1000F40F3888024
:101F10004FEA4B0343F0010354F80C0C44F8043C23
:101F200054F8083CC107CBEB63032AD501335B00AF
:101F300043F0010330E004281BD9036803F00F02CB
:101F4000092A01D14068D7E7042A09D101F07AFEB5
:101F50000378002BD2D0FFF78CFA0BF1010BF7E7D7
:101F6000032A06D1C3F30F1BC3F34173C3EB8B0BDF
:101F7000C4E719233B7068E44FEA630B0BF1FF3BA6
:101F8000C2E7042849D9026802F00F02092A11D1D8
:101F900003F1020B50F82B3049F826303B78002B28
:101FA0007FF453AC2B681E1203F07F03043558F8FE
:101FB00023302EE4042A2BD1039309EB86030093EC
:101FC00001F040FE039B83465E1C012E12DC584646
:101FD000FFF74FFAA0EB0B06304602F049F8034634
:101FE00070B1039001F02EFE3246594608F0B8FD5C
:101FF000039B05E09BF80030013E23B912223A70A2
:10200000009A1360CAE75846FFF733FA8346DCE7C5
:10201000032A02D11844037989E719233B7014E499
:102020000435BBE7029A04EB86039B1AD82B11DC1C
:102030000122002E06F1FF3310DC3B78002B7FF4E9
:1020400004AC2B681E1203F07F03043558F82330CC
:10205000FFF7DFBB1A233B70FFF7F7BB22601E467A
:102060000434E6E7029A231D9B1AD82B03DD1A23BA
:102070003B70FFF7EABB029B4B452AD254F8040C95
:10208000FFF7C6FA002821DD59F80C3C5B108342AB
:102090001CDBC3EB8373184400F180400438A4EBCD
:1020A000860359F820201A606FF003003B7800FB8C
:1020B00006440434002B7FF4C8AB2B681E1203F0D7
:1020C0007F03043558F82330FFF7A3BB20233B7070
:1020D000EAE71823FBE7C04B1A68A4EB86036FF00E
:1020E00003001A603B7800FB06440434002B7FF4A5
:1020F000ACAB2B681E1203F07F03043558F8233075
:10210000FFF787BB54F8043C042B3B78A4F104028E
:1021100004BF05EB8605224613B11446FFF795BBB5
:102120002B681E1203F07F03144658F82330043541
:10213000FFF76FBB54F8043D042B1CBF0023236042
:102140003B781CBF05EB86050434002B7FF47DAB88
:102150002B681E1203F07F03043558F82330FFF775
:1021600058BB002EA4EB860115DC1C233B7000221B
:102170006FF003003B780A6000FB06440434002B38
:102180007FF463AB2B681E1203F07F03043558F80D
:102190002330FFF73EBB0B684FF0000C5B1051F88B
:1021A0002C0010F0010202D10D233B70E0E740103B
:1021B00083420CF1010CA8BF03466645EFDC5B00CF
:1021C00043F00102D4E7002EA4EB860115DC1C23AA
:1021D0003B7000226FF003003B780A6000FB06446E
:1021E0000434002B7FF431AB2B681E1203F07F0305
:1021F000043558F82330FFF70CBB0B684FF0000C88
:102200005B1051F82C0010F0010202D10D233B703D
:10221000E0E7401083420CF1010CB8BF034666456D
:10222000EFDC5B0043F00102D4E754F8081C11F026
:10223000010F4FEA86031ED054F8042CD0071AD59C
:102240005210B2EB610FA4EB0303D4BF00220422AF
:102250001A606FF003003B7800FB06440434002B47
:102260007FF4F3AA2B681E1203F07F03043558F89D
:102270002330FFF7CEBA54F8042C6FF00100A4EB22
:10228000030BFFF70BF9CBF80000E2E754F8081C4A
:1022900011F0010F4FEA86031ED054F8042CD0072A
:1022A0001AD55210B2EB610FA4EB0303B4BF0022A6
:1022B00004221A606FF003003B7800FB06440434EC
:1022C000002B7FF4C2AA2B681E1203F07F03043593
:1022D00058F82330FFF79DBA54F8042C4FF0FF3024
:1022E000A4EB030BFFF7DAF8CBF80000E2E754E9C0
:1022F000020181424FEA860314D1E31A04221A60D4
:102300006FF003003B7800FB06440434002B7FF49D
:102310009CAA2B681E1203F07F03043558F8233063
:10232000FFF777BA0428A4EB030B01D8002315E0CC
:10233000C307FBD4036803F00F03042BF6D1CB07CC
:10234000F4D40429F2D90B6803F00F03042BEDD168
:10235000FFF780F900280CBF00230423CBF80030DE
:10236000CEE754E9020181424FEA860314D1E31A11
:1023700000221A606FF003003B7800FB064404342F
:10238000002B7FF462AA2B681E1203F07F03043532
:1023900058F82330FFF73DBA0428A4EB030B01D80B
:1023A000042315E0C307FBD4036803F00F03042BD9
:1023B000F6D1CB07F4D40429F2D90B6803F00F034C
:1023C000042BEDD1FFF746F900280CBF04230023AE
:1023D000CBF80030CEE700BF0800002054F8081CFE
:1023E00011F0010F4FEA86031ED054F8042CD007D9
:1023F0001AD55210B2EB610FA4EB0303CCBF00223D
:1024000004221A606FF003003B7800FB064404349A
:10241000002B7FF41AAA2B681E1203F07F030435E9
:1024200058F82330FFF7F5B954F8042C0120A4EB39
:10243000030BFFF733F8CBF80000E3E754F8081C70
:1024400011F0010F4FEA86031ED054F8042CD00778
:102450001AD55210B2EB610FA4EB0303ACBF0022FC
:1024600004221A606FF003003B7800FB064404343A
:10247000002B7FF4EAA92B681E1203F07F030435BA
:1024800058F82330FFF7C5B954F8042C0220A4EB08
:10249000030BFFF703F8CBF80000E3E754F8043C24
:1024A000042BA4EB860314BF042200221A606FF0F1
:1024B00003003B7800FB06440434002B7FF4C5A9DD
:1024C0002B681E1203F07F03043558F82330FFF702
:1024D000A0B954F8080CFFF79BF8834654F8040C95
:1024E000FFF796F85844A4EB8603400040F0010043
:1024F00018606FF003003B7800FB06440434002BA7
:102500007FF4A3A92B681E1203F07F03043558F84B
:102510002330FFF77EB954F8080CFFF779F88346AB
:1025200054F8040CFFF774F8ABEB0000A4EB86033F
:10253000400040F0010018606FF003003B7800FBA2
:1025400006440434002B7FF480A92B681E1203F08C
:102550007F03043558F82330FFF75BB954F8080CB3
:10256000FFF756F8834654F8040CFFF751F800FBC8
:102570000BF0A4EB8603400040F0010018606FF000
:1025800003003B7800FB06440434002B7FF45DA974
:102590002B681E1203F07F03043558F82330FFF731
:1025A00038B954F8040CFFF733F88346B8B91F2341
:1025B0003B70A4EB86036FF00300C3F800B03B78D8
:1025C00000FB06440434002B7FF43FA92B681E1245
:1025D00003F07F03043558F82330FFF71AB954F895
:1025E000080CFFF715F890FBFBFB4FEA4B0B4BF089
:1025F000010BDEE754F8040CFFF70AF88346B8B97C
:102600001F233B70A4EB86036FF00300C3F800B0F8
:102610003B7800FB06440434002B7FF416A92B689A
:102620001E1203F07F03043558F82330FFF7F1B88A
:1026300054F8080CFEF7ECFF90FBFBF303FB1B0BBD
:102640004FEA4B0B4BF0010BDCE754F8040CFEF7A0
:10265000DFFF0028B8BF4042A4EB8603400040F0F3
:10266000010018606FF003003B7800FB064404345F
:10267000002B7FF4EAA82B681E1203F07F030435B9
:1026800058F82330FFF7C5B8A4EB860B012EDBF812
:10269000000028D1FEF7BCFF3246034603930092A8
:1026A00008F074FD039B009A012BB8BF012390FB37
:1026B000F3F101FB130313445B0043F00103CBF878
:1026C00000306FF003003B7800FB06440434002B1D
:1026D0007FF4BBA82B681E1203F07F03043558F863
:1026E0002330FFF796B8FEF793FF0090DBF8040065
:1026F000FEF78EFF009A0130831ACFE7A4EB860B1A
:102700005946304601F050FE3B78CBF800006FF0A0
:10271000030000FB06440434002B7FF496A82B68CA
:102720001E1203F07F03043558F82330FFF771B809
:1027300054F8080CFEF76CFF834654F8040CFEF7BF
:1027400067FF0BEA0000A4EB8603400040F00100A5
:1027500018606FF003003B7800FB06440434002B44
:102760007FF473A82B681E1203F07F03043558F81A
:102770002330FFF74EB854F8080CFEF749FF8346A4
:1027800054F8040CFEF744FF4BEA0000A4EB860368
:10279000400040F0010018606FF003003B7800FB40
:1027A00006440434002B7FF450A82B681E1203F05B
:1027B0007F03043558F82330FFF72BB854F8080C82
:1027C000FEF726FF834654F8040CFEF721FF8BEA40
:1027D0000000A4EB8603400040F0010018606FF099
:1027E00003003B7800FB06440434002B7FF42DA843
:1027F0002B681E1203F07F03043558F82330FFF7CF
:1028000008B854F8040CFEF703FFC043A4EB86039A
:10281000400040F0010018606FF003003B7800FBBF
:1028200006440434002B7FF410A82B681E1203F01A
:102830007F03043558F82330FEF7EBBF54F8080C3B
:10284000FEF7E6FE834654F8040CFEF7E1FE0BFAB1
:1028500000F0A4EB8603400040F0010018606FF028
:1028600003003B7800FB06440434002B7EF4EDAFFC
:102870002B681E1203F07F03043558F82330FEF74F
:10288000C8BF54F8080CFEF7C3FE834654F8040C86
:10289000FEF7BEFE4BFA00F0A4EB8603400040F0CA
:1028A000010018606FF003003B7800FB064404341D
:1028B000002B7EF4CAAF2B681E1203F07F03043591
:1028C00058F82330FEF7A5BF54F80C0CFEF7A0FE15
:1028D000834654F8080CFEF79BFE8BFB002354F84C
:1028E000040CCDE90023FEF793FEDDE90023C0F1DF
:1028F000200CB0F1200103FA0CFC22FA00F040EAAF
:102900000C005CBF43FA01F10843A4EB860E4000C3
:1029100040F00100CEF800003B786FF0030000FBB0
:1029200006440434002B7EF490AF2B681E1203F093
:102930007F03043558F82330FEF76BBFA4EB860BFA
:1029400059463046FEF7C0FB3B78CBF800006FF0ED
:10295000030000FB06440434002B7EF476AF2B68A2
:102960001E1203F07F03043558F82330FEF751BFE1
:10297000A4EB860421463046FEF7C0FB3B78002BD3
:102980007EF463AF2B681E1203F07F03043558F802
:102990002330FEF73EBFA4EB860B59463046FEF7C8
:1029A000EDFB3B78CBF800006FF0030000FB064422
:1029B0000434002B7EF449AF2B681E1203F07F0312
:1029C000043558F82330FEF724BFA4EB86042146D3
:1029D0003046FEF775FC3B78002B7EF436AF2B6853
:1029E0001E1203F07F03043558F82330FEF711BFA1
:1029F000A4EB860B59463046FEF7EAFC3B78CBF851
:102A000000006FF0030000FB06440434002B7EF44A
:102A10001CAF2B681E1203F07F03043558F82330D7
:102A2000FEF7F7BE54F8040C01F00CF954F8083C1A
:102A3000DA072AD4042B0CD91B6803F00F03013BDF
:102A4000082B10D8DFE803F0052127230F0F0F0F05
:102A50002500CC4908F03EFCA4EB8603002814BFF7
:102A6000002204221A606FF003003B7800FB06444A
:102A70000434002B7EF4E9AE2B681E1203F07F03B2
:102A8000043558F82330FEF7C4BEBF49E2E7BF491A
:102A9000E0E7BF49DEE7BF49DCE7029B261DF31AEA
:102AA000D82B03DD1A233B70FEF7CFBE00F0FAFDF2
:102AB0002346400040F0010018603B783446002B6C
:102AC0007EF4C3AE2B681E1203F07F03043558F862
:102AD0002330FEF79EBE029B261DF31AD82B03DD82
:102AE0001A233B70FEF7B1BE00F0D4FDAA4B22467C
:102AF00003EA40003B7840F0010034461060002BB0
:102B00007EF4A3AE2B681E1203F07F03043558F841
:102B10002330FEF77EBE029B261DF31AD82B03DD61
:102B20001A233B70FEF791BE00F0BCFD9B4B1B6867
:102B300098423DBFC3F5830303F63713C018C01A8C
:102B40004000234640F0010018603B783446002BDB
:102B50007EF47BAE2B681E1203F07F03043558F819
:102B60002330FEF756BE00F09DFD8C4B18603B787D
:102B7000A4EB8604002B7EF468AE2B681E1203F0D3
:102B80007F03043558F82330FEF743BE00F096FD6E
:102B9000B30068B9E41A3B78002B7EF456AE2B687C
:102BA0001E1203F07F03043558F82330FEF731BEC0
:102BB000304627467A4EE41A01231A462146FEF78C
:102BC00075FD3068643002F0D7FF18B9043D3C460B
:102BD000FEF74CBE9AF801203168724803F0FFFB03
:102BE00001238AF8003000F055FD6F4A33681268FF
:102BF000063302FB0300FFF7FFB800F05FFDB300F0
:102C000068B9E41A3B78002B7EF41FAE2B681E12C5
:102C100003F07F03043558F82330FEF7FABD304641
:102C200027465F4EE41A002201232146FEF73EFDAF
:102C30003068643002F0A0FF0028C7D0594803F084
:102C400063F9CDE7FEF7B0FDA4EB860B3B78CBF83C
:102C500000006FF0030000FB06440434002B7EF4F8
:102C6000F4AD2B681E1203F07F03043558F82330AF
:102C7000FEF7CFBD3B78A4EB8604002B7EF4E5ADD8
:102C80002B681E1203F07F03043558F82330FEF73B
:102C9000C0BDA4EB860B584600F03DFD3B78CBF859
:102CA00000006FF0030000FB06440434002B7EF4A8
:102CB000CCAD2B681E1203F07F03043558F8233087
:102CC000FEF7A7BDA4EB860B584600F026FD3B7827
:102CD000CBF800006FF0030000FB06440434002B27
:102CE0007EF4B3AD2B681E1203F07F03043558F851
:102CF0002330FEF78EBDA4EB860B5946304600F01C
:102D000089FC3B78CBF800006FF0030000FB064421
:102D10000434002B7EF499AD2B681E1203F07F0360
:102D2000043558F82330FEF774BDA4EB8604204622
:102D300000F0F6FC3B78002B7EF487AD2B681E126A
:102D400003F07F03043558F82330FEF762BDA4EB8F
:102D5000860B5946304600F0D1FB3B78CBF800009B
:102D60006FF0030000FB06440434002B7EF46DADCD
:102D70002B681E1203F07F03043558F82330FEF74A
:102D800048BD00BF10C6000018C600001FC60000E6
:102D900026C600002BC60000FEFFFF7FB005002006
:102DA000A80500208502002004000020A4EB860472
:102DB000204600F09BFD3B78002B7EF446AD2B684F
:102DC0001E1203F07F03043558F82330FEF721BDAF
:102DD0000121304600F058FD3B78002B7EF435ADE4
:102DE0002B681E1203F07F03043558F82330FEF7DA
:102DF00010BD0021304600F047FD3B78002B7EF4EB
:102E000024AD2B681E1203F07F03043558F82330DD
:102E1000FEF7FFBCA4EB860B584600F0EDFC3B78B8
:102E2000CBF800006FF0030000FB06440434002BD5
:102E30007EF40BAD2B681E1203F07F03043558F8A7
:102E40002330FEF7E6BCA4EB860B584600F0E8FC06
:102E50003B78CBF800006FF0030000FB064404341D
:102E6000002B7EF4F2AC2B681E1203F07F030435B6
:102E700058F82330FEF7CDBCA4EB8604204600F0C2
:102E80009DFC3B78002B7EF4E0AC2B681E1203F017
:102E90007F03043558F82330FEF7BBBCA4EB86044F
:102EA000204603F019FF3B78002B7EF4CEAC2B6854
:102EB0001E1203F07F03043558F82330FEF7A9BC37
:102EC000A4EB860B584603F0DDFF3B78CBF80000FF
:102ED0006FF0030000FB06440434002B7EF4B5AC15
:102EE0002B681E1203F07F03043558F82330FEF7D9
:102EF00090BCA4EB8604204603F03EFE3B78002BFA
:102F00007EF4A3AC2B681E1203F07F03043558F83F
:102F10002330FEF77EBCA4EB860B584603F048FE38
:102F20003B78CBF800006FF0030000FB064404344C
:102F3000002B7EF48AAC2B681E1203F07F0304354D
:102F400058F82330FEF765BCA4EB860421463046D2
:102F500001F090FD3B78002B7EF477AC2B681E12BD
:102F600003F07F03043558F82330FEF752BCA4EB7E
:102F700086042146304601F07DFB3B78002B7EF431
:102F800064AC2B681E1203F07F03043558F823301D
:102F9000FEF73FBCA4EB86042146304601F024FC3A
:102FA0003B78002B7EF451AC2B681E1203F07F039C
:102FB000043558F82330FEF72CBCA4EB86042146D8
:102FC000304601F037FC3B78002B7EF43EAC2B689A
:102FD0001E1203F07F03043558F82330FEF719BCA6
:102FE000A4EB860B5946304604F060F83B78CBF8EA
:102FF00000006FF0030000FB06440434002B7EF455
:1030000024AC2B681E1203F07F03043558F82330DC
:10301000FEF7FFBBA4EB860B5946304604F04EF892
:103020003B78CBF800006FF0030000FB064404344B
:10303000002B7EF40AAC2B681E1203F07F030435CC
:1030400058F82330FEF7E5BBA4EB860B5946304613
:1030500004F03CF83B78CBF800006FF0030000FB75
:1030600006440434002B7EF4F0AB2B681E1203F0F0
:103070007F03043558F82330FEF7CBBBA4EB860B57
:103080005946304603F036FC3B78CBF800006FF031
:10309000030000FB06440434002B7EF4D6AB2B68FF
:1030A0001E1203F07F03043558F82330FEF7B1BB3E
:1030B000A4EB86042146304601F060FC3B78002BEF
:1030C0007EF4C3AB2B681E1203F07F03043558F85F
:1030D0002330FEF79EBBA4EB86042146304601F068
:1030E000D1FB3B78002B7EF4B0AB2B681E1203F0B3
:1030F0007F03043558F82330FEF78BBBA4EB860B17
:103100005946304601F038FB3B78CBF800006FF0B1
:10311000030000FB06440434002B7EF496AB2B68BE
:103120001E1203F07F03043558F82330FEF771BBFD
:10313000A4EB86042146304601F0E2FA3B78002BEE
:103140007EF483AB2B681E1203F07F03043558F81E
:103150002330FEF75EBB002E7CDD012E54F804BC4C
:103160003CD11BF0010F46D1BBF1040F43D9DBF872
:10317000003003F00F03042B3DD1584600F062FDF0
:10318000FEF7E4F903465A1CA4EB860462D0022E33
:1031900041D11BF0010F37D1BBF1040F34D9DBF85B
:1031A000002002F00F02092A2ED1DBF80400261FAE
:1031B000C0F347000122824220DD04EB8004FF2B94
:1031C0002BD840EA0326029B04F10C01CB1AD82B22
:1031D0007EF744AD1A233B70FEF737BB022E0AD1AF
:1031E00054F8080CC10706D4042804D9036803F076
:1031F0000F03042BC2D04FF0FF33C4E701325BF85A
:10320000221046F8041FD6E70B233B7000232360EF
:103210000434FEF71ABB0020D1E7029AA21AA4EBED
:10322000800B9210CAF81020594698472E4A002366
:1032300013603B78CBF800000BF10404002B7EF404
:1032400004AB2B681E1203F07F03043558F82330BB
:10325000FEF7DFBA002323603B78221D13B114462A
:10326000FEF7F3BA2B681E1203F07F03144658F8DA
:1032700023300435FEF7CDBA029BE31A9B10A4EB72
:103280008604CAF810302146304602F07DFE3B78B5
:10329000002B7EF4DAAA2B681E1203F07F0304359C
:1032A00058F82330FEF7B5BA029BE31A9B10A4EB43
:1032B000860BCAF810305946304602F065FE3B785E
:1032C000CBF800006FF0030000FB06440434002B31
:1032D0007EF4BBAA2B681E1203F07F03043558F856
:1032E0002330FEF796BA00BF546D01202DE9F84F48
:1032F000224D0023002B03F1FF3706DA01F0D0FB4B
:1033000002F052FF03F0CAF819270026DFF8788090
:103310003046D8F80020B24215DD2B68184C013336
:103320009342A8BF00232B60D5F80090F02303FB45
:1033300009F304EB030AE35CA346EBB1022B04D1CF
:103340005046FEF747FA3B46D4E7012B0ED108B9A9
:1033500000F0A0F9F02303FB09F39B440949DBF8D3
:103360000420821A8A429CBF0222E254F02303FB0B
:1033700009F3E35C022BE3D00136CAE7000000202A
:10338000087D01203F420F00AC0500200A4B4FF49E
:1033900080721A60094B01211964D3F84025053267
:1033A000C3F84825C3F84C254FF44022C3F8042342
:1033B000034B1970704700BF00E100E0008000403F
:1033C000D705002004207047F8B5D1E9004514F076
:1033D00001002DD015F001002AD064101C2C3CD81F
:1033E0001F4F6D1041F288363B5DAE42A8BF2E469E
:1033F000012B05D00121204605F0EEFA01233B55B3
:10340000184B1B780BB9FFF7C1FF002D4FF00003DD
:10341000154A0EDC154940F2DC50FF25D65CB4425B
:1034200004BF21F81300D5540133042BF6D1042036
:10343000F8BDD15C8C4203D10C4A22F81360F6E748
:103440000133042BF5D10023D15CFF2901D1D454E1
:10345000F2E70133042BF7D1E9E70020E8E700BFEA
:10346000B8050020D70500201C0000200E00002019
:1034700070B5D1E9004514F001001BD015F0010032
:1034800018D064101D2C28BF1B24154E335D012B52
:1034900005D00121204605F09FFA01233355114B39
:1034A0006D10A5F110029A420F4B04D94FF0FF3274
:1034B0001A60042070BD1C600C4B0D4890FBF5F0A9
:1034C00018800C4B1B780BB9FFF760FF0A4B0122E9
:1034D0009A64D3F848251044C3F84805E9E700BFCB
:1034E000B805002090860100180000200C00002084
:1034F00020A10700D70500200080004070B50C68AF
:10350000E30704D40D20FEF749F9012070BD6410D3
:103510001C2C14D8012814DD4B68042B14BF002583
:1035200002250A4E335DAB4204D02946204605F001
:1035300053FA3555204605F095FA012803D00020AE
:10354000E4E70025EDE70420E0E700BFB805002030
:1035500070B50D680128CCBF4C68012415F001003E
:1035600042D014F001003FD06D10002D05DC1F4B40
:103570000122C3F80825002036E064101C2CFAD87C
:103580001B4E335D012B05D00121204605F024FAA6
:10359000012333550A22174B93FBF5F3053393FBB5
:1035A000F2F3154A154952F824201548120242F048
:1035B0000312C1F810250D4AC2F81005C2F81415FF
:1035C0000121C2F80415A2F5A83210690020C2F842
:1035D00010054FF6FF708342A8BF0346C2F840357E
:1035E0000420C2F80012116070BD00BF00F001405D
:1035F000B805002000B4C40424D8000000600040D6
:1036000040A10040002802DC1C20FEF7C7B80120C2
:1036100070470000F8B50B68DA0707460D4604D47A
:103620000D20FEF7BBF8012007E05B10062B05D14B
:1036300003F0D0FA400040F00100F8BDF3D80C4A86
:103640000C4E52F82340335D2BB10021204605F08B
:10365000C3F900233355012F06DD6B68042B03D11A
:103660000221204605F0B8F9204605F0BFF8E1E751
:10367000A0C60000B805002004207047002802DC26
:103680001C20FEF78BB80B68DB0701D40D20F8E790
:1036900000207047024B01221A64D3F8400570479E
:1036A00000800040044B01221A64D3F840054FF417
:1036B0007A73B0FBF3F07047008000400120704740
:1036C00000487047BCC600001D20704770B5054D0E
:1036D0002B5C8B4204460E4602D005F07DF92E5538
:1036E00070BD00BFB805002070B50024084D264607
:1036F000635D012B08D10021204605F097F90021D8
:10370000204605F069F9665501341D2CF0D170BDD5
:10371000B805002070470F2070473B20704700001D
:1037200070B50468E20702D54568EB0704D40D20A4
:10373000BDE87040FEF732B864101C2C2FD8184E2C
:10374000335D012B18D00121204605F045F90123F6
:103750001B2C335510D1134BDA6E134B202AB8BFF4
:103760004FF0A04302F01F0203EB8203D3F80027BF
:1037700042F44072C3F800270C4BD3F8082132B151
:10378000D3F81821002AFBD00022C3F81821A5F392
:103790004A0120468910BDE8704005F0CBB870BDE5
:1037A000B805002024D800000003005000C00140EC
:1037B00008B50846FFF7B4FF002008BD13B50A4A54
:1037C000044692E8030022686B46042A83E803005B
:1037D00019464FF0020003D101F006F802B010BD07
:1037E00001F028F8FAE700BF38C6000008B508461F
:1037F000FFF7E4FF002008BD10B5084C63792BB13A
:103800000021052005F0E8F800236371052005F08C
:1038100029F900280CBF0420002010BDB8050020A5
:1038200010B5084CE37A2BB100210B2005F0D4F839
:103830000023E3720B2005F015F900280CBF0420CB
:10384000002010BDB805002010B50B4A0B4C0C48E9
:103850000C490023C2F80035A2F5C832C2F8103571
:103860000122626042604A60C4F80035C0F8003549
:10387000C1F8003510BD00BF00F0014000C001409C
:1038800000100240002002401C2870B504460D467E
:1038900025D8134E335C012B04D0012105F09CF890
:1038A000012333551C2C12D1FFF7CEFF0D4B1A6F9D
:1038B0000D4B202AB8BF4FF0A04302F01F0203EBCC
:1038C0008203D3F8002742F44072C3F80027291C72
:1038D000204618BF0121BDE8704005F0A7B870BDB3
:1038E000B805002024D80000000300500368D90761
:1038F00002D40D20FDF752BF41680A1F51425141C9
:103900005810FFF7C1BF08B50846FFF7EFFF0020CA
:1039100008BD0000F8B5324CD4F84831ABB10023F3
:10392000D4F84855C4F848312E4B186800280CDBF1
:103930002D4A1178B1FA81F14909117005F076F834
:103940002A4B1B882B44C4F84835254BD3F84C210F
:10395000002A37D00021264ED3F84C45C3F84C112D
:103960003378244D33B12B68032B03D8224AD05C23
:1039700005F05CF82B68204F01335A4202F0030235
:1039800003F0030358BF53422B600022042B194657
:1039900019D00133F81810F8010CFF2801D10122C9
:1039A000F4E702B12960012105F040F801233370EA
:1039B0002A68124B33F8122004F10C031344084A0E
:1039C000C2F84C35F8BD4FF0FF3304F58C44044A7F
:1039D0002B605C3400233370C2F84C45F2E700BF23
:1039E0000080004018000020D60500200C000020B8
:1039F000D5050020B40500201C0000200E0000208A
:103A0000094B0A4940F2DC521A805A809A80DA80C7
:103A1000074A00231370074AFF2008704870887017
:103A2000C8701360704700BF0E0000201C0000200B
:103A3000D5050020B4050020024B4FF0FF321A607C
:103A4000704700BF18000020024A03480C2101F013
:103A5000C5BF00BF40C6000066CF000038B54FF4B8
:103A6000E131284804F086FC274B012200211A612D
:103A7000C3F804150321C3F808150421C3F8101571
:103A80001A604FF080430221C3F818159A604FF076
:103A90001023D3F80C32DB070FD51C4BC3F80425D9
:103AA000D3F80024002AFBD04FF010226FF0010160
:103AB000C2F80C120022C3F80425082004F07EFE90
:103AC000134A0023FF21995401331D2BFBD1114BC5
:103AD000114D01221A600020104A04230146146887
:103AE000002CFCD02C681160013B44EA0020F6D188
:103AF0000B4B01221A6004F097FDBDE8384001F03D
:103B00006BB800BF887C01200080004000E00140CD
:103B1000B805002000D0004008D5004000D100408A
:103B200004D00040F8B506460948094F0C4604F099
:103B300061FC8442A8BF04463546AB1B9C4205DDB0
:103B4000384604F05DFC05F8010BF6E72046F8BDA9
:103B5000887C01200146014804F011BC887C0120CA
:103B600010B5054C204604F017FC20464FF4E13117
:103B7000BDE8104004F0FEBB887C0120C3070CD4D4
:103B8000064B1B68834208D8054B1B68984204D833
:103B900050F8043C002B18BF18467047E005002081
:103BA000DC0500200B4908B50122002341F8232041
:103BB0000133642BFAD1084B1A60084B084A1846A7
:103BC000002106F0F1FF074B40F8043F064B186058
:103BD00008BD00BF608E012008000020E405002021
:103BE00070670100A09D0500D8050020034B044A22
:103BF0001A60044B044A1A60FFF7D4BFE0050020A6
:103C0000E4050020DC050020546D0120044B1B68F6
:103C10001868C0F30F10023820EAE070704700BF48
:103C2000D805002000B59BB00246054901A807F061
:103C300015FB01A802F085F902F030FCFCE700BF9B
:103C400089C70000C30713D4042802D812D00B4838
:103C50007047036803F00F03042B01D10430704751
:103C6000092B09D0064A0748032B18BF1046704796
:103C700005487047054870470548704772C2000004
:103C800074C700007DC7000063C7000078C2000051
:103C90006DC70000064B074900201A6843F8040C62
:103CA000C2F30F12023203EB82038B42F5D370474B
:103CB000E8050020546D01202F4B304A1868304B26
:103CC0002DE9F0411C682F4D136803F00F010729FF
:103CD00028D81368C3F30F13023302EB8302AA42FE
:103CE000F2D32949002251F82200FFF747FF41F89B
:103CF00022000132642AF6D1244A1068FFF73EFF01
:103D00001060234A106810B1FFF738FF1060214B94
:103D1000214C1E680021F0274FF03C08B14214DB13
:103D2000BDE8F081C3F30F1302EB83039A42D0D0B6
:103D30001968CE0707D4884205D28C4203D351F8C4
:103D4000041C01B11960043BF0E707FB01F31A19E9
:103D50001B5D0BB90131E1E71269551E08FB012219
:103D600004EB82021832002DF4DB52F8040DFFF749
:103D700005FF013D1060F6E7E0050020E8050020A2
:103D8000DC050020546D0120608E01200800002019
:103D9000546D0120AC050020087D0120C307F0B55B
:103DA00040D4214B1C68A0423CD3204B1D68A84244
:103DB00038D850F8043CABBB03680246C3F30F137A
:103DC000012673B9904242F8046C2BD0116851F867
:103DD000043C51F82370176041F82320013B0A4648
:103DE000EFE752F82310CF0702EB830C18D48C4274
:103DF00016D88D4214D351F8047C8FB90F6807F0A0
:103E00000F0EBEF1070F08D9CCF8007042F8043C41
:103E10000B680A60C3F30F13E1E741F8046CD0E7C5
:103E2000013BCEE7F0BD00BFE0050020DC0500202F
:103E30000D4930B50D4C0B461A6853F8045CC2F3BB
:103E40000F12901C65B18B4214BF0A46002243F842
:103E5000042C01EB800103EB8003A342ECD330BDC3
:103E600012011A60F7E700BFE8050020546D012039
:103E7000144B2DE9F041144C1E464FF000083268F7
:103E8000C2F30F1712070FD07D1C9E424FEA850523
:103E900005D018462A46314606F06DFE03465A19EB
:103EA00004352B44C2F80080023706EB8706A64291
:103EB000E5D3E41AA410013C044A24011C601360F9
:103EC000BDE8F081E8050020546D0120D8050020F0
:103ED0002DE9F0419AB0FFF7DDFB214D07460024A4
:103EE00055F824000134FFF759FF642CF8D11D4B1D
:103EF0001868FFF753FF1C4B186808B1FFF74EFF17
:103F00001A4DDFF874800026D8F800309E4218DB86
:103F1000FFF78EFFFFF7D0FEFFF7AAFFFFF7BAFB10
:103F2000134B14491B681B68C3F30F13C21B023BDE
:103F300001A807F093F901A802F003F81AB0BDE850
:103F4000F0812B7813B90136F035DDE72C69013C9F
:103F5000002CF8DB05EB84039869FFF71FFFF6E7F9
:103F6000608E012008000020546D0120087D012092
:103F7000D805002043C70000AC0500202DE9F84318
:103F80001B4C23681B684D1CC3F30F139D42064650
:103F900088461746A1460CDBFFF79AFF23681B688B
:103FA000C3F30F139D4204DB0A20BDE8F843FDF77D
:103FB000F5BB08F10202D9F800009B1A1B0140F87A
:103FC0002230002340F8043C06F00F06034646EA80
:103FD0000816940043F8046B0119083CC9F8001056
:103FE0001C44A34201D3BDE8F88343F8047BF8E7FF
:103FF000D8050020F8B510F0010704460E462CD174
:10400000174B1B68834228D8164B1B68834224D960
:10401000154D28600068012200F00F00FFF7AEFF89
:104020002C682F600546C0B12146043051F8042B9E
:10403000C2F30F12B242A8BF3246920006F090FDC2
:10404000FFF728FE44F8045CFFF736FE2268074BB2
:1040500044F8047C134023602C462046F8BD00BF82
:10406000E0050020DC050020546D0120F0FF0F006A
:10407000011D0022042091FBF0F1FFF77FBF38B54E
:10408000054608460C46FFF7F3FF50B1C21C2B460D
:10409000591B8C4206DC002CACBF0419041C002305
:1040A000237138BD13F8011B02F8011FF0E7F0B5CA
:1040B00002289BB00C4604DC1C20FDF76FFB1BB0F4
:1040C000F0BD0868C20706D4042804D9036803F0C9
:1040D0000F03042B01D00E20EFE74B6813F001070C
:1040E000F9D1042BF7D91B6803F00F03042BF2D18D
:1040F0008B68DB0701D40D20DFE7FFF7A3FD064641
:104100006068FFF79FFDA5681AAC014604F8647D5E
:104110006D10304603F061FC29466423224603F00B
:10412000BEFC204607F0E0F801462046FFF7A7FF57
:10413000C5E7000010B50446ADF5806D10B9FFF776
:1041400097FF0BE003F06FFB0138062827D8DFE864
:1041500000F0080810172804230000200DF5806DDA
:1041600010BD204603F0D9FB011B2046FFF787FF57
:10417000F4E7204603F085FB400040F00100EDE746
:1041800069464FF48062204603F095FB684607F0CD
:10419000ABF801466846E9E704210348E6E700205A
:1041A000CDE70420DAE700BFD0C70000022838B509
:1041B0000C4604DC1C20BDE83840FDF7EFBA086867
:1041C000C10706D4042804D9036803F00F03042BA5
:1041D00001D00E20EFE76368DA07FAD4042BF8D990
:1041E0001B6803F00F03042BF3D1A368DB0701D492
:1041F0000D20E0E7FFF726FD05466068FFF722FD8A
:10420000A46801466410284603F0E7FB214603F04A
:1042100023FCBDE83840FFF78DBF012838B50C46B8
:1042200004DC1C20BDE83840FDF7B8BA0868C107B7
:1042300006D4042804D9036803F00F03042B01D02B
:104240000E20EFE76368DA07FAD4042BF8D91B686D
:1042500003F00F03042BF3D1FFF7F4FC054660686D
:10426000FFF7F0FC0146284603F0B7FB03F033FCF0
:10427000400040F0010038BD012870B505460C46ED
:1042800004DC1C20BDE87040FDF788BA0868C1074F
:1042900006D4042804D9036803F00F03042B01D0CB
:1042A0000E20EFE76368DA07FAD4042BF8D91B680D
:1042B00003F00F03042BF3D1FFF7C4FC064660683C
:1042C000FFF7C0FC022D014615D0A468E30712D504
:1042D0006410304603F081FB054603F0A4FA012880
:1042E00012D1002C02DD0135012C07D12846BDE892
:1042F0007040FFF71FBF4FF0FF34EAE7284603F096
:104300001BFB013C0546EFE70228EFD1002CEDDD59
:104310000135012CEAD000221146284603F036FB75
:1043200003F00AFB013C0546F3E70000086810B5FE
:1043300010F001041AD0441007EE904A9FED187A4D
:10434000F8EEE77A67EE877A17EE900A06F06AF8D9
:1043500004F090FC0022134B06F0BCF804F040FC83
:1043600006F068FB400040F0010010BD042812D99F
:10437000036803F00F03042B07D1FFF763FC0A2245
:10438000214607F075F80446D6E7032B03D10A222D
:1043900021460430F5E70D20FDF700FACCE700BF19
:1043A000D30237390000D040086808B5C30706D4E7
:1043B000042804D9036803F00F03042B04D00E2053
:1043C000BDE80840FDF7EAB9FFF73CFC0378232B72
:1043D00008BF01301022002107F04AF800F1005315
:1043E000B3F1804F01D31420EAE7400040F0010010
:1043F00008BD0000024A0348062101F0EFBA00BFE1
:10440000A0C700009AC70000002070471E20FDF7DB
:10441000C5B91E20FDF7C2B91E20FDF7BFB91E2089
:10442000FDF7BCB91E20FDF7B9B91E20FDF7B6B9DE
:104430001E20FDF7B3B91E20FDF7B0B91E20FDF711
:10444000ADB91E20FDF7AAB91E20FDF7A7B91E20A1
:10445000FDF7A4B91E20FDF7A1B91E20FDF79EB9F6
:104460001E20FDF79BB91E20FDF798B91E20FDF711
:1044700095B91E20FDF792B91E20FDF78FB91E20B9
:10448000FDF78CB91E20FDF789B91E20FDF786B90E
:104490001E20FDF783B90000024A0348182101F0ED
:1044A0009DBA00BF0CC80000CCC80000034B01221D
:1044B0001A60034B1868904010437047786D0120D4
:1044C000586D01202DE9F043EFF31084012304F02F
:1044D000010483F31088164A164912680E68013ADF
:1044E0009340154A1568154A12684FF002094FF0BB
:1044F0000E0C4FF00D0E4FF00608A3B118422A60C3
:104500000AD0774639000139FDDC32604746390070
:104510000139FDDC5B08F0E74F4639000139FDDC6D
:1045200032606746F3E784F31088BDE8F08300BF8C
:1045300020000020606D0120646D01206C6D012061
:1045400070B5084E084D002456F824000021FFF7EE
:10455000BDF855F8240000210134FFF7B7F8052C09
:10456000F2D170BD08CA000054CD00002DE9F3411E
:104570003B4D4FF441732C68ADF804300A238DF89D
:104580000630BCBBFFF7DCFFDFF8E480264658F8B6
:10459000267001213846FFF799F801360021384688
:1045A00004F044FA052EF2D100260DF1040816F8A5
:1045B000087001213846FFF789F801360121384695
:1045C00004F034FA032EF2D100210420FFF77EF824
:1045D00000213046FFF77AF800210A20FFF776F82D
:1045E00001232B60FFF756F81E4B1860204602B0DF
:1045F000BDE8F0811B4B1C68FFF74CF8844298BF64
:10460000001BB0F57A6F29DB022004F0DDF80420EE
:1046100004F0ECF80446032004F0E8F807460A200A
:1046200004F0E4F80646012004F0CEF8012004F07E
:10463000DDF8E0193044C0F532600323023090FB0E
:10464000F3F0094B0028BCBF00221A60074AA8BF3C
:10465000186000232B6013600124C7E70024C5E71E
:10466000706D01207C6D0120586D0120786D012056
:1046700054CD000008B5054B00221A60044B1B689E
:104680000BB103F06FF8002008BD00BF746D01206E
:10469000EC7A012010B5041E1CDA00241049114BDD
:1046A000114A0B6004331360104B53F824301F2B56
:1046B00081BF0F4808600F49116003F01F024FF0DF
:1046C000010303FA02F38CBF0C310B490B4A0B6058
:1046D000136010BDFEF7F8FFA042DEDDDEE700BF8D
:1046E000646D012008050050606D012024D8000091
:1046F000080800500C080050180500506C6D01208F
:1047000008B50B68DA074CBF5B104FF0FF33012888
:104710000DDD4A68042A14BF1822202205491846D4
:104720000A60FEF7F7FFFFF7B5FF002008BD18226B
:10473000F4E700BF2000002010B510F0010402D003
:104740004410204610BD042812D9026802F00F025E
:10475000042A07D1FFF776FA0A222146BDE8104065
:1047600006F086BE032A03D10A2221460430F5E76B
:104770000D20FDF713F8E4E7086810F0010370B5A9
:104780001CD0FFF7D9FF0346203B5E2B27D8154CE2
:1047900003EB83030022012110462344052A1AD08B
:1047A0009E5C052410252E4218BF4018013C4FEA9C
:1047B00041014FEA6505F6D10132EFE70428E3D95C
:1047C000026802F00F010429DED1C2F30F13002B9F
:1047D000DAD00379D8E7400040F0010070BD012035
:1047E000FCE700BF1CCA000038B508680D46FFF79B
:1047F000A3FF04466868FFF79FFF621E042A014674
:1048000012D8431E042B0FD8084803EB830313442C
:104810000568012202FA03F32B430360044B1B6873
:1048200013B1204602F09FFF002038BD746D0120B7
:10483000EC7A012038B508680D46FFF77DFF044685
:104840006868FFF779FF621E042A014614D8431EE8
:10485000042B11D8094803EB83031344012202FA05
:1048600003F3026822EA0302054B02601B681BB1D6
:104870000022204602F077FF002038BD746D012031
:10488000EC7A01202DE9F04F054685B008680C460A
:10489000FFF752FF022D01903CDD6068FFF74CFFEF
:1048A0000746A068FFF748FF0446231DDFF8C8A0AD
:1048B0000293661E4FF00108029B9E4206F1010919
:1048C00035D006EB8602531E07F1050B3D460393D8
:1048D000AB4522D0042E19D86A1E042A16D8039B91
:1048E000019ADAF800005919224B4FF0010C18EA2E
:1048F000020E0CFA01F11B6811D00143CAF8001036
:1049000023B162464946284602F02DFF4FEA480887
:104910000135DDE701242746C7E74E46CCE720EA0C
:104920000101CAF80010002BF0D07246EAE73D1DE5
:10493000042D1BD8012C19D1DFF83C80DFF834900E
:104940000026D8F8003004FA05F223EA0203C8F87A
:104950000030D9F80030013623B100223146781DED
:1049600002F001FF052E05F10505EAD1002005B092
:10497000BDE8F08FEC7A0120746D01202DE9F84339
:10498000394B1B680C461BB94FF0FF30FFF782FE16
:10499000206810F001083AD1042838D9036803F0E0
:1049A0000F03092B33D10746304D57F8044F304ED3
:1049B000641040F25969A04552DA57F8040FFFF726
:1049C000BBFEC0F30742C0F307235B43524393FB94
:1049D000F9FC92FBF9F32A68202AC1B208BFC0F3A0
:1049E00005604FEA032308BF56F8202043EA0C4332
:1049F00001FB01F191FBF9F143EA010308BF42EA2F
:104A000003231846FFF75EFD08F10108D3E7FFF71F
:104A100093FEC0F30742C0F3072340F259655B439E
:104A2000524393FBF5F492FBF5F3104A1268202AE7
:104A3000C1B204BF0E4AC0F305604FEA032308BFAA
:104A400052F8202043EA044301FB01F191FBF5F108
:104A500043EA010308BF42EA03231846FFF732FD89
:104A60000020BDE8F88300BF6C6D0120200000200D
:104A7000F8CB0000086808B5C30703D5FFF75CFE54
:104A8000054B1860054B1B681BB1034B186802F0FF
:104A90006BFE002008BD00BF746D0120EC7A012080
:104AA0002DE9F843434E326852B9434B1B683BB97A
:104AB000424B1B68002B74D0BDE8F843FFF756BD8E
:104AC0003F4D2C6884BB3D4B1B68002B65D13A4A97
:104AD000336810681146002865D13A4F3A4EDFF826
:104AE000F4800B60002157F82400FEF7EFFD56F824
:104AF000249001214846FEF7E9FDB9F1220F10D8B4
:104B000058F82920314B1F2AD8BF4FF0A04302F09C
:104B10001F0203EB8203D3F8002742F44072C3F86C
:104B200000270134052CDDD12B68264EDFF8889054
:104B3000254F002BCCBF03F1FF330423002156F88F
:104B40002300FEF7C3FD2A68214B53F8228000247E
:104B500004EB840101EB0803D9F8001057F8240096
:104B6000194101F00101013403F060FF052CEFD180
:104B70002B68012156F82300FEF7A8FD2B680021C1
:104B800056F8230003F052FF2B68013393FBF4F433
:104B900004EB84041C1B2C6003E0FFF7E7FC0028F7
:104BA00095D1BDE8F883002B97D11360BDE8F84399
:104BB000FFF7C6BC746D0120686D0120786D01207F
:104BC0005C6D012008CA000054CD000000030050B5
:104BD000F8CC000024D800004FF0FF30FFF75ABD9A
:104BE000024A0348092100F0F9BE00BF0CCD0000C5
:104BF00068CD00004FF0805310B51A69094B0224AC
:104C0000C3F8044522F00302884203D30022C3F80C
:104C1000042510BDD3F80044002CFBD0C3F80805D0
:104C20001044F1E700E00140002815BF4FF4D22105
:104C30004FF4B4214FF4B4204FF49620FFF7DABFBD
:104C400000280CBF4FF496234FF4B4231868030ECA
:104C5000532B0CBF20F07F4000207047064B0122F1
:104C6000C3F80425D3F80024002AFBD000220160F9
:104C7000C3F80425704700BF00E00140002821F080
:104C80007F4141F0A6410CBF4FF496204FF4B42071
:104C9000FFF7E4BF0A4B30B50124C3F804450029EF
:104CA00003DC0022C3F8042530BD52F8044BD3F8CE
:104CB0000054002DFBD040F8044B0139EFE700BF52
:104CC00000E0014038B54C68023405460A462146EA
:104CD000FFF7E0FF05EB840038BD0000124B1B68B6
:104CE000002B0BBF4FF4B4224FF4D2224FF4962383
:104CF0004FF4B42328B91A1DDB79522B08BF104694
:104D0000704782420DD9C378522B0AD143680233CF
:104D100000EB8300824204D9C378522B18BF0020D5
:104D200070470020704700BF806E01202DE9F041E0
:104D30000020B4B0FFF7D2FF0024DFF8A4800546BE
:104D4000274626464DBB224D2868FFF779FF3B4694
:104D50003246CDE900401F4902A806F07FFA02A8BA
:104D600001F0EFF81C4B1A682B68002B0CBF4FF4B6
:104D700096234FF4B423D21A4FF470416423534363
:104D8000009193FBF1F302A8144906F067FA02A818
:104D900001F0D7F834B0BDE8F08169682A68019164
:104DA0008B1C1F44D1B2C2F307239C42C2F30742BB
:104DB000009102A84146B8BF1C4606F04FFA02A86F
:104DC00001F0BFF82846FFF789FF01360546B9E72D
:104DD000806E012072CE0000846E01201CCE000087
:104DE0005ECE000070B50020FFF72AFF05460120C7
:104DF000FFF726FF0C4B1E68B6FA86F485424FEA91
:104E00005414B8BF054620461C60FFF70DFF074A43
:104E1000074B002E18BF1346064A691C2046BDE802
:104E200070401360FFF72ABF806E012004B00400B9
:104E300004A00500846E012070B50020FFF700FF7C
:104E400002460120FFF7FCFE1F4E204C054672B9BA
:104E500068B94FF4D2214FF49620FFF7CBFE012121
:104E60002846FFF70BFF1A4B3560236029E0AA4262
:104E700008DD00233360164B23604FF4B421236810
:104E8000002017E001233360124B23604FF4D2213E
:104E9000F5E7120E522A08D000B123600E4801F047
:104EA00050F8BDE87040FFF79DBF5A68023203EB2F
:104EB000820301208B4205D21A68551CE9D10028D3
:104EC000D3D170BD2160FCE7806E0120846E01208B
:104ED00004B0040004A0050037CE000010B5002087
:104EE000FFF7FCFE014608B9084610BD8478FFF7BD
:104EF000F5FEDA2C08BF0146F5E7000038B50021C1
:104F00004FF4FF62124805F04FFEFFF7E7FF10492C
:104F1000002400B938BD0368C3F307420A2A0BD145
:104F2000C3F30722FF2A04D001EBC20541F8320087
:104F30002B71FFF7D3FEECE7132AFAD1C3F3072353
:104F4000FF2B1EBF01EBC30241F833401471F0E7A1
:104F50006886012000B59BB0FFF76EFFFFF7CEFF1C
:104F600000230B491A4651F8330000B101320133D6
:104F7000FF2BF8D1074901A806F070F901A800F04D
:104F8000E0FF054800F0DDFF1BB05DF804FB00BF4B
:104F900068860120A7CE0000BBCE00002DE9F04FAF
:104FA0004FF480729FB0604C6048002105F0FCFD1A
:104FB0004FF4807200215E4805F0F6FDD4F80090B1
:104FC000B9FA89F84FEA58184046FFF72DFEA24675
:104FD000584B594C0020B9F1000F08BF1C46FFF791
:104FE0007DFF064648BB4846FFF72AFE534D411C4D
:104FF0004046FFF743FECAF800802C60FFF77EFFB3
:10500000FEF7AEFDDAF800302A68002B0CBF4FF433
:1050100096234FF4B423D21A4FF4704164235343C0
:10502000009193FBF1F305A8454906F017F905A88F
:1050300000F087FF1FB0BDE8F08F3568C5F3074368
:10504000A3F10A02092AC5F3072546D8374B595D53
:1050500091BB10223B48DFF8ECB005F0A5FD3746C8
:105060003A68C2F307218D4209D1C2F307410B29E7
:1050700026D013292BD00A2901D1CBF8007038464D
:10508000FFF72CFE07460028EAD12E4F396881B180
:105090002046FFF717FE0123044657F8231029B1D5
:1050A00020460393FFF70EFE039B04460133042BB7
:1050B000F3D11E4A012353553046FFF70FFE90E708
:1050C000D2B2022ADBDC0BEB82025760D7E7102258
:1050D0000021584605F068FDD1E7A3F11502082A22
:1050E000EAD8134A525D002AE6D1152B0CBF31468F
:1050F000002130460368C3F30742152A0ED01D2A4B
:1051000008BF0021FFF7EAFD0028F3D119B12046BE
:10511000FFF7D8FD04460123054ACCE7C3F3072374
:105120009D4208BF0146EDE7806E0120806D0120A1
:10513000886E012004A0050004B00400846E0120E4
:1051400001CE0000F08F0120FFF728BF2DE9F84FB6
:10515000DFF8A8B0274F03339246042293FBF2F600
:10516000DBF80030B41C002B3B684FEA84040CBF12
:105170004FF4B4224FF4D22223449A4281460D4682
:10518000B84614D2FFF70AFFDBF80030002B3B686B
:105190000CBF4FF4B4224FF4D22223449A4206D2D9
:1051A000154800F0CEFE00273846BDE8F88F2D02E6
:1051B0005FFA8AF141F0A441ADB2D8F800700D4316
:1051C0004FEA094101F47F0129433846FFF746FDC4
:1051D00007F108053146381DC8F80050FFF73EFDBD
:1051E0001EB10A9A2846FFF755FD083C2544C8F829
:1051F0000050D9E7846E0120DBCD0000806E0120D5
:105200000A4B0022C3F8002101225A60D3F8002182
:10521000002AFBD00022C3F80C2101229A60044B23
:105220000222C3F880211A60704700BF00100040BE
:1052300000E100E0074B0222C3F88020064B002269
:10524000C3F8102101221A61D3F81021002AFBD0E3
:10525000704700BF00E100E00010004008B50449BD
:105260000A780AB1FFF7E6FF0020087008BD00BF0A
:10527000896F01204FF08053586E400040F00100CC
:1052800070470000024B1868400040F00100704772
:105290000C700120024B1868400040F0010070477C
:1052A00024000020024B1868400040F001007047C5
:1052B0001070012070B504460D461646FEF7F2F94F
:1052C0004FF0805301225B6E6270E270020A23F09D
:1052D0000043A271020CE2711A0A0021607163722C
:1052E000000EA2721A0C1B0E2670A170257120727E
:1052F000E272237370BD000010B5054C204605F026
:10530000F3FF01462046BDE81040FEF7B8BE00BFDF
:1053100015700120104B1B685A1C10B514D0CBB16E
:10532000012B13D0022B13D0042B13D00B4C0C4A9F
:10533000052B08BF1446204605F0D6FF014620463F
:10534000BDE81040FEF79BBE064CF4E7044CF2E7C4
:10535000054CF0E7054CEEE72800002051CF000097
:1053600057CF00004CCF00001FC6000018C6000039
:1053700010B521480278002A3DD14FF08043C3F890
:10538000002101221A60D3F80021002AFBD01B4B18
:105390001B4C00220721C3F80C25C3F80815194936
:1053A000C3F81025C3F81C15C3F824250121C3F840
:1053B0002C250822C3F83015C3F81425C3F8184566
:1053C0000224C3F834454FF6FF74C3F83C450E4C35
:1053D000C3F838451824C3F85445C3F80423D3F858
:1053E000002242F01002C3F80022084AC3F8042544
:1053F000FFF706FF017010BD896F0120001000400B
:105400002000040274696275211001008A6F012076
:10541000F8B5104B1B7804460BB9FFF7A9FF0E4EE9
:105420003378ABB10D4A1278D21A02F003010C4A5C
:1054300002EB411202F1200710685168254603C5AE
:105440000832BA422C46F7D1013B33700120F8BD37
:105450001846FCE7896F012014700120886F012035
:105460008A6F012030B5002889B02ADD0D6815F05B
:10547000010426D1042D26D92B6803F00F03092B34
:1054800021D16B683F2B1EDD6846FFF7C1FFB0B12D
:105490009DF800200435A242A8BF1DF8043004F195
:1054A0000104A6BF5B0043F001030123202C45F853
:1054B000043FF0D1054BDDF809201A60042009B043
:1054C00030BD0020FBE72046F9E700BF1070012047
:1054D00030B5384B1B788BB00BB9FFF749FF02A8EA
:1054E000FFF796FF10B900200BB030BD9DF80830D3
:1054F0000B2BF8D99DF80930012BF4D19DF80B3016
:10550000012BF0D12C4D2D4C2D4ADDF8111000232C
:105510002B6023709DF80C3013602A4A116023B968
:10552000DDF815302B6000230FE0012B11D1DDF8E1
:1055300015309DF819202B600DF11A010E239342AE
:10554000A8BF134600229A4230D10022E254042020
:10555000CAE7022B05D19DF8152012230DF1160183
:10556000EDE7042B0DD10AAA6B4652F8130D5168D2
:1055700003C3DDE9000103F0A5FA05F05BFA28603A
:10558000D1E7052BCFD10AAA6B4652F8130D51680B
:1055900003C3DDE9000103F095FA05F04BFA9DF82D
:1055A0001D2028600A230DF11E01C8E7885CA05465
:1055B0000132C8E7896F01200C70012015700120AD
:1055C000280000201070012010B5154B1B780446F0
:1055D0000BB9FFF7CDFEFFF72DFE124B0022C3F8EB
:1055E0000445C3F8002101221A60D3F80021002AE3
:1055F000FBD00022C3F80C2101229A60094AD2F89C
:105600000C31002BFBD0084B1978084B03EB4113EE
:10561000C2F80435FFF70EFEBDE81040FFF7F0BDFD
:10562000896F012000100040886F01208A6F0120DF
:1056300000B5002889B01DDD0B6813F0010219D1F7
:10564000042B17D9196801F00F01092912D15968E3
:105650003F290FDD043353F8040F10F0010118BF88
:10566000C0F347010DF802100132202AF3D1684639
:10567000FFF7AAFF002009B05DF804FB002810B571
:1056800011DD0C68E3070ED56410532C0BD8074BC3
:105690001B780BB9FFF76CFEFFF7CCFD044BC3F88A
:1056A0000845FFF7ADFD002010BD00BF896F012048
:1056B00000100040002810B50DDD0C68E3070AD586
:1056C0006410FF2C07D8054B1B780BB9FFF750FE71
:1056D000034BC3F82445002010BD00BF896F012093
:1056E00000100040002813B515DD0C68E10712D545
:1056F00064100A4A0A4B072CCDE900230BD8094B4A
:105700001B780BB9FFF734FE02AB1C44064B14F9AF
:10571000082CC3F80C25002002B010BDE2ECF0F418
:10572000F8FC0004896F01200010004070B50028CB
:1057300088B020DD086810F001041CD104281AD9B3
:10574000036803F00F03042B15D1FEF77BFA06461E
:1057500005F0CAFD122828BF1220054600F10D02EF
:1057600002216846FFF7A6FD8DF80D50A54205DC25
:105770006846FFF729FF002008B070BD0DEB040359
:10578000325D9A730134F1E72DE9F041012888B0C8
:105790000D4630DD086810F001042CD104282AD908
:1057A000036803F00F03042B25D14B68DB0722D5D8
:1057B000FEF748FA804605F097FD6D680E2828BF71
:1057C0000E206E10074600F1110201216846FFF716
:1057D00071FD6B128DF80D606D14360E8DF80E3064
:1057E0008DF80F508DF810608DF81170A74206DC0F
:1057F0006846FFF7E9FE002008B0BDE8F0810DEB38
:10580000040318F804209A740134EFE730B5002837
:1058100089B016DD0C68E30713D5651068461022C1
:105820000021FFF747FD63128DF80D5064142D0E13
:1058300068468DF80E308DF80F408DF81050FFF748
:10584000C3FE002009B030BD174BD3F8002122B1B0
:105850000022C3F8002101229A60D3F80C2102B380
:105860000021C3F80C11D3F80024012A0F4A19D1E2
:10587000D3F848355B4213600D4A1378032B9CBF65
:10588000013313700B4A1378013303F003031370D1
:10589000094A02EB4313044AC2F80435024B0122C1
:1058A0009A6070471160F9E7001000402400002062
:1058B00014700120886F01208A6F0120024A03487A
:1058C000102100F08BB800BFCCCE0000C3CE00008A
:1058D000044A05491368C8540133C3F3090313602C
:1058E000704700BF447401204470012070B5114915
:1058F000114A0B68834202DC00230B6017E0855CD1
:10590000A5F1FA06012E00F1010405D89C420FDA38
:10591000A55C013D1F2D01D92046EBE70446151A71
:10592000165D2E550134A342FADC181A086070BDCA
:105930001570FAE7507801205074012008B5FDF782
:10594000A9FE074B1A68824284BF00221A601B68B6
:10595000C01A44F62063984294BF0020012008BD7D
:105960004070012070B5094C094D0A4E23682A6821
:10597000934200D170BDF05CFEF7ECF80028F9D03E
:1059800023680133C3F309032360EFE74874012060
:10599000447401204470012070B5074E074D044641
:1059A00033682A689B1ADB43C3F30903A34200DB75
:1059B00070BDFFF7D7FFF3E744740120487401205E
:1059C00010B5FFF78BFA044608B9204610BD83785E
:1059D0001D2B08BF0446FFF781F9F5E7F0B5074D29
:1059E0002B680B2B08DC064F0C245C433E19C6E9E0
:1059F0000112013338512B60F0BD00BF4C740120FF
:105A0000009001202DE9F04FB3B0044605F06CFC86
:105A1000012803D8002033B0BDE8F08F23785B2B3A
:105A2000F8D101382518235C5D2BF3D101343A21DC
:105A3000204605F042FC06460028EBD0071B002F4D
:105A4000E8DD21463A46684605F068FC32AB711C39
:105A500000241F446D1AA54207F8C84CDADD2A4617
:105A600019A805F05BFC32AB1D44134B134ED3F861
:105A7000009005F8644C4FF00C0AA145CADD0AFB02
:105A800004F36946985903EB060805F023FC054624
:105A900018B9D8E90187454501DB0134EDE719A9BB
:105AA00057F8350007EBC50B05F014FC10B9DBF80F
:105AB0000400B0E70135EEE74C74012000900120AE
:105AC00008B5FBF7A7FCFFF78BF8FBF7C7FCFDF762
:105AD000BBFFFEF78FFCFEF7DFFCFFF7EFFE01F0E8
:105AE000D3F801F017FE01F041FEBDE8084002F0D6
:105AF00077B8000008B54FF416620021034805F09E
:105B000053F8034B00221A6008BD00BF087D012036
:105B1000AC050020174B53F83000836803F07F0377
:105B20001C2B70B50D46144601D0002070BDC36813
:105B300003F07F02042AF8D1026902F07F02192AD9
:105B4000F3D11B0A00EB83001030FEF77BF80378DB
:105B5000064633B105F0C8FBA042E6D10023A342BC
:105B600001DB0120E2E7F15CEA5C9142DDD1013327
:105B7000F5E700BF68860120064B074A1B681268DC
:105B80009B1ADB43C3F309038342D4BF00200120E7
:105B9000704700BF4474012048740120F8B50746DF
:105BA0000E4614461D4673B90320FFF7E5FF10B3F8
:105BB000FA20FFF78DFEF8B2FFF78AFEF0B2BDE8DB
:105BC000F840FFF785BE501DFFF7D6FF98B1FB20C8
:105BD000FFF77EFEF8B2FFF77BFEF0B2FFF778FE2C
:105BE000E0B2FFF775FEC4F30720FFF771FE2E4603
:105BF000731B9C4200DCF8BD16F8010BFFF768FE32
:105C0000F6E70000F8B50C4E0C4D0024F027336881
:105C1000A34203DCBDE8F840FFF76CBF07FB04F3C9
:105C200059195B5D2BB100231A4649781120FFF703
:105C3000B5FF0134EBE700BFAC050020087D012073
:105C4000F8B50E4C0E4E07460025BC4205F1010585
:105C500011D0237853B100231A4661781120FFF741
:105C60009DFFF0220021204604F09EFF0A2D04F142
:105C7000F004EAD1F8BD3560F8E700BF087D0120E7
:105C8000AC0500202DE9F04F12F00106ADF54F7D77
:105C900082468B4617D001238DF8143042FA03F365
:105CA00054128DF8153052141B0E8DF817208DF8F4
:105CB00018308DF8164005AB0522FFF76FFF0DF584
:105CC0004F7DBDE8F08F042A2CD9116801F00F0335
:105CD000042B38D105AD022310462B70FDF7B2FF1F
:105CE000044605F001FBB0F5487F034604F1FF319F
:105CF000A8BF4FF448739E4206F101020DD1B0F5E2
:105D0000487F06D96D4B19889B78ADF832138DF812
:105D100034332B4659465046CFE7164611F8012F2B
:105D2000AA55E8E740F0C680A2F1040CDCF10002BD
:105D30004FF0030342EB0C028DF814308DF8152060
:105D400005AB0222E6E7092B40F0918015460423BB
:105D50008DF8143055F8043F4FEA6308B8F1200F6E
:105D60008DF815804FEA6323A8BF4FF020088DF807
:105D700016308DF8178006AC03220521B04502DCF1
:105D800005ABE21AC6E755F8040F10F0010706D17B
:105D9000042847D9036803F00F03022B0DD14FF0FD
:105DA000010323704310637047121B0E4014A77049
:105DB000E070237105340136E0E7042B30D123462F
:105DC0004FF0020C03F802CBCDE9012100930393BD
:105DD000FDF738FF814605F087FA0C28DDE901213F
:105DE0000AD8009B6070874201D1DC19E3E719F8FB
:105DF0000740DC550137F6E723460C2003F8010F76
:105E000009F1FF3009F1080910F8017F03F8017F5B
:105E10004845F9D12E23E372237363730E34CAE726
:105E2000012B08D12346071F03F8022B7842784143
:105E300060701C46BFE7092B09D104232370436817
:105E4000581060705B12A370E7700434B3E7032B43
:105E50000AD121700368C3F30F10C3F34173C3EB7E
:105E6000800363701B12EEE727700134A3E7032B56
:105E70007FF425AF05238DF81430C1F30F13C1F360
:105E80004171C1EB830164294FEA21238DF815107C
:105E9000A8BF64218DF816308DF8171003328E429A
:105EA00005AB01DB0A1D35E7334412F8010F187109
:105EB0000136F4E7002A7FF402AF35E782C2000022
:105EC0000F4970B5F022002402FB04135D7885426F
:105ED00003D001340A2CF7D170BDF02218460021FE
:105EE00004F062FE074A1368013BA34200D114602C
:105EF000002329461A461120BDE87040FFF74EBE28
:105F0000087D0120AC05002030B5B3B032AC0223CF
:105F1000054604F8C83D05F0E7F9C72828BFC720A3
:105F2000691E0023984207DC421C2346FE211420F0
:105F3000FFF734FE33B030BD013311F8012FE254C6
:105F4000F0E770B5B2B032AC0223054604F8C83DA4
:105F500005F0CAF9C72828BFC72006460023681ED7
:105F60009E420BDC06F13200FFF716FD2346721C41
:105F7000FF211420FFF712FE32B070BD013310F87C
:105F8000012FE254ECE700002DE9F04F0128B9B0F1
:105F90008146884603DC1B20FBF700FC57E00868BD
:105FA000C20729D4042827D9036803F00F03042B60
:105FB00022D1FDF747FE0546D8F80400C3071DD4DB
:105FC00004281BD9036803F00F03042B16D1FDF737
:105FD00039FE0646204B1B6803930027039BBB42F8
:105FE0000EDC00962B461D4AC82106A805F002F9D2
:105FF00006A8FFF7A6FFCEE7194DDDE7184EE9E743
:106000000C237B43174A2946985803EB020B05F0F3
:1060100061F9044618B9DBE9013A9C4201DB01371A
:10602000DCE70AEBC40231465AF8340005930492C7
:1060300005F050F9DDE90423834658B9536808F1A7
:106040000801A9F102009847074BC3F800B039B026
:10605000BDE8F08F0134E0E74C74012028D0000047
:1060600099C7000000900120546D01202DE9F041F6
:106070001F4F204AD7F8008005460023F02098459E
:106080000EDC0024F02000FB04F15318565C8EB1A6
:1060900001340A2CF7D11848BDE8F041FFF751BF91
:1060A00000FB03F154186478AC4201D1515CE9B9AA
:1060B0000133E4E7F0223146184604F075FD0F493C
:1060C000457051F8351085700222A0450270C0E974
:1060D0000212C0E9046601DC01343C600023294659
:1060E0001A461020BDE8F041FFF758BDBDE8F08129
:1060F000AC050020087D012071D4000068860120D5
:1061000070B5FFF77FFD094EFF246FF0070505FB13
:10611000046393F8FC37043B012B03D8E043C0B27F
:10612000FFF7A4FF013CF2D170BD00BF68860120DB
:106130002DE9F04106460F46FDF7A1FF0D4BDFF8B4
:1061400038801860002408EBC4031B79062B01D0AB
:10615000032B09D1E5B23A4631462846FFF7DAFC6F
:1061600010B12846FFF782FF0134FF2CEBD1BDE8C8
:10617000F08100BF0800002068860120F8B5094FB3
:106180000546FF246FF0070606FB047393F8FC37FF
:10619000AB4203D1E043C0B2FFF768FF013CF3D14B
:1061A000F8BD00BF688601202DE9F84FFDF772FAAF
:1061B000584B1A68824284BF00221A601A6842F261
:1061C0000F71821A8A420BD95349186000235A185A
:1061D0001279073A022A0FD90833B3F5FF6FF6D1C7
:1061E000BDE8F88F0720FFF7C9FF8AF800802EE08E
:1061F0000820FFF7C3FF3FE0FDF754FA002814BF63
:10620000044601240020FDF7F7FA81460020FDF73F
:1062100007FB424D424E0746B9F1000F17D02B68DD
:10622000002B70D133682C60002B6FD0DFF8F8B0F2
:10623000DFF8F0A09BF800304FF00108002BD1D11F
:106240000920FFF79BFF8AF800808BF80080AFB130
:1062500033689BB92B6834601BB3DFF8C8B0DFF834
:10626000C8A09BF800304FF00108002BC0D10920D6
:10627000FFF784FF8BF800808AF800802B6883B1D9
:10628000284A1178904661B99C4238BF2C602B682F
:10629000E31A312B05D90720FFF770FF012388F897
:1062A0000030326882B1204B1978984661B9A24219
:1062B00088BF34603368E41A312C05D90820FFF711
:1062C0005DFF012388F800302B685BB1B9F1000F46
:1062D00008D1144C227812B90720FFF74FFF002392
:1062E0002B6023703368002B3FF47AAF002F7FF4CC
:1062F00077AF0D4C227812B90820FFF73FFF00233B
:10630000336023706CE7002FA2D1B9E7002FA1D131
:10631000B4E700BF3C700120688601202C7001208A
:1063200034700120307001203870012037B50546E7
:10633000FFF768FC02A8002440F8044DFDF73EFA80
:1063400021462046FEF796F9FEF7AAFBFDF77CFAF8
:10635000FDF756FBFDF770FBFEF73EFCFDF7C4F9B9
:1063600025B1FDF71FFC0248FFF7EBFD03B030BD80
:1063700062D40000002301461A461120FFF70EBC2C
:1063800007B513128DF801208DF802301314120E88
:106390008DF800108DF803308DF8042001466B460F
:1063A00005221320FFF7FAFB03B05DF804FB0A4651
:1063B00001461220FFF766BC70B505460C46FDF796
:1063C0007DF958B104F13200FFF7E6FA2B46224678
:1063D00000211B20BDE87040FFF7E0BB70BD10B48A
:1063E000144603460A46142021465DF8044BFFF785
:1063F000D5BB000030B5084C01444FF0FF33884254
:1064000001D3D84330BD10F8015BDAB26A4054F8CA
:10641000222082EA1323F2E744D00000FE2837B599
:10642000044614D80B4B53F8300080B14168083053
:106430008900FFF7DFFF02AD45F8040D0920FFF7E3
:10644000ABFA2B46042221461720FFF7A7FB03B027
:1064500030BD00BF68860120F8B50746FFF7B0FAE7
:106460004FF0FF3504460CB92846F8BD2668C6F340
:106470000743152B0CD104F10801384604F02AFF1C
:1064800008B9C6F307252046FEF728FC0446EAE7CC
:106490001D2B08BF4FF0FF35F5E700002DE9F04F49
:1064A000C24CC34D9DB0FFF75DFA2068C0F5806116
:1064B0002844FDF737FB23680344064623607BB17D
:1064C000BC4F002E0FDC2B78FA2B40F0358123686F
:1064D000022B16DCFFF732FA10B10120FFF706FAA3
:1064E0001DB0BDE8F08F2068C0F580612844FDF73D
:1064F00019FB2368034406462360FDF7CBF8386098
:10650000DFE76878AC78831E182B00F20B81DFE898
:1065100013F019002D003100350038004100090149
:106520004B0080008A008E00A400E500F6000901FF
:10653000090109010901090109010901090109010B
:1065400009010401FF2C0FD02046FFF7B9FC9A4A3D
:10655000002342F8343002EBC402214613711320A9
:1065600000931A46FEF7F2FD0320B7E72046FFF737
:106570007DFDF9E72046FFF7A3FCF5E7FFF7C0FD37
:10658000F2E7FFF73FFB0020FFF7D0FE8B48FFF755
:10659000D8FCE9E7632CE7D8894B214653F824203F
:1065A0001520FFF76FFBDFE7FFF70AFA6FF0070828
:1065B0000446002CD8D02768C7F30743152B04D016
:1065C0002046FEF78BFB0446F3E704F1080630464D
:1065D00004F08AFE05460530FFF7DEF9FB20FFF7E1
:1065E00077F91D20FFF774F9C7F30720FFF770F95B
:1065F000E8B2FFF76DF9C5F30720FFF769F9A8EBDB
:106600000407F3199D42DBDD16F8010BFFF760F973
:10661000F7E7002300931A4619461D20FEF796FD62
:10662000FDF7C0FAA0E72046FFF7F8FE9CE7FDF76C
:1066300047F8644A00906421634B03A804F0DAFD34
:10664000022303A88DF80C3004F04EFE03AB024683
:1066500000211620FFF7A2FA86E75C4BDFF858818D
:106660001F680025FA2397FBF3F758F8354008EB2D
:10667000C50354B3D4F8049093F804B04FEA8906E4
:10668000B01DFFF789F9FB20FFF722F9012006F181
:10669000010AFFF71DF9E8B2FFF71AF95FFA8AF06D
:1066A000FFF716F9CAF30720FFF712F95846FFF76C
:1066B0000FF908342644A6420BD8FFF753F909FB1B
:1066C00007F001F0CFFFFFF74DF90135FF2DCCD1D9
:1066D0004AE714F8010BFFF7FBF8ECE70024FFF79B
:1066E00091FA2246214600942346DA20FEF72EFD39
:1066F0004FF4FF622146304804F056FA90E7012C2F
:1067000002D1FEF713FB2FE7022C02D1FEF71CFD8E
:106710002AE70120FFF70AFE26E700231A46214652
:106720001A2097E7A0F1C803052B3FF61DAF002202
:106730001146FAF79DFE17E7FB2B7FF4CEAE2268D9
:10674000042A7FF7C7AEB5F8037040F2F6339F42D4
:106750003FF7C3AE3B1D9A427FF7BCAEEB5CFE2B0E
:106760007FF4BBAE6878AC781B2807F1FF367DD08C
:1067700030D8072861D008283AD001282FD1FF2C23
:1067800011D02046FFF79CFB6D79114B00932146F9
:10679000BB1E2A460A20FEF7D9FC074B43F83400FB
:1067A00003EBC4042571781D98E600BF50780120E2
:1067B00050740120407001206886012044D40000FC
:1067C000608E01205BD4000056D40000040000203D
:1067D000567401201D285BD04DD31E2870D0A0F127
:1067E000C803052BDFD83F4A3146FAF741FEDAE706
:1067F000632CD8D86B79022B0CD0032B14D0012B2F
:10680000D1D1D5F80630384A5B0043F0010342F895
:106810002430C8E7002EC6DDB91E3448FDF72FFC32
:10682000314B43F82400BEE7AB79002B2E4B0CBF55
:106830000022042243F82420B5E7632EB3DC32465D
:10684000284903A804F08CF91CAB1E4403A80023BC
:1068500006F8643CFFF700FE0028A4DB224B21462B
:1068600053F820201520FFF70DFA9CE731461D480C
:10687000FFF75EFC97E7FF2C95D06A79022A92D841
:106880001A4B00932146BB1E0B20FEF75FFC8AE7E4
:10689000632EA8BF6326002303A99E420BDC1CAA1B
:1068A00026EAE6731344002203F8642C15200091B5
:1068B000731C2146E9E7EA185279CA540133ECE720
:1068C000012C7FF470AF002E7FF76DAF6B791BB199
:1068D000322BA8BF32231C4664235C43044B1C604C
:1068E00061E700BF55740120608E012056740120BD
:1068F00004000020084B01221A60084A1368002B8C
:10690000FCD0074B1868042390FBF3F006384000D6
:1069100040F00100704700BF00C0004000C10040CF
:1069200008C500400120704710B5064C204601F014
:106930006DFA0549204601F0CFFA044B01221A6096
:1069400010BD00BF107B0120801A06005478012082
:1069500010B5064C204601F059FA0549204601F0D1
:10696000BBFA044B01221A6010BD00BFCC7B012092
:10697000801A0600587801201FB500210E20FCF770
:10698000A5FE01210F20FCF7A1FE01210D20FCF73F
:106990009DFE1D4801F092F91C4B1D491B681D4AC4
:1069A0008B4212780FD84FF00073019300230393AA
:1069B0008DF8082004AB13E90E00134805B05DF80C
:1069C00004EB01F091B914498B4202D84FF0806377
:1069D000EBE712498B4202D84FF00063E5E710491C
:1069E0008B4202D84FF08053DFE70E498B4202D82A
:1069F0004FF00053D9E70C498B4294BF4FF08043CE
:106A00004FF00043D1E700BFF07A012030000020B2
:106A100048E801002C00002090D0030020A10700CE
:106A200040420F0080841E0000093D00002814DD54
:106A30000B68DA0711D50D4A5B10012813600C4A68
:106A400009D04B68D90706D55B10022B09D0032B60
:106A500009D0012B03D002231360002070470023CC
:106A6000FAE70323F8E70123F6E700BF3000002030
:106A70002C00002008682DE9F843C30704D40D203A
:106A8000BDE8F843FAF78ABE4010FCF743FE051E46
:106A90002FDBFCF719FEA8422BDB00212846FCF770
:106AA00015FE4FF4FA620121284601F013FE00B3EF
:106AB000DFF86C8000244FF00109002707264FF40F
:106AC0007A720121284601F005FE90B12828C4BF42
:106AD00009FA06F31F4316F1FF36F0D204F80870E6
:106AE0000134052CE9D1012206210920FDF746FADF
:106AF00008B900200FE003460B2243F8042F074992
:106B000000F1180411F8012F520042F0010243F87D
:106B1000042F9C42F6D1BDE8F88300BF5B780120CA
:106B20005C7801200028F8B521DD0C6814F001061E
:106B30001DD1042C1BD9236803F00F02032A16D1A0
:106B4000C3F30F15C3F34173C3EB8505FFF714FFC0
:106B5000084F0334B54207DD14F8011F384601F031
:106B6000D0F801362070F5E7024801F0C9F800209E
:106B7000F8BD00BFF07A012010B50468E30704D423
:106B80000D20BDE81040FAF709BE6410FF2C01D9B2
:106B90001720F6E7FFF7F0FEE1B2044801F0B1F884
:106BA000024801F0ADF8002010BD00BFF07A0120CE
:106BB00038B5074DFFF7E0FE0021284601F0A1F8A7
:106BC0000446284601F09CF8600040F0010038BD02
:106BD000F07A0120274A82B001210023ADF8063067
:106BE000C2F8F015C2F8001519461A0102F18042E8
:106BF00002F5E0420133082BC2F81415C2F8101553
:106C0000F3D11C4B4FF4E062C3F818250422C3F8FB
:106C10001425C3F810250DF10602C3F82C26012215
:106C2000C3F830261A60D3F80021002AFBD00022D6
:106C3000C3F8002101225A600E4B1A46D3F8041102
:106C40000029FBD00021C3F8041101219960D2F87A
:106C50001431002BFBD00020C2F81401C2F800054B
:106C6000BDF806301BB28342C8BFA3F50B704000CD
:106C700002B070470070004008B5FFF7ABFF40005E
:106C800040F0010008BD0000024A03480E21FEF753
:106C9000A5BE00BF88D40000F8D400000C4B1B68D0
:106CA00070B506460D4614460BB9FFF73DFEF1B22E
:106CB000084801F08FF9E9B2064801F06FF8E1B237
:106CC000044801F06BF80348BDE8704001F0EDB9ED
:106CD00054780120107B012008B50368D90705D539
:106CE0004168CA0702D58268D00704D40D20BDE8E8
:106CF0000840FAF753BD5810802801D91520F6E74F
:106D00004910FF2901D91620F1E75210FF2A01D9B5
:106D10001720ECE7FFF7C2FF002008BD0C4B1B68F3
:106D200070B506460D4614460BB9FFF711FEF1B2D9
:106D3000084801F04FF9E9B2064801F02FF8E1B236
:106D4000044801F02BF80348BDE8704001F0ADB9EC
:106D500058780120CC7B012001282DE9F0415EDD2F
:106D60000D68EA075BD52F4B4C681B686D100BB99B
:106D7000FFF7DAFDE9B22C4801F02CF914F0010616
:106D800013D06410FF2C02D91720FAF707FDE1B2E7
:106D9000254801F003F8244801F087F918B12320B1
:106DA000FAF7FCFC0020BDE8F081042CF3D923683D
:106DB00003F00F02092A1AD154F8047FDFF8688023
:106DC0007F10B742E7DD54F8045FEB070BD56D1079
:106DD000FF2D02D91720FAF7E1FCE9B2404600F096
:106DE000DDFF0136EDE71720FAF7D8FCF9E7032AB3
:106DF000D1D1261DC4F1FF24C3F30F1504F57F0480
:106E0000C3F34173084FC3EB8505FC343319AB4220
:106E1000C1DA16F8011B384600F0C0FFF6E7012082
:106E2000C1E700BF54780120107B012038B5134B17
:106E30001B6804460D460BB9FFF776FDE4B2214608
:106E40000F4801F0C7F8E9B20D4800F0A7FF002194
:106E50000B4801F0C9F808B1404238BD0122214673
:106E6000074801F0B4F8064800F08FFF0028F4D07E
:106E70000348BDE8384000F08BBF00BF54780120C4
:106E8000107B012008B50368D90702D54168CA07FD
:106E900004D40D20BDE80840FAF780BC58108028C3
:106EA00001D91520F6E74910FF2901D91620F1E78D
:106EB000FFF7BCFF400040F0010008BD38B5124BA1
:106EC0001B6804460D460BB9FFF742FDE4B22146AC
:106ED0000E4801F07FF8E9B20C4800F05FFF0B4864
:106EE00001F0E3F808B1404238BD012221460748CD
:106EF00001F06DF8054800F048FF0028F4D0034881
:106F0000BDE8384000F044BF58780120CC7B012018
:106F100038B50D211D20FFF7D1FF5A28174C0CD191
:106F2000012222702A211D20FFF7F8FE022001F025
:106F300099FB134B01221A6038BD0F211920FFF76E
:106F4000BDFF332805D1022323708F222021192071
:106F5000EAE70D211E20FFF7B1FFC7280AD103255C
:106F600000222A211E202570FFF7D8FE2A462A215A
:106F70001E20D9E700232370D8E700BF340000208B
:106F800064780120002838B504DC1C20BDE83840B6
:106F9000FAF704BC0B6813F0010401D10D20F5E7EA
:106FA0005B10012B2ADD022B03D0052BB4BF02247A
:106FB0000324194B1B680BB9FFF7AAFF174B93F972
:106FC0000050022D1CD0032D1ED0012D11D1032CF9
:106FD00008BF022400222A211D20FFF79FFE22461F
:106FE0000E211D20FFF79AFE2A462A211D20FFF7B9
:106FF00095FE022001F036FB002038BD0024D8E7C2
:10700000220123211920F2E7032C14BF2246022279
:107010000E211E20EBE700BF647801203400002021
:10702000204B1B6810B504460BB9FFF771FF1E4BD0
:1070300093F90030022B0AD0032B25D0012B26D147
:1070400021461D20FFF73AFF4FF0FF3405E0012CE9
:1070500013D129211920FFF731FF7F28C8BFA0F5E0
:1070600080706FF07E039842B8BF1846C82358431B
:107070007F2390FBF3F0604310BD032C0BD12B2139
:107080001920DFE72D21FBE721461E20DAE74FF02C
:10709000FF340020EAE7052CF4D04FF0FF34002045
:1070A000DFE700BF647801203400002008B501202C
:1070B000FFF7B6FF400040F0010008BD08B503200F
:1070C000FFF7AEFF400040F0010008BD08B5052005
:1070D000FFF7A6FF400040F0010008BD38B5134B94
:1070E0001B6813B90120FFF79BFF114B93F9003088
:1070F000013301D1FFF70CFF0120FFF791FF044698
:107100000320FFF78DFF05460520FFF789FF6D433C
:1071100004FB045400FB004003F072F901F0EEFDA3
:1071200003F088FC400040F0010038BD6478012085
:1071300034000020234B1B6870B506460BB9FFF7DF
:1071400007FC214C94F9001000291BDA0F211920AB
:10715000FFF7B4FE332811D11C4B68221A701C4B68
:107160001E2500221A7060210C2228462570FFF788
:10717000D5FD022261212846FFF7D0FD94F90010C9
:1071800000291EDBC9B21348124D00F023FF0F4B3C
:107190001048197800F002FE0E4800F086FF2178B2
:1071A0000C48062200F013FF741E0536284600F036
:1071B000ECFD30B1284600F0EBFD04F8010FB442BD
:1071C000F4D170BD58780120350000203700002030
:1071D00036000020CC7B012073B500236846009365
:1071E000ADF80430FFF7A6FFFFF758F91C4B9DF8E8
:1071F000015093F900609DF802009DF800309DF861
:1072000003409DF804209DF8051006B345EA0323CA
:1072100044EA00201BB200B241EA0222114991F96E
:107220000010102912B202BFDB105210C010002B48
:10723000B8BF5B420028B8BF4042002A1844B8BF1C
:1072400052421044400040F0010002B070BD43EAD9
:10725000052340EA04201BB200B242EA0122DDE726
:1072600036000020350000200128F8B535DD0F6814
:10727000FB0732D54D6815F001062ED1042D2CD90F
:107280002B6803F00F03092B27D16C68144B641093
:107290001B68202CA8BF20240BB9FFF745FBC7F3C0
:1072A000470122460F480F4F00F091FE0435A642D9
:1072B00011DA0C4800F069FD18B9700040F00100C7
:1072C000F8BD384600F064FD400040F0010045F88C
:1072D000040F0136EBE76000F0E70120F0E700BFA4
:1072E00054780120107B01200A4B0B4A30B5D3F8AB
:1072F00034450A4BA34208BF1346013B0246FF2414
:10730000151AA94205DD13F8015F02F8015B1C7034
:10731000F6E730BD008002406C7801206C790120D6
:10732000064B01225A60DA60D3F85821002AFBD0BC
:107330000022C3F80025024B1A607047008002400B
:107340006878012038B52C4B1B680D4623B92520E1
:10735000BDE83840FAF722BA012801DC1C20F7E723
:107360000C68E10709D4042C09D9236803F00F0342
:10737000DA1E012A05D92420EAE70223F8E70123CF
:10738000F6E76A68D20701D41120E1E7042B0CD19B
:107390002046FCF757FC03F0A7FF6A685210013A39
:1073A00001D4824209DB1220D2E72068C0F30F1219
:1073B000C0F34170C0EB8200EFE71049D1F82031F3
:1073C000C3B1801A80280E4AA8BF8020043400234D
:1073D000834204DA14F8015B9D540133F8E700237B
:1073E000C1F84805C1F8203101238B60400040F00E
:1073F000010038BD1846F9E7687801200080024096
:107400006C7A012070B5174D174CD5F83435174EEE
:107410009C4214BF234633464FF480721846FF2126
:1074200003F0C2FB4FF48073C5F83405C5F8383556
:107430000023C5F8083101232B60D5F834058442B8
:1074400008BF344604F1FF00A21E0178FF2900F1B5
:10745000FF3301D19A4202D1001B013070BD1846A2
:10746000F3E700BF008002406C7901206C780120B6
:10747000002838B504DC1C20BDE83840FAF78EB986
:107480000D68EB0706D4042D04D92B6803F00F0315
:10749000032B01D02420EFE7124B1B680BB92520EA
:1074A000EAE7114BD3F808310BB9012038BDFFF7DB
:1074B000A9FF041EF9D001DA1B20DDE7284650F8A9
:1074C000043BC3F30F12C3F34173C3EB82039C422B
:1074D00028BF1C462146FFF707FF600040F001006F
:1074E000E4E700BF68780120008002400028F8B57A
:1074F00004DC1C20BDE8F840FAF750B90968CB0756
:1075000001D40D20F6E71E4D1E4C2B68491023B107
:10751000D4F800350BB1FFF703FF1B4B1A68C4F812
:1075200014255B68C4F80C354FF486734B43C4F8DC
:107530002435164B4FF48072FF21184603F034FBBC
:107540004FF48073C4F83405C4F83835104BC4F8D0
:1075500044358023C4F848352023C4F8003200267F
:1075600001270823C4F800350520C4F80861276006
:10757000C4F84865A76001F075F82F603046F8BD83
:10758000687801200080024024D800006C78012037
:107590006C7A012070B5124E04460D46002D14DDA4
:1075A000D6F8203193B1802D10DC0E4B621914F8FF
:1075B000011B03F8011FA242F9D1094B0022C3F8B5
:1075C0004855C3F8202101229A6070BDFDF768FA82
:1075D000FEF7EAFDFEF762FF012001F043F8DDE768
:1075E000008002406B7A012006490A6808B52AB17A
:1075F000054BD3F800350BB1FFF792FE0020086071
:1076000008BD00BF687801200080024038B51C4BDF
:107610001B6823B92520BDE83840FAF7BFB8194BDD
:10762000D3F8083113B9184D284638BDFFF7EAFEE4
:10763000041EF8D001DA1B20EDE7E11C00228910BE
:107640000320FCF79BFC054608B90A20E3E7214626
:107650000430FFF749FEEB07E6D4042DE4D92A688D
:1076600002F00F03032BDFD104F00303C3F1040383
:107670005B0703F0C04322F0C04213432B60D3E703
:10768000687801200080024038000020002837B5CB
:1076900004DC1C20FAF782F803B030BD1C4B1B68D9
:1076A0000BB92520F6E7086810F001040CD0431050
:1076B000FF2B01D92820EDE702A8012100F8013DA8
:1076C000FFF768FF0020E7E7042813D9036803F0F9
:1076D0000F02042A10D1FCF7B5FA054603F004FEA8
:1076E0008028014603D92620FAF758F8EAE7284609
:1076F000FFF750FF2046CFE7032AFBD1C3F30F115A
:10770000C3F34173C3EB81018029ECDC0430EFE764
:1077100068780120024A03480621FEF75FB900BFDE
:1077200094D50000C4D500000020704701207047A8
:1077300000207047002070470020704701207047EC
:1077400000207047002070470020704700207047DD
:1077500000207047002070470020704700207047CD
:10776000002070477047704770470000024A034886
:107770000F21FEF733B900BFECD5000064D600003E
:107780000246104601320378013B1F2BF9D970479E
:1077900008B5FFF7F5FF0378002B39D0222B00F155
:1077A000010011D1037823B1222B00F1010204D191
:1077B0001046BDE80840FFF7E3BF5C2B02D14378D9
:1077C00003B1821C1046EDE73A2BF2D02C2BF0D0FF
:1077D0007B2B0BD1FFF7D4FF0378002BE9D07D2B57
:1077E00001D10130E5E7FFF7D3FFF5E75B2B10D0C0
:1077F0000246104612F8013B002BDAD0202BD8DDD0
:107800002C2B05D003F0DF015D2901D0222BF0D114
:1078100008BDFFF7B5FF0378002BCAD05D2BE0D081
:10782000FFF7B6FFF7E708B5F0B1FFF7A9FF037858
:10783000222B1AD07B2B1AD05B2B1AD0A3F130024B
:10784000092A05D92D2B05D14278303A092A07D8C3
:10785000032009E0742B0ED0662B0ED06E2B0ED0B9
:10786000181C18BF0120404208BD0420FCE702207C
:10787000FAE70120F8E70520F6E70620F4E70720FD
:10788000F2E738B5FFF77CFF03782D2B11D10130DB
:107890004FF0FF34431E00210A2501E005FB0121C2
:1078A00013F8012F303AD0B20928F7D904FB01F0C0
:1078B00038BD0124EEE710B51446FFF761FF0378E9
:1078C000222B02D000230B7010BD621E0130037802
:1078D000222BF7D0002BF5D05C2B07D0441C002ABC
:1078E000F0DD01F8013B013A2046F0E74378622BD6
:1078F00000F1020409D0662B09D06E2B09D0722B3F
:1079000009D0742B08BF0923E9E70823E7E70C2314
:10791000E5E70A23E3E70D23E1E710B50446FFF7A7
:1079200037FF0346A342184605D90278013A1F2AB9
:1079300003F1FF33F6D910BD08B590B1037883B1D8
:10794000FFF71EFF037803F0DF035D2B09D0FFF77D
:107950001FFF03782C2B08BF0130BDE80840FFF75C
:107960000FBF002008BD38B50D1E0DDD03785B2B61
:107970000AD10130FFF704FF0124A54205D0FFF72B
:10798000DBFF10B10134F8E7002038BD38B51546EB
:1079900009B100230B70F8B10378E3B1FFF7F0FEF3
:1079A00003782C2B044603D10130FFF7E9FE04468F
:1079B00023787D2B0FD019B12A462046FFF77BFF95
:1079C0002046FFF7E5FE03783A2B05D10130BDE8EC
:1079D0003840FFF7D5BE002038BD2DE9F0410D46F7
:1079E0009AB004462F789FB32E21284603F065FCF9
:1079F000804690B1461B303F092F13D82846FFF729
:107A000040FF01462046FFF7AEFF044604B3B8F13D
:107A1000000F1DD001363544E4E7284603F064FC2E
:107A20000646E8E723787B2B11D1601C642201A96C
:107A3000FFF7ACFF044658B13246294601A803F0CF
:107A40005BFC0028E2D02046FFF7A2FEEEE7002410
:107A500020461AB0BDE8F08138B50D1E04461CDD85
:107A6000FFF7E1FE012807D1601C012D00D138BDD0
:107A7000FFF762FF013DF8E702280ED10022114610
:107A8000601CFFF783FF012DF1D0FFF755FF0022A7
:107A90001146FFF77BFF013DF5E70020E7E7F8B56A
:107AA0000C1E074615461E4613DDFFF7BCFE0228D6
:107AB0000FD132462946781CFFF768FF012C00D110
:107AC000F8BDFFF739FF32462946FFF75FFF013C5B
:107AD000F4E70020F4E710B50446C8B1FFF750FE04
:107AE00003787B2B0AD10130002400221146FFF7D6
:107AF0004DFF68B1FFF74CFE0134F6E75B2B06D172
:107B000001300024FFF718FF10B10134FAE7002418
:107B1000204610BD002870B514DD0D68EB0711D5A7
:107B20006D10013DFDF7DAF900264FF0FF3460B922
:107B300016B3304603F0D8FB01463046BDE870402E
:107B4000FCF79DBA4FF0FF35ECE70368C3F307423B
:107B5000152A0BD1C3F307239C42B8BF1C469D4294
:107B600001D100F10806FDF7B9F8E0E71D2A04BFCE
:107B700000264FF0FF34F6E7601C400040F00100A3
:107B800070BD000010B508680C46FCF75BF8FEF706
:107B900063FC0028A2BF034B626843F8202000204A
:107BA00010BD00BF608E012008B50868FCF74AF8D8
:107BB000FEF752FC0028AABF024B012053F8200018
:107BC00008BD00BF608E012008B50868FCF73AF8D0
:107BD000FEF742FC0028ACBF0420002008BD0000D6
:107BE000024A03480421FDF7F9BE00BF00D7000098
:107BF000FAD6000008B5FBF731FFFBF7F7FFFDF7FA
:107C00005FFF0448FEF79DF9FDF7A4F9BDE80840C1
:107C1000FEF776BA4FD70000FBF768BB38B50025F2
:107C2000057329B90B4B0C4A0C48252102F02AFF99
:107C300001600B4951F82220027151F82330837101
:107C40009DF8103051F8233043710223C3718560D1
:107C500038BD00BF67D70000C6D7000075D7000049
:107C600024D80000037B23B943738373036101238A
:107C70000373704784B00DF1100C0CE90E009DF8F1
:107C80000810026800230129C2F80035039B12D0B6
:107C90000BD303290CD0C2F85435019BC2F824350C
:107CA0000123C2F8003504B0704743F00203F2E745
:107CB00043F00403EFE743F00603ECE710B5FFF7EA
:107CC000D1FF03688279C3F808254279C3F80C25EF
:107CD0000279C3F81025034BBDE810400ECBFFF727
:107CE000C9BF00BF047B012010B485B001AC84E89B
:107CF0000E0094E80E0005B05DF8044BFFF7BABF24
:107D000070470368C3F81C15D3F80821002AFBD07C
:107D1000D3F818050022C3F80821C0B2704700004C
:107D200007B5094B09490A484FF080421A60002202
:107D30009A6002221A710F2300930E220D23FFF77F
:107D40006DFF03B05DF804FB047B012000300240AE
:107D5000F07A01202DE9F84380460D46174601EBE5
:107D600002090C464C45A4EB05060BD0D8F80030B0
:107D700014F8011B1B68404698470028F2D1304692
:107D8000BDE8F8833E46FAE77047203000F03CBA81
:107D9000203000F02BBA203000F03CBA38B5437FD9
:107DA0000D460BB9002038BD00F16804204600F0F4
:107DB00039FA0028F6D12046294600F008FA0120B9
:107DC000F1E700002DE9F0411E4600254FF47A73DB
:107DD000C0E901530C4B044640F8203B8846174647
:107DE00000F0ECF904F1680000F0E8F99DF81830B3
:107DF00063769DF81C302676C4E90487A376657700
:107E00002046BDE8F08100BF0CD80000F0B5837EAD
:107E10002E4C2F4D0121C17654F82320437E54F877
:107E2000233012F0200F14BF2F464FF0A04702F06E
:107E30001F0213F0200F03F01F0308BF4FF0A045EF
:107E400002F5E07203F5E07340F20C6647F8226039
:107E500045F8236003694FF0CC72C3F82425036909
:107E60000622C3F80025827E036954F82220C3F855
:107E70000825427E036954F82220C3F80C2590F9A6
:107E80001830144A5C0903F01F03994004F16003A1
:107E900042F8231090F91830002BBDBF03F00F03F8
:107EA00002F6FC32D2189B18B5BF4023402213764D
:107EB00083F8002390F918300122590903F01F03B9
:107EC00002FA03F3034A42F82130F0BD24D800003F
:107ED0000003005000E100E0C37EA3B1036900226B
:107EE000C3F800250A4B99420ED90A4B994294BF18
:107EF0004FF080614FF0C8610369C3F8241503692E
:107F00000622C3F8002570474FF0CC71F4E700BF9C
:107F1000A086010090D003002DE9F0410446884678
:107F20001F461546002A50D000F12006304600F0CA
:107F300059F92369C3F88885236901221A622369E4
:107F4000C3F834652369C3F8385523691A60226978
:107F5000D2F84C311BB9D2F82431002BF8D00023D1
:107F6000C2F84C312269D2F85C311BB9D2F8243105
:107F7000002BF8D00023C2F85C3122696FB9D2F827
:107F8000243153B90123D3612369D3F84821002A4E
:107F9000FBD00022C3F8482109E001235361236983
:107FA000D3F80421002AFBD00022C3F8042123695E
:107FB000D3F8242112B10022C3F824212369D3F875
:107FC0003C052066C0B2BDE8F0811046FBE7012306
:107FD000FFF7A2BF10B5044680F8B010683000F07B
:107FE00001F90123637710BDF8B5002343770369D6
:107FF00090F8B020C3F88825036901261E62036942
:1080000000F168050446C3F8445528460F4600F0C1
:10801000FBF82369C3F8480523699E602369D3F8F8
:1080200050211AB9D3F82421002AF8D00022C3F82D
:108030005021284600F0E8F8236930B1D3F86021D8
:108040001AB9D3F82421002AF8D00022C3F86021FD
:1080500023696FB9D3F8242152B90122DA61236967
:10806000D3F84821002AFBD00022C3F8482109E0B8
:1080700001225A612369D3F80421002AFBD000228F
:10808000C3F804212369D3F8240168B10022C3F89E
:1080900024212369D3F8C404C3F8C404022803D0FC
:1080A00004280CBF03200420F8BD0121FFF79CBF6A
:1080B00070B54369D3F86421044692B100220125CA
:1080C00000F12006C3F864210577304600F08AF8F5
:1080D0006369C3F8346563694022C3F8382563696E
:1080E0001D636369D3F86821DAB10025C3F86851CC
:1080F00004F16806012363772577304600F072F8B3
:10810000D4F8B43003B19847636965773046C3F853
:10811000446500F079F86369C3F848056369012292
:108120005A636369D3F8042162B10022C3F80421C1
:10813000237F3BB16369D3F83C05D4F8B83020669F
:1081400003B198476369D3F8242152B10022C3F8E0
:1081500024216369D3F8D024C3F8D02463690122B1
:108160005A6170BD0148FFF7A3BF00BF107B01201B
:108170000148FFF79DBF00BFCC7B012007B514234A
:108180001322CDE900324FF0402211460423084863
:10819000FFF718FE074A08481E231F21CDE90031CA
:1081A00003231146FFF70EFE03B05DF804FB00BF8A
:1081B000107B012000300040CC7B012008B540221C
:1081C000002102F0F1FC0022C0E9102208BD026C7F
:1081D00010B5531C446C03F03F039C421CBF8154F8
:1081E000036410BD0023C0E910337047D0E91023A9
:1081F00093421FBFC25C013303F03F03436414BFCB
:1082000010464FF0FF307047D0E91030181A48BFC1
:1082100040307047D0E91023934214BFC05C4FF048
:10822000FF307047036C406C013303F03F031B1AAF
:1082300058425841704700000649074A074B9B1AAD
:1082400003DD043BC858D050FBDC00F013F8F7F70F
:10825000F7FF0000C8DC00000000002044020020FE
:10826000FEE7FEE7FEE7FEE7FEE7FEE7FEE7FEE7E6
:10827000FEE7FEE7394B1A680D2A08D14FF080421D
:108280000021C2F80C11C2F81011C2F838151B6891
:108290000D2B46D14FF08052314BD2F80414C3F865
:1082A0002015D2F80814C3F82415D2F80C14C3F81A
:1082B0002815D2F81014C3F82C15D2F81414C3F8EA
:1082C0003015D2F81814C3F83415D2F81C14C3F8BA
:1082D0004015D2F82014C3F84415D2F82414C3F87A
:1082E0004815D2F82814C3F84C15D2F82C14C3F84A
:1082F0005015D2F83014C3F85415D2F83414C3F81A
:108300006015D2F83814C3F86415D2F83C14C3F8D9
:108310006815D2F84014C3F86C15D2F84424C3F899
:1083200070250E4B1B680D2B09D14FF08043D3F8FD
:108330000024D20744BF6FF00102C3F80024094AA9
:10834000D2F8883043F47003C2F88830BFF34F8FFF
:10835000BFF36F8F044B054A1A607047300100105D
:1083600000C0004000ED00E03C0000200090D00381
:108370000120704703681322DB69184770470369BF
:10838000C3F81C150369D3F81C21002AFBD0002276
:10839000C3F81C210120704710B490F95C30144CD4
:1083A00059090122203103F01F0302FA03F344F8B4
:1083B000213003695DF8044B0421C3F808130369F5
:1083C0005A600369DA6003690022C3F80025026974
:1083D0004FF0FF33C2F80C350269C2F81435026958
:1083E000C2F8083502691430C2F81035FFF7FABE3A
:1083F00000E100E01430FFF707BF1430FFF70ABFB9
:108400001430FFF7F3BE0000036990F85E2010B54A
:10841000C3F80C25036990F85D20C3F8142590F883
:1084200061200369012A01BF90F85F40C3F810453D
:10843000036990F8604006BFC3F80845036900224D
:10844000B1F5966FC3F86C2569D9B1F5166F69D986
:10845000B1F5965F69D9B1F5165F68D9B1F5615F7D
:1084600067D9B1F5964F66D9B1F5E14F65D9B1F548
:10847000164F64D9B1F5614F64D9B1F5963F64D90F
:10848000B1F5E13F63D9B1F5613F63D9364B99420C
:1084900063D9B1F5E12F63D9B1F5612F94BF4FF0E6
:1084A00070634FF080530269C2F8243503690422D7
:1084B000C3F8002501690023C1F808310169C1F83A
:1084C0001C31016901230B6001698B600169C1F8EE
:1084D000042390F95C20510902F01F02934060319F
:1084E000224A42F8213090F95C30002BBDBF03F0E6
:1084F0000F0302F6FC32D2189B18B5BF602360222E
:10850000137683F8002390F95C300122590903F0B7
:108510001F0302FA03F3154A42F8213010BD4FF44D
:108520009E23C0E74FF41D23BDE7114BBBE7114B62
:10853000B9E7114BB7E7114BB5E7114BB3E74FF470
:108540001D03B0E74FF46B03ADE70E4BABE74FF005
:10855000EB73A8E74FF06C73A5E74FF08063A2E7D9
:108560004FF0E8639FE700BF90D0030000E100E018
:1085700000B013000050270000F03A0000A04E00A9
:1085800000C0750000903A012DE9F0411E4600251B
:108590004FF47A73C0E901530D4B044640F8143B85
:1085A00017468846FFF70AFE0A4AC4F8108084F886
:1085B0005C7052F8263084F85D309DF8183052F81F
:1085C000233084F85E3084F861502046BDE8F081A5
:1085D000B8D8000024D8000010B50369D3F80821EA
:1085E00004464AB1D3F818151430C9B2FFF7EFFDAD
:1085F00023690022C3F8082110BD00000148FFF7DD
:10860000EBBF00BF887C012007B522230093022224
:10861000212303490348FFF7B7FF03B05DF804FBCC
:1086200000200040887C012008B102F08BBD70471B
:108630000A4B19680A4B30B5D3F804050C060D0A2D
:1086400044EA00024FF47A712B46A2FB014501FB7C
:108650000355E00B40EA454030BD00BFEC7C0120F3
:108660000010014038B5044648B1FFF7E1FF054668
:1086700000F01AF8FFF7DCFF401BA042F8D338BD2A
:10868000074B0022C3F8042182B0D3F80431054A15
:108690000193019B13680133DBB2136002B0704792
:1086A00000100140EC7C01207047704708B500F0D5
:1086B00067F8FFF7FAFF0120FFF7D4FFFFF79AFAF8
:1086C000034CFFF7A9FA002CFBD0AFF30080F8E7CA
:1086D0000000000038B5174B174D53F820301748ED
:1086E00013F0200F4FF0010403F01F0304FA03F40A
:1086F00008BF4FF0A04000292B681149B3FBF1F3EC
:1087000000F5A26002FB03F321464FF00A02B3FB1F
:10871000F2F314BF2246002200F014F842F2107364
:1087200058434FF47A722B68B3FBF2F3B0FBF3F0CB
:1087300038BD00BF24D800003C00002000030050DA
:1087400040420F0030B504680C40944206D1013B12
:10875000002BF8D112E0013B002B0FD004680C4035
:108760009442F8D1002405680D40954204D10134AB
:108770009C42F8D1002002E0201C00E0181C30BD13
:108780000D4BE02283F811234FF40032C3F880210F
:108790001A604FF080430122C3F818259A6003F550
:1087A00088330021C3F808150221C3F80413C3F865
:1087B00044131A60704700BF00E100E0014B1860ED
:1087C000704700BF580000200228064A064B1BBF16
:1087D000002111600121012212BF1A60116018608E
:1087E000704700BFF87C012054000020222837B5D4
:1087F0000CD84B4B53F82030052B00F0828007D863
:10880000032B12D07BD8022B00F08180002074E073
:108810001D2B78D003D81C2BF8D1052206E01E2B87
:1088200073D01F2BF2D1082200E002223D4B1968C1
:1088300008296EDD0A296FDD0D29B5BF0C240E2431
:10884000022303233848C0F8F0350123C0F800356F
:1088500000200546030103F1804303F5E0430130A6
:108860000828C3F81455C3F81055F3D12F4B1868D6
:108870002F4B1B6800021B0303F4805300F4E060DD
:108880001843294BC3F81805C3F81425C3F810255D
:108890000DF10602C3F82C260122C3F830261A6017
:1088A000D3F80021002AFBD00022C3F800210122C6
:1088B0005A601D4B1A46D3F804010028FBD0002053
:1088C000C3F8040101209860D2F81431002BFBD0CA
:1088D0000023C2F81431BDF906209A42124AB8BFEB
:1088E000ADF80630A142C2F80035BDF9060004D04B
:1088F00035BF611A091BC840884003B030BD032250
:1089000094E7042292E7062290E707228EE70122ED
:108910008CE70824002395E70A24012392E700BF8F
:1089200024D80000500000200070004054000020B7
:10893000F87C0120222830B53CD8224B53F8200087
:10894000214B00221D4653F82240B4F1FF3F32D1A3
:108950001E4C45F822006FEA41411D4D1D4B246815
:1089600053F822306FEA514125F81210012101FA23
:1089700004F4C3F86005013CC3F8640505EB42024A
:10898000C3F86805C3F86C050020C3F80015C3F8E8
:108990000C05C3F80405C3F80845C3F81405C3F86B
:1089A0001005C3F82025C3F82415C3F82815C3F80B
:1089B0002C05996030BD8442CAD00132042AC2D14C
:1089C000F8E700BF24D80000400000205800002035
:1089D000F07C0120E0D80000222815D8114B124A63
:1089E00053F8203013F0200F08BF4FF0A04203F0DF
:1089F0001F03032908D8DFE801F00210080C03F573
:108A0000E073002142F82310704703F5E0730C2156
:108A1000F8E703F5E0730421F4E703F5E0730321BD
:108A2000F0E700BF24D8000000030050222813D82C
:108A30000A4B53F820000A4B10F0200F4FF00102B0
:108A400000F01F0008BF4FF0A043824011B9C3F8E7
:108A50000C257047C3F80825704700BF24D80000D4
:108A600000030050222810D8094B0A4A53F820303E
:108A700013F0200F08BF4FF0A04203F01F03D2F8FD
:108A80001005D84000F0010070470020704700BF7B
:108A900024D80000000300502DE9F04106460D46A1
:108AA00001EB02080C464445A4EB050707D03368E8
:108AB00014F8011B1B68304698470028F3D138464C
:108AC000BDE8F0812DE9F041C1F30A57A7F2FF3567
:108AD000132D82B002460B460C464FEAD17806466B
:108AE00033DC002D4EDB3C49294103EA01001043F1
:108AF00026D049080B4052EA03060CD04FF48023DD
:108B0000132D24EA010143FA05F444EA01040CBFE1
:108B10004FF000460026314901EBC8082346D8E94A
:108B2000004532462046294601F01EFBCDE90001F2
:108B300022462B46DDE9000101F014FB02460B46FC
:108B40001046194602B0BDE8F081332D07DDB5F5BA
:108B5000806FF5D101F008FB02460B46F0E7A7F263
:108B600013474FF0FF31F9400842E9D04908084265
:108B7000D1D04FF0804320EA010143FA07F741EAE0
:108B80000706C8E721F000410143D9D0C3F3130120
:108B900001434E420E43114D5C0C360B640406F447
:108BA000002305EBC80243EA0401D2E900450B4665
:108BB00002462946204601F0D7FACDE900012246B7
:108BC0002B46DDE9000101F0CDFA21F0004102461B
:108BD00041EAC873B4E700BFFFFF0F00F0D8000000
:108BE000F8B5C1F30A57A7F2FF35132D02460B461D
:108BF0000C4610DC002D29DB8C461D4929410B4217
:108C00002AD04FF400242C41644424EA01040026B5
:108C100021463046F8BD332D05DDB5F5806F1ED0F9
:108C200010461946F8BDA7F213474FF0FF3121FA5D
:108C300007F73842F4D00123C5F1330503FA05F5EF
:108C4000461928BFE41826EA0706E1E7013501F0D6
:108C5000004407D00026DBE70028D2D1E0E701F08E
:108C600083FAF8BD44F07F5444F440140026CFE763
:108C7000FFFF0F0030B51F4A21F00043934287B039
:108C80001CDD1D4A934205DD02460B4601F06AFADF
:108C900007B030BD02AA00F08FF800F003000128F1
:108CA000DDE9042312D002281CD0A0B1DDE90201C5
:108CB00000F066FB01F1004107B030BD00230093D6
:108CC0000022002301F084F807B030BDDDE9020185
:108CD00000F056FBDCE70124DDE90201009401F01D
:108CE00077F8D5E70124DDE90201009401F070F87E
:108CF000E0E700BFFB21E93FFFFFEF7F2DE9F04FE9
:108D00008BB004460D4600F079FA294B93F900A088
:108D1000BAF1FF3F06460F4612D022462B462046A8
:108D2000294601F071FE834650B94FF000084FF01C
:108D300000092046294642464B4601F03DFE20B937
:108D4000304639460BB0BDE8F08F0122194BCDF803
:108D500020B00092CDE90445CDE902450193BAF176
:108D6000000F17D042464B464046494601F0DCFC16
:108D7000BAF1020FCDE906010ED101F0A1FE2123C7
:108D80000360089B73B9DDE90667304639460BB0CE
:108D9000BDE8F08FCDE90689684601F055F9002855
:108DA000EFD1EAE701F08CFE089B0360EBE700BF20
:108DB0005C00002000D900002DE9F047CA4B21F0EB
:108DC00000479F4290B08046894640F38F80C74B52
:108DD0009F420C46924626DC0029B9A3D3E9002322
:108DE00040F38F8001F0BEF9C14B9F4204460D460F
:108DF00000F04781B4A3D3E9002301F0B3F90246A0
:108E00000B46CAE900232046294601F0ABF9AEA380
:108E1000D3E9002301F0A6F90125CAE90201284699
:108E200010B0BDE8F087B34B9F4240F38980B24B4E
:108E30009F4200F31C813D15A5F21645A7EB055393
:108E400019461F46064601F0F5FD01F0D9FA8046A5
:108E5000894642464B4630463946CDE90A8901F0FB
:108E600081F90022A54B01F035FB8946804601F0CF
:108E7000E1FD01F0C5FA06460F4632463B46404644
:108E80004946CDE90C6701F06DF900229B4B01F0DA
:108E900021FB00220023CDE90E0101F083FD002813
:108EA00000F06081002330463946002201F07AFD4F
:108EB000002814BF01230223914A019202212A466D
:108EC00000910AA8514600F083FB002C054614DAF5
:108ED000DAF80420DAF80C3002F1004203F1004322
:108EE0004542CAF80420CAF80C3006E000200021F0
:108EF000C2E90089C2E902010025284610B0BDE898
:108F0000F08701F031F97A4B9F4204460D4600F09C
:108F10000B816DA3D3E9002301F026F902460B462D
:108F2000CAE900232946204601F01CF966A3D3E9CB
:108F3000002301F019F94FF0FF35CAE90201DCE71F
:108F400000F0FCFF62A3D3E900238046894601F0CC
:108F5000C1FA00226B4B01F007F901F06BFD0546E9
:108F600001F04EFA56A3D3E90023CDE9060101F042
:108F7000B1FA02460B464046494601F0F3F852A3C7
:108F8000D3E9002380468946DDE90601CDE902895F
:108F900001F0A0FA1F2D02460B46CDE9042340F351
:108FA000B380DDE90423DDE9020101F0DBF880464E
:108FB00089463F15C9F30A53FB1A102B40F3B180C1
:108FC00045A3D3E90023DDE9060101F083FA8046D9
:108FD000894602460B46DDE9020101F0C3F802466C
:108FE0000B46DDE90201CDE9082301F0BBF842465A
:108FF0004B4601F0B7F83AA3D3E9002380468946EF
:10900000DDE9060101F066FA42464B4601F0AAF896
:109010000B46CDE904010246DDE9080101F0A2F8A2
:10902000C1F30A53FF1A312F8046894600F39C8012
:109030009DED087BCAE900898DED027B42464B46D7
:10904000DDE9020101F08EF8DDE9042301F08AF880
:10905000002CCAE90201BFF650AF09F1004401F14A
:1090600000436D42CAE90084CAE9020345E70246AB
:109070000B4601F077F80025CAE90201CAE90001B0
:109080003BE715A3D3E9002301F06CF814A3D3E95F
:1090900000230D46044601F065F802460B46CAE976
:1090A00000232946204601F05DF80DA3D3E90023F3
:1090B00001F058F80125CAE902011EE7AFF300806C
:1090C00000004054FB21F93F3163621A61B4D03D86
:1090D00083C8C96D305FE43F0000601A61B4D03DC1
:1090E0007370032E8A19A33BFB21E93F7BD9024011
:1090F000FB21F93FFB213941FFFFEF7F0000704169
:1091000088D900000000E03F4046494601F02AF8B7
:10911000394B6A1E804653F82230BB4289463FF4E1
:1091200048AFCAE9008989E72BA3D3E9002301F0FE
:109130001BF82BA3D3E900230D46044601F014F8D5
:1091400002460B46CAE900232946204601F00AF8E8
:1091500023A3D3E9002301F007F84FF0FF35CAE954
:109160000201CAE60323A7E61FA3D3E90023DDE932
:10917000060101F0AFF906460F4602460B46DDE94F
:10918000080100F0EFFF8046894602460B46DDE904
:109190000801CDE9028900F0E5FF32463B4600F0C8
:1091A000E1FF13A3D3E9002306460F46DDE90601DC
:1091B00001F090F932463B4600F0D4FF02460B46E0
:1091C00040464946CDE9042300F0CCFF804689465D
:1091D000A7E700BFAFF300800000601A61B4D03D84
:1091E0007370032E8A19A33B0000002E8A19A33B3B
:1091F000C14920259A837B3908D900005E4A8A43F9
:109200002DE9F04104460D4600F0958000290B46FB
:109210000646844656DD0F1500F0A580C3F3130300
:10922000A7F2FF3743F480134FEADC72F80702EB32
:1092300043034FEA4C0504D5ED0F05EB43034FEA1A
:109240008C0500267F10B44616224FF400110CEB5B
:10925000010098424FEAD5744FEA450503DC1B1A1A
:1092600000EB010C0E44013A04EB43034FEA5101B9
:10927000EDD11046964620244FF0004209E051D02F
:109280005B00013C03EBD5734FEA52024FEA450500
:1092900037D0634502EB0E01F1DD002901EB020E30
:1092A0000ADBE046A3EB0C03A94288BF03F1FF33BE
:1092B0006D1A1044C446E3E7BEF1000FF1DB0CF178
:1092C0000108EFE721F00042024329D0002942D1F2
:1092D0000146CA0A153B4905002AFAD012F480104B
:1092E00001D044E060465200D40200F1010CF9D5EF
:1092F000CCF1200401FA0CFCE1401F1A41EA020300
:109300008CE72B4321D14408731003F17F53F207FC
:1093100003F5001348BF44F0004403EB0751204617
:10932000BDE8F081A942ABD8002901EB020EC3DBF6
:1093300098460023BCE702460B4601F0CBF82246D4
:109340002B4600F011FFBDE8F081411C16BF421C06
:1093500001365408D8E7024600F004FF02460B46E7
:1093600001F0E2F9DCE71A4631463B46B6E78C46A7
:1093700020244FF0FF30BFE70000F07F0000000026
:109380002DE9F04F21F00048B8F1795F85B006462D
:109390000F4692469B466BDA01F04CFB002800F02A
:1093A000E18032463B463046394601F093F874A3DB
:1093B000D3E9002304460D4601F08CF872A3D3E9EB
:1093C000002300F0D1FE22462B4601F083F870A363
:1093D000D3E9002300F0C6FE22462B4601F07AF8BE
:1093E0006DA3D3E9002300F0BFFE22462B4601F017
:1093F00071F86BA3D3E9002300F0B4FE22462B469C
:1094000001F068F868A3D3E9002300F0ADFE22461E
:109410002B4601F05FF8CDE900010022664B2046A3
:10942000294601F057F8DDE90023804689462046A9
:10943000294601F04FF8524604460D465B46304639
:10944000394601F047F802460B462046294600F00F
:1094500089FE02460B464046494600F083FE02461E
:109460000B460020554900F07DFE05B0BDE8F08FA9
:1094700002460B4601F02EF841A3D3E9002304462F
:109480000D4601F027F840A3D3E9002300F06CFE5D
:1094900022462B4601F01EF83DA3D3E9002300F03D
:1094A00061FE22462B4601F015F83BA3D3E90023C9
:1094B00000F05AFE22462B4601F00CF838A3D3E9FF
:1094C000002300F04FFE22462B4601F003F836A39E
:1094D000D3E9002300F048FE2B46224600F0FAFFB5
:1094E000374B9845CDE9000197DD364B98453EDC7A
:1094F000A8F500130022002030499046994600F05C
:1095000031FECDE9020100222B4B2046294600F016
:10951000E1FF42464B4600F025FEDDE90023804690
:1095200089462046294600F0D5FF524604460D469E
:109530005B463046394600F0CDFF02460B462046DA
:10954000294600F00FFE02460B464046494600F011
:1095500009FE02460B46DDE9020100F003FE05B0FC
:10956000BDE8F08F1549002005B0BDE8F08F9FEDF4
:10957000107B4FF000088DED027BDFF84C90C2E7C6
:10958000D43888BEE9FAA8BDC4B1B4BD9EEE213E70
:10959000AD529C804F7E923E9015CB19A001FA3EB1
:1095A0007751C1166CC1563F4C5555555555A53F81
:1095B000000000000000E73F0000E03F0000F03F37
:1095C0003233D33F0000E93F0000D23F00000000EB
:1095D0002DE9F04FADF5197DBE4CA29EBE4D54F85D
:1095E00026600793D41E85FB0475E417C4EBA5041D
:1095F00024EAE4741D46631CA3EB8303013D02EBE4
:10960000C3030593731904960994019503900B9174
:10961000A4EB05071AD43B44002400255E1C0DF181
:109620008008DDF88C9208E059F8270000F0E8FE89
:109630000137B742E8E8020108D0002FF4DA013719
:1096400020462946B742E8E80201F6D1049B002BE8
:10965000079B4FEAC30302932ADB039A20A902EB7C
:10966000030801EB0309049B72AA02EBC30B0DF57F
:10967000E07A019B002B4FF000064FF0000711DB52
:10968000039C4D4675E90223F4E8020100F022FF35
:1096900002460B463046394600F066FD4445064614
:1096A0000F46EFD1EAE80267DA4509F10809E0D18F
:1096B000DDE90204049920448B0082460BA8A3F143
:1096C0000802C31808930CAB13440A938B4698AB5B
:1096D00003EBCB03BBF1000F53E9284529DD70AB49
:1096E00003EBCB080DF1300900227C4B20462946C4
:1096F00000F0F0FE01F09EF900F082FE0022784BAF
:1097000006460F4600F0E6FE02460B462046294676
:1097100000F028FD01F08EF978E9022349F8040BE6
:109720003946304600F020FD70AB984504460D46A2
:10973000DAD1DDF81490204629464A4600F088FC2C
:1097400000224FF07F5304460D4600F0C3FE00F0A8
:10975000FBFB0022634B00F0BDFE02460B46204699
:10976000294600F0FFFC0D46044601F063F98046EF
:1097700000F046FE0B4602462946204600F0F2FC69
:109780004B46002B06460F4640F3E1800BF1FF32BB
:109790000CA9C9F1180351F8225045FA03F101FA56
:1097A00003F30CA8EB1A40F82230C9F117058844DE
:1097B00043FA05F5002D2CDDBBF1000F08F101087F
:1097C00040F381820C9C002C40F0A780BBF1010F7C
:1097D0000AD00CA9012251F8044F531C002C40F070
:1097E0009E809B451A46F6D1059B002B0EDD012B72
:1097F00000F0D980022B09D10BF1FF320CAB0CA980
:1098000053F82230C3F3150341F82230022D00F043
:10981000AF80002200233046394601F0C3F800280B
:1098200000F05382049B0BF1FF394B4510DC0BF128
:1098300080430CAA013B089802EB8303002253F8F3
:109840000419834242EA0102F9D1002A40F0B680AD
:10985000049B0CAA013B52F82330002B40F0A1805E
:109860000A9A012352F8041901330029FAD05B4403
:109870000BF10109994506934CDC099A079909EB0C
:10988000020801EB0B0508F1804802EB030BA39BD8
:1098900008F1FF3803EB880870AB03EBC909A39B01
:1098A00020A903EB8B0301EBC505029358F8040FC5
:1098B00000F0A6FD0B4601990246002905F1080BB0
:1098C000C5E900234FF000064FF000071CDB039CA6
:1098D0000CE000BFD0DA0000ABAAAA2A0000703E5C
:1098E000000070410000204075E90223F4E8020105
:1098F00000F0F0FD02460B463046394600F034FCDD
:10990000544506460F46EFD1029B9845E9E80267A9
:109910005D46CBD1DDF818B0D9E6012300220CA9B1
:10992000C4F180749B4541F822400EDD51F823209C
:1099300001EB8B0001EB83036FF07F4100E01A68BD
:109940008A1A43F8042B8342F9D101244CE706D14B
:109950000BF1FF330CAA52F82350ED152AE7002231
:109960007B4B01F03DF8002840F0A381054650E70D
:1099700032463B460020774900F0F4FB06460F468E
:10998000002C3FF446AF059A7249002000F060FBBE
:1099900002460B463046394600F0E4FB06460F46C9
:1099A00037E7012363E70BF1FF320CAB0CA953F847
:1099B0002230C3F3160341F8223027E70CAB059A97
:1099C00053F82930183ACDE9068505926BB909F1AB
:1099D0008043013B0CA901EB830353F8041909F1FF
:1099E000FF39183A0029F8D00592059A5949002004
:1099F00000F02EFBB9F1000F04460D46C0F2C08105
:109A00004FEAC90370AA02EB030808930CAB03EBFF
:109A10008906DFF844B14FF0000A08F10807043660
:109A200056F8040D00F0ECFC22462B4600F052FDE7
:109A30005B4667E9020152462046294600F04AFD8E
:109A40000CAB9E4204460D46EAD148AB039301930A
:109A5000CDF8149009F10103DDF810900293C3468C
:109A60004FF0000AB9F1000FC0F22A81DFF8EC8054
:109A70005D4635A3D3E9002300260027002403E038
:109A8000544510DCF8E80223F5E8020100F022FD5D
:109A900002460B463046394600F066FB0134A145CC
:109AA00006460F46ECDA019BE3E802670193029B4E
:109AB0000AF1010A9A45ABF1080BD3D1A29BDDF85C
:109AC0001490032B39D8DFE813F0D9000600060004
:109AD0004D0048AB0393B9F1000F4FF000004FF079
:109AE000000109DB039D05EBC904083474E9022376
:109AF00000F03AFBA542F9D1079B002B40F01E81F4
:109B00000B9BC3E900010B4603990246D1E9000112
:109B100000F028FBB9F1000F0CDD4AAD012401343F
:109B2000F5E8022300F020FBA145F8DA079B002BA3
:109B300040F014810B9BC3E90201069B03F0070070
:109B40000DF5197DBDE8F08F00000040FB21F93FC5
:109B50000000E03F0000F03F0000703E98DA000097
:109B600048AB0393B9F1000F40F32781039ACDF876
:109B700010904FEAC9030193D318D3E900AB09F160
:109B80000053013B02EBC9080293914678E9026752
:109B900052465B463046394600F0E6FA04460D462A
:109BA00002460B463046394600F0DCFA52465B4628
:109BB00000F0DAFAC145A246AB46C8E90201C8E99D
:109BC0000045E3D1DDF81090B9F1010F40F3F580C5
:109BD000019B039A02991344C900D3E9006701F17C
:109BE000080A019192440DF5947B7AE90289324684
:109BF0003B464046494600F0B7FA04460D46024649
:109C00000B464046494600F0ADFA32463B4600F06E
:109C1000ABFAD34526462F46CAE90201CAE90045F8
:109C2000E3D1019C039B1034002000211C4403F16C
:109C3000100574E9022300F097FAA542F9D1039CBC
:109C4000079ED4E90023D4E90245002E00F08A8063
:109C500003F1004701F100430B99C1E90403069B9E
:109C60002646944605F1004403F00700C1E900C709
:109C7000C1E902640DF5197DBDE8F08F089C039DD4
:109C80000834002000212C4474E9022300F06CFA0F
:109C9000A542F9D1079B13B101F1004319460B9B73
:109CA000C3E90001069B03F007000DF5197DBDE82F
:109CB000F08FBBF1000F08F1010874DD022581E58A
:109CC00000260027EFE600248EE5CDE90685059DF8
:109CD000304639466A4200F0BBF90022384B06464E
:109CE0000F4600F07DFE00B30022364B3046394669
:109CF00000F0F0FB00F09EFE044600F081FB002225
:109D00002F4B00F0E7FB0B4602463946304600F089
:109D100029FA00F08FFE0BF101090CAB183543F85E
:109D20002B00059543F829405FE63046394600F0A0
:109D300081FE0CABD94643F82B0056E60B9C01F193
:109D40000043C4E900030B4603990246D1E9000130
:109D500000F008FAB9F1000F3FF7DFAE01F1004360
:109D60001946E7E60B9EC6E90023069BC6E90401F7
:109D700003F00700C6E902450DF5197DBDE8F08F37
:109D8000A29B032B3FF6D9AE01A252F823F000BFED
:109D9000A19D0000D39A0000D39A0000619B0000AF
:109DA0000020002176E732463B460020064900F0BD
:109DB000D9F9022506460F462BE5002000213EE793
:109DC000000070410000703E0000F03F0000000005
:109DD0002DE9F04F21F00046B6F1795F85B00446D9
:109DE0000D469046994604DA00F024FE002800F063
:109DF000858022462B462046294600F06BFB06460E
:109E00000F4602460B462046294600F063FB41A35D
:109E1000D3E9002382468B463046394600F05AFB90
:109E20003EA3D3E9002300F09DF932463B4600F003
:109E300051FB3CA3D3E9002300F096F932463B46A0
:109E400000F048FB39A3D3E9002300F08BF9324638
:109E50003B4600F03FFB37A3D3E9002300F084F931
:109E60000E9BCDE900019BB30022294B4046494699
:109E700000F030FBDDE90023CDE9020150465946F0
:109E800000F028FB02460B46DDE9020100F06AF90A
:109E900032463B4600F01EFB42464B4600F062F95C
:109EA00019A3D3E9002306460F465046594600F051
:109EB00011FB02460B463046394600F055F9024682
:109EC0000B462046294600F04DF905B0BDE8F08F5D
:109ED00002460B463046394600F0FCFA0AA3D3E9A5
:109EE000002300F03FF952465B4600F0F3FA2246A9
:109EF0002B4600F039F905B0BDE8F08F2046294621
:109F000005B0BDE8F08F00BF495555555555C53FC3
:109F10000000E03F7CD5CF5A3AD9E53DEB9C2B8A37
:109F2000E6E55A3E7DFEB157E31DC73ED561C11936
:109F3000A0012A3FA6F810111111813F21F0004322
:109F400019467047000000002DE9F041C1F30A579F
:109F5000A7F2FF35132D02460B460C4688460646EF
:109F60001DDC002D3CDB364F2F4101EA070C5CEA7B
:109F7000000C19D030A3D3E9002300F0F5F800223B
:109F8000002300F037FDC8B3002C04DA4FF480132F
:109F900043FA05F5A84428EA070400262EE0332DED
:109FA00006DDB5F5806F2DD010461946BDE8F0816D
:109FB000A7F213474FF0FF3C2CFA07F70742F3D004
:109FC0001DA3D3E9002300F0CFF80022002300F006
:109FD00011FD98B1002C21DB26EA070644460DE06E
:109FE00015A3D3E9002300F0BFF80022002300F0FE
:109FF00001FD18B1002C08DB00263446214630460E
:10A00000BDE8F08100F0B0F8D0E724F000430D4A3D
:10A010001E43002E18BF14460026EFE7142D08D06B
:10A020000123C5F1340503FA05F5AE1928BF98449C
:10A03000D2E704F10108CFE79C7500883CE4377E45
:10A04000FFFF0F000000F0BF00207047000000007D
:10A05000F8B5C1F30A5304460D460E4617460BBB2E
:10A0600021F00046034633431BD0354B002200F05D
:10A0700031FA344B9F4204460D4635DBC1F30A5397
:10A080000E46363B3B4440F2FE72934232DC002BDC
:10A0900011DD26F0FF4626F4E00646EA0355204689
:10A0A0002946F8BD40F2FF729342EBD102460B46BF
:10A0B00000F05AF8F8BD13F1350F28DA4CF250339E
:10A0C0009F4222462B460ADD19A1D1E9000100F08A
:10A0D0003DF817A3D3E9002300F0FCF9F8BD16A161
:10A0E000D1E9000100F032F813A3D3E9002300F016
:10A0F000F1F9F8BD22462B460DA1D1E9000100F08F
:10A1000025F80BA3D3E9002300F0E4F9F8BD26F00D
:10A11000FF4626F4E006363346EA03552046294634
:10A120000022094B00F0D6F9F8BD00BFAFF3008064
:10A130009C7500883CE4377E59F3F8C21F6EA50178
:10A1400000005043B03CFFFF0000903C03F0004390
:10A1500021F0004242EA0301704700BF81F0004154
:10A1600002E000BF83F0004330B54FEA41044FEAFC
:10A17000430594EA050F08BF90EA020F1FBF54EA97
:10A18000000C55EA020C7FEA645C7FEA655C00F033
:10A19000E2804FEA5454D4EB5555B8BF6D420CDD04
:10A1A0002C4480EA020281EA030382EA000083EA87
:10A1B000010180EA020281EA0303362D88BF30BD27
:10A1C00011F0004F4FEA01314FF4801C4CEA11317D
:10A1D00002D0404261EB410113F0004F4FEA0333DC
:10A1E0004CEA133302D0524263EB430394EA050F67
:10A1F00000F0A780A4F10104D5F1200E0DDB02FAD6
:10A200000EFC22FA05F2801841F1000103FA0EF269
:10A21000801843FA05F359410EE0A5F120050EF12F
:10A22000200E012A03FA0EFC28BF4CF0020C43FA60
:10A2300005F3C01851EBE37101F0004507D54FF06D
:10A24000000EDCF1000C7EEB00006EEB0101B1F5BD
:10A25000801F1BD3B1F5001F0CD349085FEA300003
:10A260004FEA3C0C04F101044FEA445212F5800F0E
:10A2700080F09A80BCF1004F08BF5FEA500C50F1AB
:10A28000000041EB045141EA050130BD5FEA4C0C8E
:10A29000404141EB010111F4801FA4F10104E9D117
:10A2A00091F0000F04BF01460020B1FA81F308BF0E
:10A2B0002033A3F10B03B3F120020CDA0C3208DDDA
:10A2C00002F1140CC2F10C0201FA0CF021FA02F1B5
:10A2D0000CE002F11402D8BFC2F1200C01FA02F125
:10A2E00020FA0CFCDCBF41EA0C019040E41AA2BF4A
:10A2F00001EB0451294330BD6FEA04041F3C1CDA12
:10A300000C340EDC04F11404C4F1200220FA04F031
:10A3100001FA02F340EA030021FA04F345EA0301DB
:10A3200030BDC4F10C04C4F1200220FA02F001FA9D
:10A3300004F340EA0300294630BD21FA04F029461F
:10A3400030BD94F0000F83F4801306BF81F48011B8
:10A350000134013D4EE77FEA645C18BF7FEA655C2B
:10A3600029D094EA050F08BF90EA020F05D054EAFD
:10A37000000C04BF1946104630BD91EA030F1EBF02
:10A380000021002030BD5FEA545C05D14000494106
:10A3900028BF41F0004130BD14F580043CBF01F5F9
:10A3A000801130BD01F0004545F0FE4141F47001DF
:10A3B0004FF0000030BD7FEA645C1ABF19461046BA
:10A3C0007FEA655C1CBF0B46024650EA013406BFBB
:10A3D00052EA033591EA030F41F4002130BD00BF7A
:10A3E00090F0000F04BF0021704730B54FF4806437
:10A3F00004F132044FF000054FF0000150E700BFB8
:10A4000090F0000F04BF0021704730B54FF4806416
:10A4100004F1320410F0004548BF40424FF0000103
:10A420003EE700BF42004FEAE2014FEA31014FEA46
:10A4300002701FBF12F07F4393F07F4F81F0605195
:10A44000704732F07F4208BF704793F07F4F04BFE0
:10A4500041F40021704730B54FF4607401F00045BD
:10A4600021F000411CE700BF50EA010208BF70471D
:10A4700030B54FF000050AE050EA010208BF70470E
:10A4800030B511F0004502D5404261EB41014FF477
:10A49000806404F132045FEA915C3FF4D8AE4FF07F
:10A4A00003025FEADC0C18BF03325FEADC0C18BF62
:10A4B000033202EBDC02C2F1200300FA03FC20FAB3
:10A4C00002F001FA03FE40EA0E0021FA02F1144400
:10A4D000BDE600BF70B54FF0FF0C4CF4E06C1CEA19
:10A4E00011541DBF1CEA135594EA0C0F95EA0C0F8A
:10A4F00000F0DEF82C4481EA030621EA4C5123EAFD
:10A500004C5350EA013518BF52EA033541F480112B
:10A5100043F4801338D0A0FB02CE4FF00005E1FBDE
:10A5200002E506F00042E0FB03E54FF00006E1FB28
:10A5300003569CF0000F18BF4EF0010EA4F1FF046B
:10A54000B6F5007F64F5407404D25FEA4E0E6D41AB
:10A5500046EB060642EAC62141EA55514FEAC520BC
:10A5600040EA5E504FEACE2EB4F1FD0C88BFBCF538
:10A57000E06F1ED8BEF1004F08BF5FEA500E50F1E9
:10A58000000041EB045170BD06F0004646EA0101AF
:10A5900040EA020081EA0301B4EB5C04C2BFD4EBE1
:10A5A0000C0541EA045170BD41F480114FF0000EDA
:10A5B000013C00F3AB8014F1360FDEBF002001F048
:10A5C000004170BDC4F10004203C35DA0C341BDCC2
:10A5D00004F11404C4F1200500FA05F320FA04F094
:10A5E00001FA05F240EA020001F0004221F00041C8
:10A5F00010EBD37021FA04F642EB06015EEA430E3B
:10A6000008BF20EAD37070BDC4F10C04C4F120056A
:10A6100000FA04F320FA05F001FA04F240EA02001D
:10A6200001F0004110EBD37041F100015EEA430EEE
:10A6300008BF20EAD37070BDC4F1200500FA05F20E
:10A640004EEA020E20FA04F301FA05F243EA02038D
:10A6500021FA04F001F0004121FA04F220EA02009C
:10A6600000EBD3705EEA430E08BF20EAD37070BDE2
:10A6700094F0000F0FD101F00046400041EB0101C2
:10A6800011F4801F08BF013CF7D041EA060195F0A4
:10A69000000F18BF704703F00046520043EB03035E
:10A6A00013F4801F08BF013DF7D043EA060370474B
:10A6B00094EA0C0F0CEA135518BF95EA0C0F0CD056
:10A6C00050EA410618BF52EA4306D1D181EA03019C
:10A6D00001F000414FF0000070BD50EA410606BF96
:10A6E0001046194652EA430619D094EA0C0F02D1DB
:10A6F00050EA013613D195EA0C0F05D152EA033620
:10A700001CBF104619460AD181EA030101F000413D
:10A7100041F0FE4141F470014FF0000070BD41F086
:10A72000FE4141F4780170BD70B54FF0FF0C4CF460
:10A73000E06C1CEA11541DBF1CEA135594EA0C0F7F
:10A7400095EA0C0F00F0A7F8A4EB050481EA030ECC
:10A7500052EA03354FEA013100F088804FEA0333B3
:10A760004FF0805545EA131343EA12634FEA022281
:10A7700045EA111545EA10654FEA00260EF0004142
:10A780009D4208BF964244F1FD0404F5407402D294
:10A790005B084FEA3202B61A65EB03055B084FEA25
:10A7A00032024FF480104FF4002CB6EB020E75EB22
:10A7B000030E22BFB61A754640EA0C005B084FEA4A
:10A7C0003202B6EB020E75EB030E22BFB61A7546C7
:10A7D00040EA5C005B084FEA3202B6EB020E75EB12
:10A7E000030E22BFB61A754640EA9C005B084FEA8A
:10A7F0003202B6EB020E75EB030E22BFB61A754697
:10A8000040EADC0055EA060E18D04FEA051545EA85
:10A8100016754FEA06164FEAC30343EA52734FEA2E
:10A82000C2025FEA1C1CC0D111F4801F0BD141EAA7
:10A8300000014FF000004FF0004CB6E711F4801F0C
:10A8400004BF01430020B4F1FD0C88BFBCF5E06FEC
:10A850003FF6AFAEB5EB030C04BFB6EB020C5FEAFC
:10A86000500C50F1000041EB045170BD0EF0004E51
:10A870004EEA113114EB5C04C2BFD4EB0C0541EA83
:10A88000045170BD41F480114FF0000E013C90E680
:10A8900045EA060E8DE60CEA135594EA0C0F08BF44
:10A8A00095EA0C0F3FF43BAF94EA0C0F0AD150EA43
:10A8B00001347FF434AF95EA0C0F7FF425AF1046D6
:10A8C00019462CE795EA0C0F06D152EA03353FF4FE
:10A8D000FDAE1046194622E750EA410618BF52EA7B
:10A8E00043067FF4C5AE50EA41047FF40DAF52EA4F
:10A8F00043057FF4EBAE12E74FF0FF3C06E000BFEC
:10A900004FF0010C02E000BF4FF0010C4DF804CDF8
:10A910004FEA410C7FEA6C5C4FEA430C18BF7FEAB8
:10A920006C5C1BD001B050EA410C0CBF52EA430CE6
:10A9300091EA030F02BF90EA020F0020704710F166
:10A94000000F91EA030F58BF994208BF90422CBFF5
:10A95000D8176FEAE37040F0010070474FEA410CEE
:10A960007FEA6C5C02D150EA013C07D14FEA430C0C
:10A970007FEA6C5CD6D152EA033CD3D05DF8040B7D
:10A98000704700BF8446104662468C4619466346AF
:10A9900000E000BF01B5FFF7B7FF002848BF10F186
:10A9A000000F01BD4DF808EDFFF7F4FF0CBF0120CB
:10A9B00000205DF808FB00BF4DF808EDFFF7EAFF47
:10A9C00034BF012000205DF808FB00BF4DF808ED02
:10A9D000FFF7E0FF94BF012000205DF808FB00BFF7
:10A9E0004DF808EDFFF7CEFF94BF012000205DF881
:10A9F00008FB00BF4DF808EDFFF7C4FF34BF01208E
:10AA000000205DF808FB00BF4FEA410C7FEA6C5C58
:10AA100002D150EA013C0AD14FEA430C7FEA6C5C58
:10AA200002D152EA033C02D14FF0000070474FF0D0
:10AA3000010070474FEA410212F5001215D211D5FC
:10AA40006FF47873B3EB625212D94FEAC12343F02B
:10AA5000004343EA505311F0004F23FA02F018BFAD
:10AA6000404270474FF00000704750EA013005D176
:10AA700011F0004008BF6FF0004070474FF0000039
:10AA8000704700BF1FB51C46094B1B680546D868B8
:10AA900052B1084B0091CDE9013207492B462246BD
:10AAA00000F028F800F0BAFD044B1A46F2E700BFA8
:10AAB00060000020E0DA0000EDDA000099C7000035
:10AAC000014B1868704700BF6000002008B5074BB5
:10AAD000044613B10021AFF30080054B1868836A68
:10AAE00003B19847204601F075FB00BF000000004D
:10AAF0001CDB00000EB403B5014603AB054853F858
:10AB0000042B0068019300F081F802B05DF804EBBB
:10AB100003B070476000002070B50D4E0D4CA41BB3
:10AB2000A4100025A54209D10B4E0C4C01F054FB9A
:10AB3000A41BA4100025A54205D170BD56F82530F0
:10AB400098470135EEE756F8253098470135F2E78A
:10AB5000300200203002002030020020400200209D
:10AB600010B5431E0A44914200D110BD11F8014BAB
:10AB700003F8014FF7E7884210B501EB020307D84D
:10AB8000421E99420AD011F8014B02F8014FF8E732
:10AB90008342F5D98118D21AD34200D110BD13F8DF
:10ABA000014D01F8014DF7E702440346934200D1FD
:10ABB000704703F8011BF9E79368013B002B10B4C1
:10ABC000936008DA9469A34201DB0A2903D15DF896
:10ABD000044B00F063BC1368581C106019700846E1
:10ABE0005DF8044B7047F8B506460F461446D51875
:10ABF000AC4201D1002007E03A4614F8011B304670
:10AC0000FFF7DAFF431CF3D1F8BD00002DE9F04F48
:10AC10009DB00C4617460393064618B183690BB9DD
:10AC200000F0F4FD7B4B9C4257D17468A389180750
:10AC30005DD52369002B5AD00023099320238DF87A
:10AC4000293030238DF82A304FF0010BB8464546A5
:10AC500015F8013B0BB1252B54D1B8EB070A0BD0EB
:10AC600053463A4621463046FFF7BDFF013000F01B
:10AC7000C280099B5344099398F80030002B00F0E0
:10AC8000BA8000234FF0FF32CDE9052304930793E8
:10AC90008DF853301A93A846052218F8011B5E4818
:10ACA00000F0C6FE049B78BBD90644BF20228DF875
:10ACB00053201A0744BF2B228DF853202A782A2AC2
:10ACC0002AD0079AA84600200A25414611F8013BE0
:10ACD000303B092B69D960B324E0504B9C4201D131
:10ACE000B468A3E74E4B9C4208BFF4689EE7214638
:10ACF000304600F025FC00289ED04FF0FF301DB0FC
:10AD0000BDE8F08FA846A2E7434A801A0BFA00F08C
:10AD1000184304904546BEE7039A111D126803913B
:10AD2000002A01DB079204E0524243F0020307923B
:10AD3000049398F800302E2B0ED198F801302A2B6E
:10AD400038D1039B1A1D1B680392002BB8BF4FF02C
:10AD5000FF3308F102080593324D98F800100322E2
:10AD6000284600F065FE40B14023401B03FA00F086
:10AD7000049B034308F10108049398F800102A4843
:10AD80008DF82810062208F1010700F051FE002876
:10AD900037D0264B1BBB039B073323F00703083335
:10ADA0000393099B4B44099350E705FB02320120B2
:10ADB00088468AE7002308F10108059319460A2509
:10ADC000404610F8012B303A092A03D9002BC3D092
:10ADD0000591C1E705FB012101238046F0E703ABA4
:10ADE00000932246124B04A93046AFF30080B0F125
:10ADF000FF3F8146D5D1A3895B063FF57EAF099819
:10AE00007DE703AB00932246094B04A9304600F0CE
:10AE100087F8ECE774DB000020DB000094DB000027
:10AE200054DB000026DB00002ADB000000000000ED
:10AE3000E7AB00002DE9F04791461F468A680B6991
:10AE4000DDF820809342B8BF1346C9F8003091F86E
:10AE5000432006460C4612B10133C9F8003023687E
:10AE6000990642BFD9F800300233C9F8003025688E
:10AE700015F0060507D104F1190AE368D9F8002096
:10AE80009B1AAB4228DC94F843302268003318BF89
:10AE9000012392062DD404F1430239463046C047BF
:10AEA000013020D02368E568D9F8002003F00603BC
:10AEB000042B08BFAD1AA36822690CBF25EAE5750B
:10AEC00000259342C4BF9B1AED184FF000091A34B5
:10AED0004D451AD1002008E001235246394630463C
:10AEE000C047013003D14FF0FF30BDE8F087013596
:10AEF000C3E7E1185A1C302081F84300224494F83B
:10AF0000451082F843100233C5E701232246394633
:10AF10003046C0470130E6D009F10109D8E700000A
:10AF20002DE9F04301F1430C0C46097E85B06E29F2
:10AF30001746064698460C9A00F0B38022D863293B
:10AF400036D00AD8002900F0B980582900F0838053
:10AF500004F1420584F8421032E0642901D06929E5
:10AF6000F6D120681368050603F104012AD51B6891
:10AF70001160002B03DA2D225B4284F843206F48D6
:10AF80000A2239E0732900F09D8008D86F2920D06B
:10AF90007029DDD1236843F02003236003E0752985
:10AFA00017D07829D4D1782384F84530644855E007
:10AFB0001368191D1B68116004F1420584F84230C2
:10AFC00001238CE01B68116010F0400F18BF1BB20A
:10AFD000CFE713682568181D1060280601D51B6887
:10AFE00002E06806FBD51B8854486F2914BF0A226B
:10AFF0000822002184F843106568A560002DC0F286
:10B000009580216821F004012160002B3DD1002DA5
:10B0100040F08E806546082A0BD12368DB0708D5EF
:10B02000236962689A42DEBF302305F8013C05F1CE
:10B03000FF35ACEB05032361CDF800803B4603AA46
:10B0400021463046FFF7F6FE01304DD14FF0FF307C
:10B0500005B0BDE8F083394884F8451013682168CD
:10B060001D1D1B6815600A060BD5CA0744BF41F0B9
:10B07000200121601BB9226822F0200222601022E8
:10B08000B7E74D0648BF9BB2EFE76546B3FBF2F169
:10B0900002FB1133C35C05F8013D0B460029F5D1D5
:10B0A000B9E7136825686169181D106028061B68D8
:10B0B00001D5196002E06A06FBD5198000232361DF
:10B0C0006546B9E71368191D11601D6862680021A3
:10B0D000284600F0ADFC08B1401B60606368236146
:10B0E000002384F84330A7E723692A4639463046CF
:10B0F000C0470130AAD023689B0713D4E068039BA4
:10B100009842B8BF1846A3E701234A46394630465D
:10B11000C04701309AD00135E368039A9B1AAB42CD
:10B12000F2DCEBE7002504F11909F5E7002BACD1BF
:10B13000037884F8423004F142056CE731DB00000B
:10B1400042DB000038B50D4B1C68A36B05467BB98C
:10B15000182000F04DFC0A4A0A4BA063C0E9002306
:10B16000094B83600B23838101220023C0E9042360
:10B17000A36B00221D615A6138BD00BF6000002032
:10B180000E33CDAB34126DE6ECDE050038B5134B53
:10B190001C68A36B7BB9182000F02AFC104A114BE5
:10B1A000A063C0E90023104B83600B23838101223D
:10B1B0000023C0E90423A16B0C480A694B690C4CBD
:10B1C000504304FB0300A2FB04230344541C43F13B
:10B1D0000005C1E9044525F0004038BD60000020AD
:10B1E0000E33CDAB34126DE6ECDE05002DF4515874
:10B1F0002D7F954C0CB430B5174B0C1E9DB01D68BF
:10B2000008DA8B232B604FF0FF301DB0BDE83040D3
:10B2100002B070474FF40273ADF8143014BF04F15C
:10B22000FF332346049307934FF6FF730290069073
:10B23000ADF81630209A21AB02A92846019300F000
:10B240006FFD431CBCBF8B232B60002CDDD0029B09
:10B2500000221A70D9E700BF600000200EB400B5CC
:10B260009CB01DAB029006906FF000410948079119
:10B270000491094953F8042B05910068019302A930
:10B2800000F04EFD029B00221A701CB05DF804EB2A
:10B2900003B07047600000200802FFFF10B50346AE
:10B2A0001A785C1C3AB9013B11F8012B03F8012F05
:10B2B000002AF9D110BD2346F2E7C9B2034610F8BF
:10B2C000012B1AB18A42F9D118467047002918BFDC
:10B2D0000023F9E710F8012B11F8013B012A28BFE0
:10B2E0009A42F7D0D01A7047034613F8012B002A70
:10B2F000FBD1181A0138704710B56AB101398418AA
:10B3000010F8013B11F8012F934203D1A04201D064
:10B31000002BF5D1981A10BD1046FCE770B5013925
:10B32000044602B970BD234611F8015F03F8015BC2
:10B33000561E2DB91444A342F4D003F8015BFAE77A
:10B340001C463246EDE7F0B503787BB1044623781E
:10B350002046661C7BB14A1E631E12F8015F4DB188
:10B3600013F8017FAF423446F7D0F0E70B78002B9B
:10B3700018BF0020F0BD1846FCE72DE9F0478046D5
:10B38000894692461E460F463D46089815F8014BE1
:10B3900000F0C6FA2044437813F0080332D12D2C74
:10B3A00032D17C78BD1C0122002E5DD0102E09D137
:10B3B000302C07D12B7803F0DF03582B4FD16C785A
:10B3C00010260235002A14BF4FF000416FF00041F3
:10B3D0000027B1FBF6FC384606FB1C1EA4F1300327
:10B3E000092B17D81C46A64223DD7B1C07D08445B9
:10B3F0001CD301D1A64519DB00FB0640012715F837
:10B40000014BEBE72F46BFE72B2C04BFBD1C7C781C
:10B410001A46C9E7A4F14103192B01D8373CE2E7EA
:10B42000A4F16103192B04D8573CDCE74FF0FF3738
:10B43000E5E77B1C08D12223C8F800300846BAF1A2
:10B44000000F07D1BDE8F08702B14042BAF1000F0A
:10B45000F8D00FB105F1FF39CAF80090F2E73024B7
:10B46000002EAFD10826ADE7302CA3D00A26A9E7DD
:10B47000084B37B51C68084D236A002B08BF2B46C4
:10B48000009313460A4601462046FFF776FF03B0B5
:10B4900030BD00BF60000020C4000020F8B50E469B
:10B4A0001446054618B183690BB900F0AFF9214B7A
:10B4B0009C422AD16C68A369A360A3891A072ED580
:10B4C000236963B323692068C01A6369F6B28342B3
:10B4D000374604DC2146284600F02EF928BBA36835
:10B4E000013BA36023685A1C22601E70636901300F
:10B4F000834204D0A389DB0719D50A2E17D1214630
:10B50000284600F019F990B10FE00B4B9C4201D195
:10B51000AC68D0E7094B9C4208BFEC68CBE72146FA
:10B52000284600F00DF80028CCD04FF0FF37384601
:10B53000F8BD00BF74DB000094DB000054DB0000AA
:10B54000324B70B51D6806460C4625B1AB6913B980
:10B55000284600F05BF92E4B9C420FD16C68B4F981
:10B560000C309AB215072CD4D00611D409223260BF
:10B5700043F04003A3814FF0FF303EE0254B9C4257
:10B5800001D1AC68EBE7244B9C4208BFEC68E6E7CE
:10B59000510712D5616B41B104F14403994202D0C5
:10B5A000304600F095FA00236363A38923F0240357
:10B5B000A3810023636023692360A38943F0080308
:10B5C000A38123694BB9A38903F42073B3F5007FEA
:10B5D00003D02146304600F0CBF9A28912F00103D6
:10B5E0000CD00023A36063695B42A361236953B954
:10B5F000B4F90C3013F08000BAD170BD920758BF77
:10B600006369A360F2E70020F7E700BF6000002055
:10B6100074DB000094DB000054DB000008B506205A
:10B6200000F0ACFC012000F0D5FD00008A892DE976
:10B63000F041054610070C4658D44B68002B05DC3A
:10B640000B6C002B02DC0020BDE8F081E66A002EC6
:10B65000F9D0002312F480522F68216A2B6032D077
:10B66000606DA3895A0705D56368C01A636B0BB177
:10B67000236CC01A00230246E66A216A2846B047B6
:10B68000431CA38906D129681D2948D8294ACA40E4
:10B69000D60744D500226260D9042269226004D50D
:10B6A000421C01D12B6803B96065616B2F600029D2
:10B6B000C9D004F14403994202D0284600F008FAA8
:10B6C00000206063C0E701232846B047411CC8D171
:10B6D0002B68002BC5D01D2B01D0162B01D12F605C
:10B6E000B1E7A38943F04003A381ADE70F69002FC1
:10B6F000A9D093070E6808BF4B690F6018BF0023DD
:10B70000A6EB07088B60B8F1000F9CDD43463A4674
:10B71000216AA66A2846B047002806DCA38943F0C0
:10B720004003A3814FF0FF308EE70744A8EB0008E9
:10B73000E9E700BF0100402038B50B6905460C461B
:10B74000DBB118B183690BB900F060F80C4B9C4277
:10B7500009D16C68B4F90C307BB121462846BDE8AC
:10B760003840FFF763BF074B9C4201D1AC68F1E75B
:10B77000054B9C4208BFEC68ECE7002038BD00BFD9
:10B7800074DB000094DB000054DB0000002310B5E4
:10B790000446C0E90033836081814366C281C0E909
:10B7A00004338361194608225C30FFF7FDF9054B2D
:10B7B0006362054BA362054BE362054B246223637E
:10B7C00010BD00BFB5BF0000D7BF00000FC0000014
:10B7D00033C00000014900F085B800BF39B7000050
:10B7E00070B54A1E682555430E4605F1740100F0F8
:10B7F000BDF9044640B10021C0E900160C30A0603C
:10B8000005F16802FFF7D0F9204670BD836910B5D5
:10B81000044633BBC0E912330365124B124A1B685E
:10B820008262984204BF0123836100F01FF86060C8
:10B83000204600F01BF8A060204600F017F8002218
:10B84000E06004216068FFF7A1FF01220921A068E0
:10B85000FFF79CFF02221221E068FFF797FF012308
:10B86000A36110BD1CDB0000D5B70000F8B51B4B71
:10B870001E68B369074613B93046FFF7C7FF48365D
:10B88000D6E90134013B03D5336833B13668F7E7B5
:10B89000B4F90C506DB16834F4E704213846FFF771
:10B8A0009FFF30600028F1D10C233B600446204606
:10B8B000F8BD0B4B6566C4E90055A560C4E90335C6
:10B8C000C4E905550822294604F15C00FFF76CF92C
:10B8D000C4E90D55C4E91255E9E700BF1CDB0000BF
:10B8E0000100FFFF2DE9F8438046894600F1480436
:10B8F000002614B93046BDE8F883D4E90175013F4C
:10B9000001D52468F5E7AB89012B07D9B5F90E30CD
:10B91000013303D029464046C84706436835EEE761
:10B92000D0F8EC00704770B50E46B1F90E10002942
:10B9300096B014461D4607DA00232B60B3891A0619
:10B9400010D44FF480630EE06A4600F0A5FB002897
:10B95000F2DB019A02F47042A2F500535A425A41B6
:10B960002A60EEE740230020236016B070BD00007F
:10B970008B8973B59D0706460C4607D504F147032E
:10B98000236023610123636102B070BD01AB6A468D
:10B99000FFF7C9FF00990546304600F0E7F848B9BF
:10B9A000B4F90C309A05EFD423F0030343F00203FB
:10B9B000A381E3E70D4BB362A389206043F08003CA
:10B9C000A381009B6361019B20615BB1B4F90E1000
:10B9D000304600F073FB28B1A38923F0030343F042
:10B9E0000103A381A3891D43A581CDE7D5B700003D
:10B9F000024B0146186800F0B9B800BF6000002093
:10BA000082B001B901A942B14BB113780B60127831
:10BA1000101C18BF012002B070471046FBE76FF002
:10BA20000100F8E700000000000000000000000036
:10BA300001F0FF01102A2BDB10F0070F08D010F8DF
:10BA4000013B013A8B422DD010F0070F42B3F6D1E3
:10BA5000F0B441EA012141EA014122F007047FF0FC
:10BA600000070023F0E80256083C85EA010586EA53
:10BA7000010685FA47F5A3FA87F586FA47F6A5FA8F
:10BA800087F68EB9EED1F0BC01F0FF0102F007029B
:10BA900032B110F8013B013A83EA010313B1F8D146
:10BAA0000020704701387047002D06BF3546033827
:10BAB000073815F0010F07D1013015F4807F02BF60
:10BAC000013015F4C03F0130F0BC0138704700BFB1
:10BAD00038B50546002945D051F8043C0C1F002B11
:10BAE000B8BFE41800F00CFB1F4A1368104633B9C6
:10BAF000636014602846BDE8384000F002BBA342F2
:10BB00000CD921686218934204BF1A685B686360AD
:10BB100004BF521822600460ECE713465A680AB169
:10BB2000A242FAD919685818A0420BD120680144E2
:10BB3000581882421960DDD1106852685A60014479
:10BB40001960D7E702D90C232B60D3E720682118AE
:10BB50008A4204BF11685268626004BF09182160FC
:10BB60005C60C7E738BD00BFFC7C012070B5CD1C10
:10BB700025F0030508350C2D38BF0C25002D064691
:10BB800001DBA94203D90C233360002070BD00F013
:10BB9000B7FA214A1468214691B9204C23681BB991
:10BBA000304600F0B3F920602946304600F0AEF987
:10BBB000431C24D10C233360304600F0A2FAE4E7A2
:10BBC0000B685B1B18D40B2B0FD90B60CD50CC1816
:10BBD000304600F096FA04F10B00231D20F0070018
:10BBE000C31AD3D05A42E250D0E78C424B6816BFFA
:10BBF000636013600C46EBE70C464968CCE7C41C55
:10BC000024F00304A04205D0211A304600F07EF94A
:10BC10000130CFD02560DBE7FC7C0120007D0120D6
:10BC2000F8B5074614460E4621B91146BDE8F8405E
:10BC3000FFF79CBF22B9FFF74BFF25462846F8BD0A
:10BC400000F060FAA0420FD221463846FFF78EFF7F
:10BC500005460028F2D031462246FEF781FF3146E4
:10BC60003846FFF735FFE9E73546E7E72DE9F047C6
:10BC70008E689E4282460C469046994637D88A89FD
:10BC800012F4906F31D0256809696F1A6569022333
:10BC900005EB450595FBF3F509F101033B449D4296
:10BCA00038BF1D46530530D52946FFF75FFF0646CE
:10BCB00050B90C23CAF80030A38943F04003A38194
:10BCC0004FF0FF30BDE8F0873A462169FEF748FFA4
:10BCD000A38923F4906343F08003A3812661656107
:10BCE0003E44ED1B2660A5604E464E4500D94E46AB
:10BCF000324641462068FEF73EFFA3689B1BA360C7
:10BD000023681E4426600020DCE72A46FFF788FFF0
:10BD100006460028E2D121695046FFF7D9FEC8E760
:10BD20002DE9F04F9DB0804603938B891D060C468C
:10BD300016460FD50B696BB94021FFF717FF20603E
:10BD4000206128B90C23C8F800304FF0FF30C7E05D
:10BD5000402363610023099320238DF82930302389
:10BD60008DF82A304FF0010B37463D4615F8013B60
:10BD70000BB1252B3ED1B7EB060A0BD0534632460A
:10BD800021464046FFF772FF013000F0A480099B76
:10BD9000534409933B78002B00F09D8000234FF023
:10BDA000FF32CDE90523049307938DF853301A939E
:10BDB0002F46052217F8011B4F48FFF739FE049B59
:10BDC000D0B9D90644BF20228DF853201A0744BFAA
:10BDD0002B228DF853202A782A2A15D0079A2F462D
:10BDE00000200A25394611F8013B303B092B4DD97B
:10BDF000B8B10FE02F46B8E73F4A801A0BFA00F0BF
:10BE0000184304903D46D3E7039A111D126803912D
:10BE1000002A01DB079204E0524243F0020307923A
:10BE200004933B782E2B0CD17B782A2B33D1039BA8
:10BE30001A1D1B680392002BB8BF4FF0FF33023767
:10BE400005932E4D397803222846FFF7F1FD38B1CE
:10BE50004023401B03FA00F0049B03430137049383
:10BE6000397827488DF8281006227E1CFFF7E0FD60
:10BE7000002838D0234B13BB039B073323F0070361
:10BE800008330393099B4B4409936DE705FB02328A
:10BE900001200F46A6E700230137059319460A251E
:10BEA000384610F8012B303A092A03D9002BC8D0A4
:10BEB0000591C6E705FB012101230746F0E703AB27
:10BEC00000932246104B04A94046AFF30080B0F126
:10BED000FF3F8146D6D1A3895B063FF536AF09986F
:10BEE0001DB0BDE8F08F03AB00932246064B04A9BA
:10BEF0004046FFF715F8EAE720DB000026DB0000EC
:10BF00002ADB0000000000006DBC000038B5064CC4
:10BF1000002305460846236000F046F9431C02D181
:10BF2000236803B12B6038BD909001201F2938B5DC
:10BF300004460D4604D9162303604FF0FF3038BD88
:10BF4000426C12B152F821304BB9204600F030F863
:10BF50002A4601462046BDE8384000F017B8012BBC
:10BF60000AD0591C03D1162303600120E7E70024FF
:10BF700042F82540284698470020E0E7024B01465A
:10BF80001868FFF7D3BF00BF6000002038B5074C2A
:10BF90000023054608461146236000F0EDF8431CD7
:10BFA00002D1236803B12B6038BD00BF90900120FF
:10BFB00000F0D2B810B50C46B1F90E1000F0AAF896
:10BFC0000028ABBF636DA3891B1823F48053ACBF5B
:10BFD0006365A38110BD2DE9F0411F468B89DB0508
:10BFE00005460C46164605D502230022B1F90E106F
:10BFF00000F074F8A389B4F90E1023F48053A381E0
:10C0000032463B462846BDE8F04100F023B810B563
:10C010000C46B1F90E1000F061F8431CA38915BF5E
:10C02000606523F4805343F48053A38118BFA38138
:10C0300010BDB1F90E1000F01FB849B1FF2A85BF3D
:10C040008A2303600A704FF0FF3098BF01207047C9
:10C050000846704738B5074C054608461146002289
:10C0600022601A4600F0AEF8431C02D1236803B1E7
:10C070002B6038BD9090012038B5064C0023054652
:10C080000846236000F058F8431C02D1236803B12E
:10C090002B6038BD9090012038B5074C0023054631
:10C0A00008461146236000F04FF8431C02D1236874
:10C0B00003B12B6038BD00BF9090012038B5064C0D
:10C0C000002305460846236000F04EF8431C02D1C9
:10C0D000236803B12B6038BD9090012038B5074C20
:10C0E000054608461146002222601A4600F04CF828
:10C0F000431C02D1236803B12B6038BD909001200E
:10C100007047704751F8043C181F002BBCBF0B58F8
:10C11000C018704738B5074C05460846114600223E
:10C1200022601A4600F038F8431C02D1236803B19C
:10C130002B6038BD90900120024B58221A604FF0BE
:10C14000FF30704790900120024B58221A604FF048
:10C15000FF30704790900120024B58221A604FF038
:10C16000FF30704790900120024B58221A60002047
:10C17000704700BF90900120024B58221A604FF088
:10C18000FF30704790900120024B58221A604FF008
:10C19000FF30704790900120024B58221A604FF0F8
:10C1A000FF30704790900120044A05491368002B26
:10C1B00008BF0B461844106018467047047D0120E4
:10C1C00098900120024B58221A604FF0FF307047C0
:10C1D00090900120FEE700BFF8B500BFF8BC08BC96
:10C1E0009E467047F8B500BFF8BC08BC9E46704735
:10C1F000646174610000000086C200001D0300003D
:10C200008FC200000D04000097C20000E10B000087
:10C210009EC200000D0D0000A3C200001906000020
:10C22000A9C20000F1070000B4C2000077040000BA
:10C23000B9C20000490F0000C5C200004F03000052
:10C24000CFC20000B90A0000DDC20000950700005F
:10C25000EAC200007D090000F6C200005D07000090
:10C2600072616E646F6D00616C6C006C6173740060
:10C27000300066616C7365007472756500252E313F
:10C2800035732E2E2E006D616B654C6973740061E1
:10C2900064644C6173740064656C657465006A6FF6
:10C2A000696E0073706C697400636F707946726FA9
:10C2B0006D546F0066696E64006A6F696E537472C4
:10C2C000696E677300756E69636F646541740075AC
:10C2D0006E69636F6465537472696E67006E65772B
:10C2E0004279746541727261790061734279746553
:10C2F000417272617900667265654D656D6F727924
:10C300000000000069C30000291400006EC3000093
:10C310004314000097C200004714000074C30000DB
:10C320002D1400007EC300004B14000087C30000E2
:10C330004F14000091C30000531400009CC3000080
:10C3400057140000A8C3000031140000B1C300005E
:10C350003B140000BBC3000035140000C6C300003E
:10C360003F14000066696C65006F70656E00636C59
:10C370006F736500656E644F6646696C6500726533
:10C3800061644C696E6500726561644279746573BD
:10C3900000617070656E644C696E650061707065F7
:10C3A0006E6442797465730066696C6553697A6579
:10C3B0000073746172744C697374006E65787449AB
:10C3C0006E4C6973740073797374656D496E666F32
:10C3D0000000000018180000281800003C18000099
:10C3E000B0180000E2180000121900004419000003
:10C3F00066190000A6190000E0190000301A0000BC
:10C400006E1A0000CE1A00000E1B00002E1B00004A
:10C41000621B0000A21B0000C41B0000EE1B0000FA
:10C42000181C0000C6310000C41C00008C1D000058
:10C43000FE1D0000481E0000AC1E0000C81E0000CB
:10C44000E61E00002420000064200000D62000002A
:10C45000042100003421000062210000C6210000F8
:10C460002A2200008C220000EE220000622300003D
:10C47000DC2300003C2400009C240000D2240000A7
:10C48000162500005C250000A2250000F425000010
:10C490004A26000088260000FC2600003027000005
:10C4A00076270000BC270000022800003C2800007E
:10C4B00082280000C8280000242A0000EE1B00008B
:10C4C000621B00003C2900001818000070290000C1
:10C4D00096290000CA290000F02900001818000061
:10C4E0001818000018180000181800009A2A0000F8
:10C4F000D62A0000162B0000662B00008C2B0000B3
:10C50000FA2B0000442C0000742C000018180000C6
:10C5100018180000922C0000C42C0000F62C00001B
:10C520002A2D00004E2D0000AC2D0000D02D000063
:10C53000F22D0000142E0000462E0000782E000080
:10C540009C2E0000C02E0000F22E0000162F0000CE
:10C55000181800001818000018180000181800001B
:10C5600018180000482F00006E2F0000942F0000C4
:10C57000BA2F0000E02F0000143000004830000007
:10C580007C300000B0300000D6300000FC300000ED
:10C5900030310000181800001818000018180000AA
:10C5A00018180000181800001818000018180000CB
:10C5B00018180000181800001818000018180000BB
:10C5C0001818000056310000563100007832000083
:10C5D000A83200005B2564206974656D206C697366
:10C5E000745D002825642062797465732900286FC2
:10C5F000626A65637420747970653A202564290045
:10C60000537461636B20756E646572666C6F77003E
:10C61000626F6F6C65616E006E756D62657200733E
:10C620007472696E67006C69737400627974652056
:10C6300061727261790000000700000003000000D1
:10C64000C9C60000C5330000D1C600007134000027
:10C65000DAC6000079360000E3C60000C9330000E6
:10C66000ECC600007D360000F4C600000536000070
:10C67000FDC600005135000008C70000ED3700007E
:10C6800013C70000153600001EC70000B1370000B8
:10C690002AC70000FD34000036C70000073900003B
:10C6A0000000000001000000020000000300000084
:10C6B000040000000A0000001D0000006D696372A4
:10C6C0006F3A62697420763200686173546F6E65E8
:10C6D00000706C6179546F6E6500686173536572A8
:10C6E000766F00736574536572766F006461634999
:10C6F0006E69740064616357726974650073717563
:10C700006172655761766500736574557365724C27
:10C71000454400616E616C6F675265616400616ED3
:10C72000616C6F67577269746500646967697461E9
:10C730006C52656164006469676974616C57726901
:10C74000746500474320746F6F6B202564207573F8
:10C750006563733B206672656520256420776F7280
:10C760006473003C496E74656765723E003C4C69B9
:10C7700073743E003C4F626A6563743E003C4279CC
:10C78000746541727261793E000D0A564D20506108
:10C790006E69633A2025730D0A006D6973630000AA
:10C7A000D5C70000A9430000DEC700002D430000EC
:10C7B000E2C7000079420000EAC700001B42000007
:10C7C000F4C70000AD41000000C80000AF40000009
:10C7D0006E756C6C00686578546F496E740073698F
:10C7E0006E006A736F6E476574006A736F6E436F95
:10C7F000756E74006A736F6E56616C756541740076
:10C800006A736F6E4B65794174000000D0C80000F8
:10C8100009440000D8C800000D440000E2C8000030
:10C820001F440000EBC8000025440000F6C80000CB
:10C830002B44000002C900003144000010C9000070
:10C840003744000018C900003D4400001EC9000024
:10C850004344000033C900004944000048C90000B7
:10C860004F44000054C900005544000064C9000052
:10C870005B44000070C90000614400007DC90000F5
:10C88000674400008CC900006D4400009FC900008F
:10C8900073440000B5C9000079440000C1C900001C
:10C8A0007F440000D1C9000085440000E0C90000B9
:10C8B0008B440000EEC9000091440000F6C900005E
:10C8C00013440000FEC90000194400006E657400A6
:10C8D0006861735769466900737461727457694679
:10C8E000690073746F7057694669007769666953A8
:10C8F0007461747573006D79495041646472657335
:10C9000073007374617274535349447363616E00AE
:10C9100067657453534944006D794D414300687411
:10C92000747053657276657247657452657175658A
:10C93000737400726573706F6E64546F48747470B2
:10C94000526571756573740068747470436F6E6EB0
:10C9500065637400687474704973436F6E6E6563C9
:10C9600074656400687474705265717565737400E1
:10C9700068747470526573706F6E7365007765626A
:10C98000536F636B6574537461727400776562539F
:10C990006F636B65744C6173744576656E74007774
:10C9A0006562536F636B657453656E64546F436C5B
:10C9B00069656E74004D515454436F6E6E656374B7
:10C9C000004D5154544973436F6E6E6563746564D2
:10C9D000004D515454446973636F6E6E6563740007
:10C9E0004D5154544C6173744576656E74004D51CD
:10C9F0005454507562004D515454537562004D515A
:10CA00005454556E7375620004000000030000006A
:10CA10000A000000070000000600000000000000FF
:10CA20000008080800080A4A4000000A5FEA5FEAB6
:10CA30000ED92ED36E19324489330C924C924D0884
:10CA40000800000004880808040804848488000A98
:10CA5000448A4000048EC480000000048800000E58
:10CA6000C000000000080001224488100C925252BD
:10CA70004C048C84848E1C824C901E1EC244924CAA
:10CA800006CA525FE21FF01EC13E02448ED12E1F25
:10CA9000E24488100ED12ED12E0ED12EC48800086B
:10CAA00000080000048004880244880482000EC04C
:10CAB0000EC008048244880ED126C0040ED135B3BE
:10CAC0006C0C925ED2521C925C925C0ED010100ED6
:10CAD0001C9252525C1ED01C901E1ED01C90100E38
:10CAE000D013712E12525ED2521C8808081C1FE20D
:10CAF00042524C1254981492101010101E113B7593
:10CB0000B131113935B3710C9252524C1C925C9078
:10CB1000100C92524C861C925C92510ED00C825C8E
:10CB20001FE4848484125252524C1131312A441130
:10CB30003135BB7112524C9252112A4484841EC466
:10CB400088101E0EC808080E10080482410EC2424A
:10CB5000424E048A400000000000001F08048000CC
:10CB600000000ED2524F10101C925C000ED0100E1E
:10CB700002424ED24E0C925C900E06C81C88080EE3
:10CB8000D24EC24C10101C925208000808080240F5
:10CB900002424C10149814920808080806001B75ED
:10CBA000B131001C925252000C92524C001C925C0B
:10CBB00090000ED24EC2000ED010100006C804988D
:10CBC00008080EC807001252524F0011312A4400C3
:10CBD000113135BB00124C8C9200112A4498001E72
:10CBE000C4881E06C48C8486080808080818080C27
:10CBF000881800000C8360000000000001000000A5
:10CC00000200000003000000040000000500000016
:10CC100006000000070000000800000009000000F6
:10CC20000A0000000B0000000C0000000D000000D6
:10CC30000E0000000F0000001000000012000000B5
:10CC40001400000016000000180000001A00000088
:10CC50001C0000001E000000200000002300000057
:10CC600026000000290000002C0000002F0000001A
:10CC700032000000360000003A0000003E000000D4
:10CC800042000000460000004B0000005000000081
:10CC9000550000005A00000061000000680000001C
:10CCA0006F000000760000007D000000840000009E
:10CCB0008B0000009200000099000000A00000001E
:10CCC000A7000000AE000000B5000000BC0000009E
:10CCD000C3000000CA000000D1000000D80000001E
:10CCE000DF000000E6000000ED000000F40000009E
:10CCF000FB000000FF000000000000000200000038
:10CD000004000000010000000300000070CD0000DE
:10CD1000AD4400007BCD0000754A000085CD0000C9
:10CD20007546000092CD0000E947000099CD000053
:10CD300035480000A2CD000085480000AECD0000BF
:10CD400079470000BFCD00007D490000CCCD000038
:10CD50000147000015000000160000001700000049
:10CD60001800000019000000646973706C6179009C
:10CD70006C696768744C6576656C006D62446973B4
:10CD8000706C6179006D62446973706C61794F6693
:10CD900066006D62506C6F74006D62556E706C6FE2
:10CDA00074006D62447261775368617065006D62F2
:10CDB0005368617065466F724C6574746572006E7D
:10CDC000656F506978656C53656E64006E656F5071
:10CDD0006978656C53657450696E004E6F74206598
:10CDE0006E6F75676820726F6F6D206576656E2057
:10CDF000616674657220636F6D70616374696F6ED4
:10CE000000436F6D70616374656420466C61736884
:10CE100020636F64652073746F72650A25642062F5
:10CE20007974657320757365642028256425252928
:10CE3000206F6620256400426164207265636F7212
:10CE40006420666F756E6420647572696E67206910
:10CE50006E697469616C697A6174696F6E002564CA
:10CE60002025642025642028256420776F72647350
:10CE700029002564207265636F7264732C20256419
:10CE800020776F7264732C206D617849442025648B
:10CE90002C20636F6D70616374696F6E20637963BA
:10CEA0006C657320256400526573746F726564202D
:10CEB00025642073637269707473005374617274B3
:10CEC000656400726164696F000000005CCF00005F
:10CED0005D52000069CF0000D154000079CF0000FE
:10CEE0006554000087CF00003156000092CF00004B
:10CEF00085520000A2CF000015530000B6CF0000FD
:10CF0000F9520000C5CF00000D580000D1CF00003D
:10CF100089570000DACF00002D570000E5CF000050
:10CF20007D560000F0CF0000B5560000F9CF00009C
:10CF3000E556000002D000009552000011D000001C
:10CF4000755200001AD00000A55200006E6F6E6589
:10CF5000006F746865720070616972006469736162
:10CF6000626C65526164696F006D657373616765BA
:10CF70005265636569766564007061636B657452C0
:10CF8000656365697665007061636B657453656E92
:10CF900064007265636569766564496E746567658A
:10CFA000720072656365697665644D657373616768
:10CFB000655479706500726563656976656453745C
:10CFC00072696E670073656E64496E746567657239
:10CFD0000073656E64506169720073656E645374AA
:10CFE00072696E67007365744368616E6E656C008C
:10CFF00073657447726F757000736574506F7765F1
:10D0000072007369676E616C537472656E677468E1
:10D01000006465766963654944006C6173744D65AD
:10D020007373616765494400556E6B6E6F776E2050
:10D030007072696D6974697665205B25733A257332
:10D040005D00000000000000963007772C610EEEB6
:10D05000BA51099919C46D078FF46A7035A563E94F
:10D06000A395649E3288DB0EA4B8DC791EE9D5E076
:10D0700088D9D2972B4CB609BD7CB17E072DB8E775
:10D08000911DBF906410B71DF220B06A4871B9F3CA
:10D09000DE41BE847DD4DA1AEBE4DD6D51B5D4F403
:10D0A000C785D38356986C13C0A86B647AF962FD68
:10D0B000ECC9658A4F5C0114D96C0663633D0FFAB5
:10D0C000F50D088DC8206E3B5E10694CE44160D5BB
:10D0D000727167A2D1E4033C47D4044BFD850DD2A5
:10D0E0006BB50AA5FAA8B5356C98B242D6C9BBDBB8
:10D0F00040F9BCACE36CD832755CDF45CF0DD6DCB3
:10D10000593DD1ABAC30D9263A00DE518051D7C859
:10D110001661D0BFB5F4B42123C4B3569995BACFE4
:10D120000FA5BDB89EB802280888055FB2D90CC605
:10D1300024E90BB1877C6F2F114C6858AB1D61C17E
:10D140003D2D66B69041DC760671DB01BC20D2989D
:10D150002A10D5EF8985B1711FB5B606A5E4BF9F2A
:10D1600033D4B8E8A2C9077834F9000F8EA809961D
:10D1700018980EE1BB0D6A7F2D3D6D08976C649188
:10D18000015C63E6F4516B6B62616C1CD8306585A1
:10D190004E0062F2ED95066C7BA5011BC1F408827E
:10D1A00057C40FF5C6D9B06550E9B712EAB8BE8BBF
:10D1B0007C88B9FCDF1DDD62492DDA15F37CD38C48
:10D1C000654CD4FB5861B24DCE51B53A7400BCA346
:10D1D000E230BBD441A5DF4AD795D83D6DC4D1A478
:10D1E000FBF4D6D36AE96943FCD96E34468867AD4F
:10D1F000D0B860DA732D0444E51D03335F4C0AAAEE
:10D20000C97C0DDD3C710550AA41022710100BBEF0
:10D2100086200CC925B56857B3856F2009D466B937
:10D220009FE461CE0EF9DE5E98C9D9292298D0B06C
:10D23000B4A8D7C7173DB359810DB42E3B5CBDB719
:10D24000AD6CBAC02083B8EDB6B3BF9A0CE2B6039A
:10D250009AD2B1743947D5EAAF77D29D1526DB044F
:10D260008316DC73120B63E3843B64943E6A6D0D9A
:10D27000A85A6A7A0BCF0EE49DFF099327AE000AE5
:10D28000B19E077D44930FF0D2A3088768F2011E78
:10D29000FEC206695D5762F7CB67658071366C190F
:10D2A000E7066B6E761BD4FEE02BD3895A7ADA1030
:10D2B000CC4ADD676FDFB9F9F9EFBE8E43BEB71711
:10D2C000D58EB060E8A3D6D67E93D1A1C4C2D8389B
:10D2D00052F2DF4FF167BBD16757BCA6DD06B53F01
:10D2E0004B36B248DA2B0DD84C1B0AAFF64A033640
:10D2F000607A0441C3EF60DF55DF67A8EF8E6E31BF
:10D3000079BE69468CB361CB1A8366BCA0D26F2507
:10D3100036E2685295770CCC03470BBBB916022254
:10D320002F260555BE3BBAC5280BBDB2925AB42B69
:10D33000046AB35CA7FFD7C231CFD0B58B9ED92C7E
:10D340001DAEDE5BB0C2649B26F263EC9CA36A75E3
:10D350000A936D02A906099C3F360EEB856707729A
:10D3600013570005824ABF95147AB8E2AE2BB17B01
:10D37000381BB60C9B8ED2920DBED5E5B7EFDC7C88
:10D3800021DFDB0BD4D2D38642E2D4F1F8B3DD68DF
:10D390006E83DA1FCD16BE815B26B9F6E177B06FDA
:10D3A0007747B718E65A0888706A0FFFCA3B0666C7
:10D3B0005C0B0111FF9E658F69AE62F8D3FF6B6154
:10D3C00045CF6C1678E20AA0EED20DD75483044EF6
:10D3D000C2B30339612667A7F71660D04D47694984
:10D3E000DB776E3E4A6AD1AEDC5AD6D9660BDF4097
:10D3F000F03BD83753AEBCA9C59EBBDE7FCFB2474A
:10D40000E9FFB5301CF2BDBD8AC2BACA3093B3532E
:10D41000A6A3B4240536D0BA9306D7CD2957DE5437
:10D42000BF67D9232E7A66B3B84A61C4021B685D10
:10D43000942B6F2A37BE0BB4A18E0CC31BDF055A89
:10D440008DEF022D416C6C207461736B73207374CB
:10D450006F707065640076313432002025732025AA
:10D4600073004D656D6F727920636C6561726564E0
:10D47000004E6F2066726565207461736B20656E67
:10D48000747269657300000000D50000DD70000053
:10D490000DD50000F568000019D50000AD70000042
:10D4A0001FD50000BD70000025D50000CD70000024
:10D4B0002BD50000856F000041D50000D971000018
:10D4C0004FD500002569000059D5000069720000A1
:10D4D00061D50000596D00006AD50000256B000081
:10D4E00076D500002D6A00007FD50000756A000027
:10D4F00087D50000796C000073656E736F727300DE
:10D50000616363656C65726174696F6E0074656DEB
:10D5100070657261747572650074696C745800741A
:10D52000696C74590074696C745A00736574416352
:10D5300063656C65726F6D6574657252616E676567
:10D54000006D61676E657469634669656C6400743B
:10D550006F75636852656164006932635265616426
:10D560000069326357726974650073706945786346
:10D5700068616E67650073706953657475700072D9
:10D58000656164444854006D6963726F70686F6EC2
:10D590006500000069C30000ED7400006EC3000068
:10D5A000E9750000CBD500000D760000D0D5000055
:10D5B00071740000D9D500008D760000DFD5000021
:10D5C0004573000073657269616C00726561640087
:10D5D00072656164496E746F007772697465007773
:10D5E00072697465427974657300000068D6000042
:10D5F0002977000076D600003977000083D6000036
:10D600002D7700008CD600003D77000096D60000F4
:10D61000417700009FD6000045770000A4D60000A7
:10D6200049770000A9D600004D770000B5D600006C
:10D6300051770000BCD6000055770000C5D6000029
:10D6400059770000CAD600005D770000D5D60000EB
:10D6500061770000DFD6000031770000E9D60000D6
:10D660003577000074667400656E61626C654469AC
:10D6700073706C6179007365744261636B6C696788
:10D6800068740067657457696474680067657448F6
:10D69000656967687400736574506978656C006CBF
:10D6A000696E65007265637400726F756E6465649F
:10D6B0005265637400636972636C650074726961BA
:10D6C0006E676C65007465787400746674546F7569
:10D6D0006368656400746674546F75636858007499
:10D6E0006674546F7563685900746674546F75631B
:10D6F00068507265737375726500766172730000AD
:10D7000020D70000C97B00002AD70000A97B0000B9
:10D7100033D70000857B00003FD70000157B000059
:10D72000766172457869737473007661724E616DCB
:10D730006564007365745661724E616D6564007650
:10D7400061724E616D65466F72496E64657800570F
:10D75000656C636F6D6520746F204D6963726F42F5
:10D760006C6F636B732100705F73706920213D20C3
:10D770004E554C4C002F686F6D652F6769742F2EC6
:10D78000706C6174666F726D696F2F7061636B612D
:10D790006765732F6672616D65776F726B2D61724D
:10D7A0006475696E6F6E6F726469636E7266352F31
:10D7B0006C69627261726965732F5350492F5350BF
:10D7C000492E63707000535049436C6173733A3A49
:10D7D000535049436C617373284E52465F5350490E
:10D7E0005F547970652A2C2075696E74385F742CCB
:10D7F0002075696E74385F742C2075696E74385F9B
:10D800007429000000000000000000009D7D000061
:10D81000557D00008B7D0000917D0000977D00000C
:10D82000897D0000020000000300000004000000E9
:10D830001F0000001C0000000E000000250000007A
:10D840000B0000000A000000090000001E0000009C
:10D85000170000000C000000110000000100000093
:10D860000D00000022000000FFFFFFFFFFFFFFFF91
:10D870001A00000020000000150000001600000043
:10D880000F0000001800000013000000240000003A
:10D89000000000001400000005000000100000005F
:10D8A0000800000019000000280000000600000029
:10D8B00000000000000000007F830000998A000043
:10D8C000F583000001840000FB8300007D830000DD
:10D8D00075830000098400009983000071830000B3
:10D8E00000C00140001002400020024000D0024071
:10D8F000000000000000304300000000000030C3C2
:10D900007371727400000000FB21F93FFB21094094
:10D910007CD91240FB2119407A6A1F407CD92240F1
:10D92000BBFD2540FB2129403A462C407A6A2F4016
:10D930005C4731407CD932409C6B3440BBFD354064
:10D94000DB8F3740FB2139401BB43A403A463C401C
:10D950005AD83D407A6A3F404C7E40405C47414047
:10D960006C1042407CD942408CA243409C6B4440A6
:10D97000AC344540BBFD4540CBC64640DB8F4740FD
:10D98000EB584840FB21494083F9A200444E6E0009
:10D99000FC291500D1572700DD34F50062DBC000FB
:10D9A0003C999500419043006351FE00BBDEAB0003
:10D9B000B761C5003A6E2400D24D42004906E0002E
:10D9C00009EA2E001C92D100EB1DFE0029B11C00BB
:10D9D000E83EA700F535820044BB2E009CE9840098
:10D9E000B4267000417E5F00D69139005383390020
:10D9F0009CF439008B5F840028F9BD00F81F3B00C0
:10DA0000DEFF97000F980500112FEF000A5A8B00D8
:10DA10006D1F6D00CF7E360009CB2700464FB70043
:10DA20009E663F002DEA5F00BA277500E5EBC70050
:10DA30003D7BF100F739070092528A00FB6BEA0048
:10DA40001FB15F00085D8D00300356007BFC46006F
:10DA5000F0AB6B0020BCCF0036F49A00E3A91D00A8
:10DA60005E619100081BE60085996500A0145F00C7
:10DA70008D40680080D8FF0027734D0006063100F6
:10DA8000CA561500C9A873007BE260006B8CC00009
:10DA900000000040FB21F93F000000002D44743ECF
:10DAA000000000809846F83C0000006051CC783BB4
:10DAB00000000080831BF0390000004020257A38E8
:10DAC000000000802282E336000000001DF369356B
:10DAD0000200000003000000040000000600000037
:10DAE0002C2066756E6374696F6E3A2000617373E3
:10DAF000657274696F6E2022257322206661696CDD
:10DB000065643A2066696C6520222573222C206C9E
:10DB1000696E65202564257325730A006400002062
:10DB2000232D302B2000686C4C0065666745464706
:10DB30000030313233343536373839414243444589
:10DB400046003031323334353637383961626364F8
:10DB500065660000000000000000000000000000FA
:10DB600000000000000000000000000000000000B5
:10DB700000000000000000000000000000000000A5
:10DB80000000000000000000000000000000000095
:10DB90000000000000000000000000000000000085
:10DBA0000000000000000000000000000000000075
:10DBB00000000000504F5349580000202020202032
:10DBC000202020202828282828202020202020202D
:10DBD000202020202020202020202088101010101D
:10DBE0001010101010101010101010040404040471
:10DBF000040404040410101010101010414141419D
:10DC00004141010101010101010101010101010184
:10DC10000101010101011010101010104242424296
:10DC20004242020202020202020202020202020254
:10DC30000202020202021010101020000000000078
:10DC400000000000000000000000000000000000D4
:10DC500000000000000000000000000000000000C4
:10DC600000000000000000000000000000000000B4
:10DC700000000000000000000000000000000000A4
:10DC80000000000000000000000000000000000094
:10DC90000000000000000000000000000000000084
:10DCA0000000000000000000000000000000000074
:10DCB0000000000000000000000000000000000064
:08DCC0008025FF7F0100000038
:10DCC800FFFFFFFFE803000001000000E803DC0598
:10DCD800DC05DC05DC050000FFFFFFFFFFFFFFFFA1
:10DCE8001800000019FCFFFFFFFFFFFF0200000003
:10DCF80040420F00FFFF01FF030000000090D00327
:10DD0800FFFFFFFFFFFFFFFFFFFFFFFFFFFFFFFF1B
:10DD18000A000000010000000800000001000000E7
:10DD2800640000200000000074DB000094DB0000A9
:10DD380054DB0000000000000000000000000000AC
:10DD480000000000000000000000000000000000CB
:10DD580000000000000000000000000000000000BB
:10DD680000000000000000000000000000000000AB
:10DD7800000000000000000000000000000000009B
:10DD88000000000043000000000000000000000048
:10DD9800000000000000000000000000000000007B
:10DDA8000000000043000000000000000000000028
:10DDB800000000000000000000000000000000005B
:10DDC8000000000043000000000000000000000008
:10DDD800000000000000000000000000000000003B
:10DDE80000000000430000000000000000000000E8
:10DDF800000000000000000000000000000000001B
:10DE080000000000430000000000000000000000C7
:10DE180000000000000000000000000000000000FA
:10DE280000000000430000000000000000000000A7
:10DE380000000000000000000000000000000000DA
:10DE48000000000043000000000000000000000087
:10DE580000000000000000000000000000000000BA
:10DE6800000000003BC0000001BA000000000000F4
:10DE7800BADB000084C2000099C7000099C70000FF
:10DE880099C7000099C7000099C7000099C700000A
:10DE980099C7000099C7000099C70000FFFFFFFF5E
:10DEA800FFFFFFFFFFFFFFFFFFFF000001004153DF
:10DEB8004349490000000000000000000000000085
:10DEC80000000000000000000000000000004153B6
:10DED8004349490000000000000000000000000065
:10DEE800000000000000000000000000000000002A
:10DEF80025020000217D00007D81000009860000C8
:04DF08000102000012
:04000003000082393E
:00000001FF
